:020000040000FA
:1000000000EFF6F08FEF00F0E9CF0BF1EACF0CF143
:10001000D9CF0DF124EF19F0D8CF30F0E8CF31F07F
:10002000E0CF32F0E9CF33F0EACF34F0E1CF35F072
:10003000E2CF36F0D9CF37F0DACF38F0F3CF39F05E
:10004000F4CF3AF0F6CF3BF0F7CF3CF0F8CF3DF0ED
:10005000F5CF3EF09DA001D001D00AD09EA001D0E6
:1000600001D006D09FB001D001D002D0B2ECABF0ED
:10007000A0A201D001D00AD0A1A201D001D006D007
:10008000A2B201D001D002D0ADEC0AF09DA401D003
:1000900001D00AD09EA401D001D006D09FB401D0D7
:1000A00001D002D0B0EC38F09DAA01D001D00AD026
:1000B0009EAA01D001D006D09FBA01D001D002D0B3
:1000C00019ECEBF0A3AA01D001D00AD0A4AA01D068
:1000D00001D006D0A5BA01D001D002D0EDEC32F0AB
:1000E0003EC0F5FF3DC0F8FF3CC0F7FF3BC0F6FF48
:1000F0003AC0F4FF39C0F3FF38C0DAFF37C0D9FF88
:1001000036C0E2FF35C0E1FF34C0EAFF33C0E9FF8B
:1001100032C0E0FF31C0E8FF30C0D8FF100045EF2B
:1001200014F0FFFFFFFFFFFFFFFFFFFFFFFFFFFFD9
:10013000FFFFFFFFFFFFFFFFFFFFFFFFFFFFFFFFCF
:10014000FFFFFFFFFFFFFFFFFFFFFFFFFFFFFFFFBF
:10015000FFFFFFFFFFFFFFFFFFFFFFFFFFFFFFFFAF
:10016000FFFFFFFFFFFFFFFFFFFFFFFFFFFFFFFF9F
:100400001F1F1F1B1B1B1B1B13131313131319116C
:10041000130919191919191919191B1D1919190075
:100420000005310791073207920733079307340716
:1004300094073505950599073907360537053805B9
:1004400098050000960544070A0314000101020004
:100450000000EFFF009091A5FE123400000303009E
:1004600033CC123403010104000A0206010000002B
:100470000F02033C02020800000000000000000020
:10048000090909090911780585054005410588050F
:100490008907900770007105696E7465726E6574E6
:1004A0002E6C6D742E6C76000000000000000000C1
:1004B00000000031313131313131310000000000B4
:1004C00000000000000000003932330000323133F8
:1004D0002E32312E3139362E363800000047736DFA
:1004E00054736300000000000000000000000000E2
:1004F00000000000000000000000000000000000FC
:1005000000000000000000000000000000000000EB
:1005100000000000000000000000000000000000DB
:1005200000000000000000000000000000000000CB
:1005300000000000000000000000000000000000BB
:1005400000000000000000000000000000000000AB
:10055000000000000000000000000000000000009B
:10056000000000000000000000000000000000008B
:10057000000000000000000000000000000000007B
:10058000000000000000000000000000000000006B
:10059000000000000000000000000000000000005B
:1005A000000000000000000000000000000000004B
:1005B000000000000000000000000000000000003B
:1005C000000000000000000000000000000000002B
:1005D000000000000000000000000000000000001B
:1005E000000000000000000000000000000000000B
:1005F00000000000000000000000000000000000FB
:1006000000000000000000000000000000000000EA
:1006100000000000000000000000000000000000DA
:1006200000000000000000000000000000000000CA
:1006300000000000000000000000000000000000BA
:1006400000000000000000000000000000000000AA
:10065000000000000000000000000000000000009A
:10066000000000000000000000000000000000008A
:10067000000000000000000000000000000000007A
:10068000000000000000000000000000000000006A
:10069000000000000000000000000000000000005A
:1006A000000000000000000000000000000000004A
:1006B00000000000460545054205430501A0A1A232
:1006C000A3A4A5A6A7A8A9AAABACADAEAF01B0B133
:1006D000B2B3B4B5B6B7B8B9BABBBCBDBEBF01C042
:1006E000C1C2C3C4C5C6C7C8C9CACBCCCDCECFD082
:1006F000D1D2D3D4D5D6D7D8D9DADBDCDDDEDFE072
:10070000E1E2E3E4E5E6E7E8E9EAEBECEDEEEF0051
:1007100000000000000000000000000000000000D9
:10072000696E7465726E6574000000000000000060
:1007300000000000000000000000000000000000B9
:1007400000000000000000000000000000000000A9
:10075000033E033E033E033E033E00000000000054
:100760000000000000000000000000000000000089
:100770000000000000000000000000000000000079
:100780000000000000000000000000000000000069
:100790000000000000000000000000000000000059
:1007A0000000000000000000000000000000000049
:1007B0000000000000000000000000000000000039
:1007C0000000000000000000000000000000000029
:1007D0000000000000000000000000000000000019
:1007E0000000000000000000000000000000000009
:1007F00000000000000000000000000000000000F9
:10080000E8CF5AF1000114B202D0D890120005C509
:1008100015F101015A5131EC40F0F7E30501D351D4
:10082000070AF3E11F0ED325D96EDA6A050EDA2224
:10083000DF6A220E0101556F050E566F55C11BF17F
:1008400056C11CF1A2EC1AF01BC157F11CC158F1A2
:1008500057C11FF158C120F1AFEC3EF0D6E306BA04
:100860004ED0000115A82ED0068A078809900201F3
:10087000CA6B08BE8A9C468405012051300A10E1EB
:10088000020E0101166FFE0E156FE5EC19F0010165
:10089000186B540E176F3F0E196F50EC35F00FD0D8
:1008A000020E0101166FCC0E156FE5EC19F0010177
:1008B000186B540E176F1F0E196F50EC35F00001B6
:1008C000469410D080ECF5F001015A39F00B596FC5
:1008D000480E406F595188ECF0F00501055198EC35
:1008E00044F002E2D88012005A5169EC3DF0010157
:1008F000596F59C14EF15A5113ECE6F0F3D70A9CE7
:100900000A9A0B9409900201CA6B08BE8A9C069A47
:10091000468419A410D0020E0101166FDD0E156F6A
:10092000E5EC19F00101186B540E176F2F0E196FBB
:1009300050EC35F00FD0020E0101166FDD0E156F71
:10094000E5EC19F00101186B540E176F0F0E196FBB
:1009500050EC35F00798B3D72DC133F12EC134F1E7
:100960002E512D110AE12BC115F12CC116F1CFEC3E
:1009700036F015C133F116C134F133C115F134C16C
:1009800016F1F4EC24F015C135F116C136F120EE64
:1009900002F03551D9263651DA22DF505BEC43F0B4
:1009A000306F20EE03F03551D9263651DA22DF5070
:1009B0005BEC43F0316F20EE04F03551D92636510F
:1009C000DA22DF505BEC43F0326F09A409D0FA0E53
:1009D0000101176F1F0E166F010E4EEC32F008D09A
:1009E000FA0E0101176F140E166F010E4EEC32F065
:1009F00001013051CBEC42F001013151CBEC42F01E
:100A000001013251CBEC42F00D0ECBEC42F01BEC6D
:100A100045F00AD0EAEC44F007E317EC45F0010199
:100A20002F6F2F513E0A0DE0FFEC44F0890E0101BB
:100A3000295D130E2A59EEE31B0ECBEC42F0D89041
:100A400012002BC116F12CC117F1000E4EEC32F042
:100A50000301B26BB36B02941CD0C4ECE7F002A4A8
:100A600018D002940201CE6701D013D0080E010104
:100A70001C6FA00E1B6FFD0E1E6F6A0E1D6F206B8C
:100A8000070E1F6F47EC27F01C511B1102E1D880A5
:100A90001200310E0301B25D750EB359DEE31B0E79
:100AA000CBEC42F0CCD7E8CF1AF1C1C1FAF4C1299E
:100AB00065E1200E01011A25D96EDA6A0501050EDD
:100AC000DA22DF5027EC43F0186F1F0E01011A25C0
:100AD000D96EDA6A0501050EDA22DF5027EC43F001
:100AE0007BD8FA6F280E01011A25D96EDA6A050142
:100AF000050EDA22DF5027EC43F0186F270E0101B4
:100B00001A25D96EDA6A0501050EDA22DF5027ECC4
:100B100043F062D8FB6F2C0E01011A25D96EDA6AF8
:100B20000501050EDA22DF5027EC43F0186F290E7D
:100B300001011A25D96EDA6A0501050EDA22DF50A5
:100B400027EC43F049D8FC6F2E0E01011A25D96E0F
:100B5000DA6A0501050EDA22DF5027EC43F0186F40
:100B60002D0E01011A25D96EDA6A0501050EDA2269
:100B7000DF5027EC43F030D8FD6F28D0C10506E1E7
:100B80000401FB6BFC6BC4C1FDF420D0C151020A0F
:100B900003E0C151030A07E1C4C1FBF4C5C1FCF481
:100BA000C6C1FDF413D0C151060A03E0C151070AC2
:100BB0000DE1C4C1FBF4C6C118F10F0E1817C551E1
:100BC000F00B18110401FC6FC7C1FDF4040E010104
:100BD000176FFA0E166F1200196F193BF00E1917E6
:100BE00019511811040112000101476B03AA96D094
:100BF000039A880E0101296F130E2A6F2B6B2C6B41
:100C0000010E2D6FF2EC9FF001014B6F4B51370A33
:100C100003E04B510C0AEDE14B51370A70E106013C
:100C20009551220A6CE105011E6B01014B6B960E7A
:100C300001014B25D96EDA6A0601060EDA22220E70
:100C4000DF6201D016D0960E01014B25D96EDA6A0B
:100C5000060EDA220E0E4B25E16EE26A0501050E44
:100C6000E222DFCFE7FF1E2B01014B2B0F0E4B655E
:100C7000DED762ECE0F04A6F4A5141E0050E4A616E
:100C80003ED04A0504E1020E496F520E11D04A517E
:100C9000020A04E1020E496F630E0AD04A51030AA8
:100CA00004E1020E496F740E03D0020E496F850EE7
:100CB000486F0501D36B01014B6B1F0E01014B25E2
:100CC000D96EDA6A050EDA224B514825186F000EEC
:100CD0004921196F90EC2EF0DF6E1F0E01014B259C
:100CE000D96EDA6A0501050EDA22DF5006E0D32B51
:100CF00001014B2B100E4B65E0D74AC147F1FF0EA7
:100D00000101176FE40E166F010E4EEC32F0130E58
:100D100001012A6F880E296F2BEC37F00101475132
:100D2000120020EE04F01E51D9261F51DA2210EED7
:100D300006F01E51E1261F51E222DFCFE7FF20EE31
:100D400003F01E51D9261F51DA2210EE05F01E5174
:100D5000E1261F51E222DFCFE7FF20EE02F01E5115
:100D6000D9261F51DA2210EE04F069D810EE03F0F4
:100D700066D8D051DF6E20EE02F01E51D9261F51E9
:100D8000DA22CFC1DFFF20EE05F01E51D9261F5118
:100D9000DA22DF50216F206B226B0F0E2115236F9B
:100DA00020EE06F01E51D9261F51DA22DF50221103
:100DB000246F2351256F24C115F125C116F1F4ECE0
:100DC00024F015C126F116C127F120EE06F01E51C0
:100DD000D9261F51DA22DF6A20EE06F01E51D926ED
:100DE0001F51DA2210EE04F02651E1262751E222AB
:100DF000E750206F10EE03F02651E1262751E22242
:100E0000E750216F2139F00B2011DF6E20EE05F045
:100E10001E51D9261F51DA22F00EDF1620EE02F005
:100E20002651D9262751DA22DF50206F20EE05F017
:100E30001E51D9261F51DA222051DF1212001E51F5
:100E4000E1261F51E222DFCFE7FF20EE01F01E5125
:100E5000D9261F51DA221200E8CF37F1000111A480
:100E6000000C11A41200130E0101196F6A0E186F05
:100E700090EC2EF0386F3851800A500F04E338514F
:100E8000800A460F03E33751ADEC31F03DEC1FF023
:100E900004E33DEC1FF001E3020C0101386B280E66
:100EA00001013825D96EDA6A0601060EDA22DF5012
:100EB0006CE00101376733D0370E3825D96EDA6A16
:100EC000060EDA226A0E336F130E346F3351382553
:100ED000186F000E38BFFF0E3421196F90EC2EF002
:100EE000DF6E280E01013825D96EDA6A060EDA2285
:100EF000DF50336F346B33BF34076A0E356F130E18
:100F0000366F35513825186F000E38BFFF0E362169
:100F1000196F90EC2EF033193411BEE131D0370E39
:100F200001013825D96EDA6A060EDA22790E336F9E
:100F3000130E346F33513825186F000E38BFFF0E73
:100F40003421196F90EC2EF0DF6E280E0101382548
:100F5000D96EDA6A060EDA22DF50336F346B33BF94
:100F60003407790E356F130E366F35513825186FEB
:100F7000000E38BFFF0E3621196F90EC2EF0CBD744
:100F8000382B3851800A710F8AE3010C010E54ECA2
:100F9000D9F004E2010E54ECD9F014E3426B0AD00C
:100FA0003D6B6AD80E0E0101422583D850EC35F016
:100FB0000101422B6CD8F4E33D6B5ED8000E196B37
:100FC00050EC35F0020E54ECD9F004E2020E54EC71
:100FD000D9F016E3426B0BD0110E3D6F4DD80E0EBB
:100FE0000101422566D850EC35F00101422B4FD863
:100FF000F3E3110E3D6F40D8000E196B50EC35F045
:10100000030E54ECD9F004E2030E54ECD9F016E3CD
:10101000426B0BD0220E3D6F2FD80E0E01014225E0
:1010200048D850EC35F00101422B31D8F3E3220EC1
:101030003D6F22D8000E196B50EC35F0040E54ECC5
:10104000D9F005E2040E54ECD9F0D8A01200426B9E
:101050000BD0330E3D6F10D80E0E0101422529D85A
:1010600050EC35F00101422B12D8F3E3330E3D6F03
:1010700003D8196B50EF35F0010E3E6F3D514225FC
:10108000176F000E42BFFF0E3E21186F12001EC5E3
:101090003DF101013E6B42C13FF1406B3FBF400754
:1010A0004051800A416F3D513F5D3E51800A415998
:1010B0001200D96EDA6A050EDA22DF50196F1200BB
:1010C0008C0EF66EEB0EF76E000EF86E21EE2CF025
:1010D000060E0900F5CFDEFFE82EFBD7070E366FB0
:1010E00036C128F1F90E28272C0E2825D96EDA6A88
:1010F000010EDA22DF50296F73D8291902E0D89047
:101100001200362B0B0E3665EBD7030E2425286F05
:10111000000E2521296F28C11BF129C11CF1A2EC69
:101120001AF01BC134F11CC135F1326B336B070E61
:10113000366F0DD032C115F133C116F151D8176F8A
:1011400084EC3FF015C132F116C133F1362B070E96
:101150003425286F000E3521296F36C12AF12B6BFB
:1011600028512A5D29512B59E5E320EE02F0245144
:10117000D9262551DA22DF50286F296B28BF29078D
:1011800020EE01F02451D9262551DA22DF502B6FB1
:101190002A6B28512A11346F29512B11356F355183
:1011A000331902E134513219AAE10C0E2425286FBB
:1011B000000E2521296F28C11BF129C11CF1FCEC6F
:1011C00017F01BC134F11CC135F135510301B519BC
:1011D00004E1010134510301B41991E1D8801200F6
:1011E00036512425D96E000E2521DA6EDF5012000B
:1011F000E8CF3EF13F6B406B05010E512B0A15E124
:10120000010E0101406F11D00E0E01014025D96E73
:10121000DA6A050EDA22280E3F25E16EE26A010E37
:10122000E222DFCFE7FF402B3F2B05011E510101DA
:10123000405DEAE3280E3F25D96EDA6A010EDA2214
:10124000DF6A166F280E156FCFEC36F015513F6F21
:101250003FC11DF11E6B206B020E1F6F49EC3BF06E
:101260001DC13AF11EC13BF11FC13CF120C13DF14E
:101270003B51800A800F010ED8B43A5D0AE3010E9B
:10128000166F280E156FFB0E186FEB0E176F67ECBD
:101290003AF0406B2CD040C125F1252B280E252596
:1012A000D96EDA6A010EDA221F0E266F050E276F3D
:1012B00040512627000E27233E512625E16E000EC1
:1012C0002721E26EDFCFE7FF280E4025D96EDA6ACC
:1012D000010EDA2218D82527000E26232529E16ED3
:1012E000000E2621E26EDFCFE7FF020E40273F51BE
:1012F000405DD1E308D82525D96E000E2621DA6E8F
:10130000000EDF6E000C1F0E256F050E266F40517C
:101310002527000E26233E51120064502FE10401C0
:101320000031E8320F0B0D0A0FE104BF046B04011A
:10133000BF6B0401C06B0401C56BC46B6BEC26F082
:1013400041EC25F0C0EF23F00401C051020A44E152
:10135000070E0401CB6F040EC86F280EC76F040E72
:10136000CA6FCE0EC96F64EC3CF0010E0401D56F5C
:10137000040E0401036F200E026F12006450040A71
:10138000D8A412000401CD51080A0AE122C45EFF6C
:10139000040ECD6F0F015E5103E0100E0401CD6FFE
:1013A0000401C00519E1040E0401076F280E066F41
:1013B0008DEC21F00401BF51020A04E1840E040106
:1013C000046F840C040104BD03D0C80E046FC80C64
:1013D000880E0401046F880C0401C16B0401C05124
:1013E000020AD8B465A81CD004010151080A18E10A
:1013F0000031E8320F0B0D0A13E100BF11D0040ECB
:10140000036F200E026F040E0401C86F280EC76F11
:10141000040ECA6F200EC96F080ECB6F80EF3CF030
:101420000401C06B080E0401016F040E036F200E4F
:10143000026F8C0E006F046B120064502FE10401E8
:101440000031E8320F0B0D0A0FE104BF046B0401F9
:10145000BF6B0401C06B0401C56BC46BD7EC25F0F6
:101460008CEC25F05AEF24F00401C051020A44E14B
:10147000070E0401CB6F040EC86F280EC76F040E51
:10148000CA6FCE0EC96F20EC3CF0010E0401D56F7F
:10149000040E0401036F200E026F12006450040A50
:1014A000D8A412000401CD51080A0AE122C45EFF4B
:1014B000040ECD6F0F015E5103E0100E0401CD6FDD
:1014C0000401C00519E1040E0401076F280E066F20
:1014D000DFEC21F00401BF51020A04E1840E040193
:1014E000046F840C040104BD03D0C80E046FC80C43
:1014F000880E0401046F880C0401C16B0401C05103
:10150000020AD8B465A81CD004010151080A18E1E8
:101510000031E8320F0B0D0A13E100BF11D0040EA9
:10152000036F200E026F040E0401C86F280EC76FF0
:10153000040ECA6F200EC96F080ECB6F3CEF3CF053
:101540000401C06B080E0401016F040E036F200E2E
:10155000026F8C0E006F046B1200A192F60E7B6E70
:101560003C0E7A260101D86701D03C0C010ED80749
:10157000D8A4010C00010FAE010C0FBA09D010A8BD
:101580001088416A0F9C10960001109CF19C12007B
:1015900010A86AD010AC02D0109C66D0412A81A459
:1015A00002D0D89001D0D8800301EE370301EF3785
:1015B0000301F0370301F1370301F2370301F33779
:1015C0000301F4370301F5370301F6370301F73759
:1015D0004150070B03E10301EE5140260FAC20D030
:1015E00010A403D04150500A05E010B43DD0415042
:1015F000400A3AE1108C0301EE51405EEE51406228
:101600000CD009B20AD0030E216EEE0E206EBCEC97
:101610001BF0416A8F80138A27D01080416A09D05D
:1016200010A609D041502A0A03E041502B0A1CE1C0
:101630001082F18C19D04150080A16E1EEC340F037
:10164000108C0301EE51110A02E110861A8210A4D7
:1016500004D00301EE51EB0A06E010B405D00301FB
:10166000EE51A50A01E10F8C140E0101D86F0001A3
:101670000F9A140C2FC176F130C177F1510E7B6FA8
:101680007A6B31051CE1196B750E186F90EC2EF01A
:10169000786F7851080B756F755167E0510E196FAF
:1016A000750E186F90EC2EF0786F7887510E186FCA
:1016B000750E176F78C119F150EC35F056D0196BD3
:1016C000750E186F90EC2EF0E3D7C00E7625326FB2
:1016D000FF0E7721336F3351800A800F010ED8B48B
:1016E000325D20E3796B47D890EC2EF0DF6E7A4BB9
:1016F0007B2B792B3F0E7965F6D72DC126F12EC1B4
:1017000027F1010E296F350E286F400E2A6FA8ECC5
:101710003CF0400E2D27000E2E23C00E7627FF0E24
:10172000772323D0796B07D026D890EC2EF0DF6E8C
:101730007A4B7B2B792B79C132F1336B3351800A91
:10174000346F7651325D7751800A3459EDE32DC103
:1017500026F12EC127F1010E296F350E286F76C1B3
:101760002AF1A8EC3CF0766B776B0101775176118A
:10177000D8B41200AAD7350E7925D96EDA6A010ECF
:10178000DA227AC118F17BC119F11200E8CF23F1F6
:10179000C839E8461F0B156F166BF4EC24F015C121
:1017A00021F116C122F15BD862D85BEC43F0DF6E09
:1017B000232B55D864D85BEC43F0DF6E232B4FD836
:1017C0003A0EDF6E232BC939E842070BC8C11FF15F
:1017D000206BD8901F372037D8901F37203757D825
:1017E000F4EC24F015C121F116C122F138D83FD80C
:1017F0005BEC43F0DF6E232B32D841D85BEC43F037
:10180000DF6E232B2CD83A0EDF6E232BCA45010B3B
:10181000C9C11FF1206B3BD8F4EC24F015C121F1B4
:1018200016C122F11CD823D85BEC43F0DF6E232BCA
:1018300016D825D85BEC43F0DF6E232B1E5104E055
:101840000ED8200EDF6E232B1F0E01012325D96E2B
:10185000DA6A0501050EDA22000EDF6E000C1F0E9B
:1018600001012325D96EDA6A050EDA22120010EE84
:1018700003F02151E1262251E222E750120010EE3E
:1018800004F02151E1262251E222E7501200D890C3
:101890001F3720371F133F0E1F15156F166B000CD7
:1018A000E8CF54F100010CBC02D0D890120057C60A
:1018B00015F10101545131EC40F0F7E3050125EE3B
:1018C000D3F0020EDF64F1D725EED3F0050EDF640E
:1018D00001D0EBD700010CACE8D7020E0101536F29
:1018E0000ED01F0E010153255AD8500FDEE31F0EF4
:1018F0000101532554D8460FD8E20101532B0501AD
:10190000D3510101535DEDE305011F0ED325D96EBF
:10191000DA6A050EDA22DF6A210E01014E6F050E2A
:101920004F6F4EC11BF14FC11CF1FCEC17F01BC1F6
:1019300051F11CC152F1000E515D010E5259B5E238
:101940008A8E51C1F2F452C1F3F40001148080EC8C
:10195000F5F001015439F00B506F080E406F5051F3
:1019600088ECF0F040C151F141C152F106015751EC
:1019700098EC44F002E2D8801200545169EC3DF03A
:101980000101506F51C139F152C13AF154C13BF1DB
:1019900050C13CF1030E3D6F56EC34F0ECD7D96EDC
:1019A000DA6A0501050EDA22DF50800A1200E8CF5C
:1019B00030F10101326BFD0E176F520E166F010EE2
:1019C0004EEC32F0880E0101296F130E2A6F000EC3
:1019D0002B6B2C6B2D6BF2EC9FF00101346F3451AB
:1019E000080A02E1010E326F3451360A17E0345111
:1019F000280A14E03451290A11E034510C0A0EE08F
:101A000034512C0A0BE0880E296F130E2A6F2B6BB2
:101A10002C6B010E2D6FF2EC9FF0DFD734510C0AC6
:101A200008E0320506E0130E2A6F880E296F2BECB2
:101A300037F00101336BFD0E176F5A0E166F010E52
:101A40004EEC32F0880E0101296F130E2A6F000E42
:101A50002B6B2C6B2D6BF2EC9FF00101316F130E91
:101A60002A6F880E296F2BEC37F001013151380AAB
:101A70000EE01BEC45F0FFEC44F0D10E0101295DB6
:101A8000070E2A59F8E3332B020E3365D4D73351AE
:101A9000030A02E10C0E346F1BEC45F0FFEC44F03E
:101AA000B90E0101295D0B0E2A59F8E31894305143
:101AB000310A01E1188401013451120000010D9C2A
:101AC0001BEC45F059D0F4EC05F00301EA6F00017E
:101AD0000DAC52D00A010051300A01E1010C005155
:101AE000310A03E00051320A47E1010E01014F6F54
:101AF0004E6B0AD060D83A0EDF6204D04F074FC158
:101B00004EF105D001014F2B56D8DF50F3E1010112
:101B10004E6701D0020C4F6B13D0BB0E01014F2555
:101B2000D96EDA6A070EDA22DF504C6F010E4F25AC
:101B3000D96EDA6A0A0EDA22DF504C1904E14F2B13
:101B40004E514F5DEAE34F514E19E4E14F6B06D021
:101B500023D81F0E01014F2518D84F2B1DD8DF5059
:101B6000F7E14FC1D3F50A010051310A01E1030C3D
:101B70000051320A01E1040CFFEC44F0E90E0101CE
:101B8000295DFD0E2A599FE3000CE16EE26A050E05
:101B9000E222DFCFE7FF1200020E4C6F0A0E4D6FFC
:101BA0004E514C27000E4D234F514C25D96E000E3F
:101BB0004D21DA6E1200000E01014F25D96EDA6A4E
:101BC0000A0EDA221200E8CF5AF1000114B202D054
:101BD000D890120005C515F101015A5131EC40F0C1
:101BE000F7E30501D351070AF3E11F0ED325D96EA0
:101BF000DA6A050EDA22DF6A220E0101556F050E40
:101C0000566F55C11BF156C11CF1A2EC1AF01BC155
:101C100057F11CC158F157C11FF158C120F1AFEC69
:101C20003EF0D6E3000115A835D0068A19940501C7
:101C30002051300A02E1198401D00788099002017D
:101C4000CA6B08BE8A9C468405012051300A10E107
:101C5000020E0101166FFE0E156FE5EC19F0010181
:101C6000186B540E176F3F0E196F50EC35F00FD0F4
:101C7000020E0101166FCC0E156FE5EC19F0010193
:101C8000186B540E176F1F0E196F50EC35F00001D2
:101C9000469410D080ECF5F001015A39F00B596FE1
:101CA000480E406F595188ECF0F00501055198EC51
:101CB00044F002E2D88012005A5169EC3DF0010173
:101CC000596F59C14EF15A5113ECE6F0F3D7E8CFF2
:101CD00054F100010CBA02D0D890120054C615F18C
:101CE0000101545131EC40F0F7E300010CAAF4D7A4
:101CF000050125EED3F0020EDF64EED725EED3F01A
:101D0000050EDF6401D0E8D7020E0101536F10D039
:101D10001F0E01015325CFEC0CF0500FDDE31F0E19
:101D200001015325CFEC0CF0460FD6E20101532BF5
:101D30000501D3510101535DEBE305011F0ED325CE
:101D4000D96EDA6A050EDA22DF6A210E01014E6FC2
:101D5000050E4F6F4EC11BF14FC11CF1FCEC17F08B
:101D60001BC151F11CC152F1000E515D010E5259BF
:101D7000B3E28A8C51C1D8F452C1D9F4000106866D
:101D800080ECF5F001015439F00B506F050E406FF7
:101D9000505188ECF0F040C151F141C152F10601BF
:101DA000545198EC44F002E2D8801200545169EC8E
:101DB0003DF00101506F51C139F152C13AF154C1A6
:101DC0003BF150C13CF1030E3D6F56EC34F0ECD7C3
:101DD000040122050EE120511F0B0BE10401C48F09
:101DE0000401C66B04012151030A03E1010E040141
:101DF000C66F04012267120020511F0B020AD8A4EB
:101E0000120024510F0BD8B412000401C48F06EC49
:101E100042F0C7C4F6FFC8C4F7FF000EF86E0F0EFD
:101E2000F76404D0840EF56E0C0006D0F6CFE9FFFF
:101E3000F7CFEAFF840EEF6E04012151030AD8B4F4
:101E4000120024510F0B0101006F4C0E016F0F0E99
:101E5000026F00510127E86A00BFE868022301C150
:101E6000D9FF02C1DAFFFE0EDE16000EDD16C7C472
:101E7000F6FFC8C4F7FF000EF86E0F0EF76404D02B
:101E8000C80EF56E0C0006D0F6CFE9FFF7CFEAFFDB
:101E9000C80EEF6E040124AF1200C7C4F6FF0401A0
:101EA000C8C4F7FF000EF86E0F0EF76404D0400EA2
:101EB000F56E0C0006D0F6CFE9FFF7CFEAFF400E33
:101EC000EF6E12000301D02BFC0E0101176FB20E52
:101ED000166F010E4EEC32F0880E0101296F130EC1
:101EE0002A6F000E2B6B2C6B2D6BF2EC9FF0010117
:101EF000306F3051160A03E03051170A11E118B45F
:101F000007D017A80BD0179812AE178A0E9206D0DA
:101F100018A004D0189012AC1882F8D7048027D0EB
:101F20003051180A09E03051190A06E030511A0AF6
:101F300003E030511B0A0DE1000104901BEC45F059
:101F4000FFEC44F0210E0101295D4E0E2A590FE2EB
:101F5000F7D730510C0A0BE0880E296F130E2A6F49
:101F60002B6B2C6B010E2D6FF2EC9FF0C0D7010193
:101F700030510C0A06E0130E2A6F880E296F2BECE5
:101F800037F0010130511B0A0CE030511A0A09E008
:101F90003051190A06E03051180A03E00301D06BF2
:101FA00007D0020E0301D06503D0D06BD890120089
:101FB000D88012002E0E0101166FE00E156F01D0B1
:101FC000040068D8D8B41629FBE19B8CEA0E166F82
:101FD000600E156F01D004005DD8D8B41629FBE15E
:101FE000F26AF06A9D6AA06ABB6AB66AC66AAC6A9F
:101FF000C26A060EC16EC088C16AF80EC26EC09871
:10200000896A8C6A2F0E926E4F0E956E868E8A6A42
:102010008D6A050E936E020E966EF19E8B6A8E6A25
:10202000D40E946EBC0E976E8B828F6A656A1C0EFE
:10203000986ED56A810ECD6ED10ECF6E200ECE6E0B
:102040009E909F909D80810E796EF60E7B6E3C0E69
:102050007A6EA192A292A082C088020ECE6EC09823
:10206000D0B805D0A80E0301BD6FC00E04D0020E7B
:102070000301BD6FD00EBC6F0B9C750E0101166F76
:10208000300E156F01D0040005D8D8B41629D8B485
:102090001200F9D701011507D8A01607152912005B
:1020A0000001F9510A0A10E015BC0ED0000E4424BC
:1020B000D96EDA6A0B0EDA22F9C0DFFF442AA00ECD
:1020C0004464A00C446A12000001F9510A0A2FE18D
:1020D00015BC2DD00B01000E4424D96EDA6A0B0E0C
:1020E000DA22DF6A446A0B0E206E000E1F6EEE0EBF
:1020F000226EF10E216E246A110E236ED7EC27F0AA
:1021000020501F1014E10001158C110E2E6E0B0EC5
:102110002F6E2EC025F02FC026F060EC18F0FF0EB9
:1021200025240401DC6FFF0E2620DD6F1200000164
:1021300015AC12000401DD51DC1104E0DC07D8A06D
:10214000DD0701D0159C0001F9510A0A0FE10201D7
:10215000DC07000EDC25D96EDA6A0A0EDA22000EE0
:10216000DF6A0D8CDCC2E4F2DC6B1200F9510A0A62
:10217000D8B41200000E0201DC25D96EDA6A0A0E0C
:10218000DA22F9C0DFFFDC2B120004921EC543F1F6
:1021900005010E512B0A03E1010143070482050EDC
:1021A0000101226F1F0E216FFE0E246F4B0E236F55
:1021B00086ECCEF02151446F44C145F151D84339EA
:1021C0000F0B5BEC43F0DF6E452B4AD843510F0BEE
:1021D0005BEC43F0DF6E452B04A209D01F0E39D80B
:1021E000FF0E246FF00E236F86ECCEF008D01F0E8A
:1021F00030D8FF0E246FF30E236F86ECCEF0215102
:10220000446F445145274551F8EC08F01F0E416FCB
:10221000050E426F41C115F142C116F1CFEC36F007
:102220001551456F1F0E15D8FF0E246F970E236FA3
:1022300086ECCEF02151446F445145271F0E010119
:102240004525D96EDA6A0501050EDA22000EDF6E29
:10225000000C01014525216F226B050E222312007F
:102260001F0E01014525D96EDA6A050EDA22120029
:102270004D0E0201006FA36B5ED8DF501BE1A3C2BD
:1022800037F10101372B5FD80D0EDF6EA3C237F196
:10229000020E372758D80A0EDF6EA3C237F1030E9D
:1022A0003727000E3725D96EDA6A0201020EDA22CC
:1022B000DF6A12D040D8A3C237F10101372B000EDC
:1022C0003725E16EE26A0201020EE222DFCFE7FF6C
:1022D000A32B9F0EA365D0D79F0EA36505D00D0E2F
:1022E000A06F0A0EA16FA26B020E01012C6F000EEF
:1022F0002B6F000E2E6B2D6BACEC04F002E2D8902D
:102300001200199A00010D9C1BEC45F00BD0000146
:102310000DAC08D00A010051300A02E1D880120049
:1023200000010D9CFFEC44F0E90E0101295DFD0E5A
:102330002A59E5E2ECD71F0E0201A325D96EDA6A0D
:10234000050EDA221200000E3725D96EDA6A020E67
:10235000DA221200E8CF9DF2010E02019F6F9D511B
:1023600002E0030E9F6F01011B6B1C6B060E020146
:102370009F25D96EDA6A0501050EDA22DF5027ECB7
:1023800043F01D6F050E02019F25D96EDA6A050123
:10239000050EDA22DF5027EC43F01E6F000E83ECAF
:1023A00032F01B5102019E6F9D6702D0039003D053
:1023B0009D0501E1039202019C6B9E513CECEEF005
:1023C00011E300011B9462ECE0F002019F6F9F514A
:1023D000800A7A0F07E29F510CECC4F003E3010E70
:1023E00002019C6F02019C6721D0FB0E0101176F57
:1023F0008A0E166F010E4EEC32F0130E01012A6F99
:10240000880E296F2BEC37F002019E513CECEEF068
:102410000DE300011B9462ECE0F002019F6F9F51FD
:10242000800A7A0F03E29F510CECC4F002019E5126
:1024300085EF1DF0E8CF30F13051360A06E030511B
:102440002C0A03E030510C0A02E1D89012003051FE
:10245000290A5EE1196B5C0E186F90EC2EF02D6F5F
:10246000196B5B0E186F90EC2EF02F6F2D512E6FA5
:10247000FC0E176FCA0E166F010E4EEC32F02EC115
:1024800015F12FC116F1F4EC24F015C131F116C18C
:1024900032F120EE01F03151D9263251DA22DF50EB
:1024A0005BEC43F0CBEC42F0010120EE02F0315145
:1024B000D9263251DA22DF505BEC43F0CBEC42F00C
:1024C000010120EE03F03151D9263251DA22DF50DA
:1024D0005BEC43F0CBEC42F0010120EE04F0315113
:1024E000D9263251DA22DF505BEC43F0CBEC42F0DC
:1024F000F10E0101176F390E166F000E4EEC32F01F
:10250000130E01012A6F880E296F2BEC37F09DE323
:10251000D8801200040122050EE120511F0B0BE1AF
:102520000401C48F0401C66B04012151030A03E1B5
:10253000010E0401C66F04012267120020511F0B17
:10254000020AD8A4120024510F0BD8B412000401BF
:10255000C48F6AEC42F058EC28F0F76404D0840E83
:10256000F56E0C0006D0F6CFE9FFF7CFEAFF840E38
:10257000EF6E04012151030AD8B4120024510F0B4D
:102580000101156F4C0E166F0F0E176F15511627A0
:10259000E86A15BFE868172316C1D9FF17C1DAFF2B
:1025A000FE0EDE16000EDD1658EC28F0F76404D09F
:1025B000C80EF56E0C0006D0F6CFE9FFF7CFEAFFA4
:1025C000C80EEF6E040124AF1200C7C4F6FF040169
:1025D000C8C4F7FF000EF86E0F0EF76404D0400E6B
:1025E000F56E0C0006D0F6CFE9FFF7CFEAFF400EFC
:1025F000EF6E1200E8CF19F186860001FA6B3A0EF1
:10260000DEEC42F03A0E06EC45F00101176702D00D
:102610000F0E176F18051DE11751F00B0CE017395D
:102620000F0B5BEC43F01A6F1A51DEEC42F0010124
:102630001A5106EC45F0010117510F0B5BEC43F00A
:102640001A6F1A51DEEC42F001011A5106EC45F006
:102650000DD017510F0B5BEC43F00301C16FC1515B
:10266000DEEC42F00301C15106EC45F001011951C5
:10267000DEEC42F00101195106EC45F00101165162
:10268000DEEC42F00101165106EC45F0FA390F0B71
:102690005BEC43F0DEEC42F00001FA510F0B5BEC17
:1026A00043F0DEEC42F00D0EDEEC42F00A0EDEEC02
:1026B00042F00301A86BA96B000EA76F0A0EA66F6C
:1026C00000011D9AADB203D000011DAAFBD786966A
:1026D00012000301F15127EC43F0166F0301F05192
:1026E00027EC43F0176F1739F00B16110301EE6F4B
:1026F00005AE1DD0F35127EC43F0166F0301F251E4
:1027000027EC43F0176F1739F00B16110301EF6F29
:10271000F55127EC43F0166F0301F45127EC43F019
:10272000176F1739F00B16110301F06F06D0010176
:10273000D0510301EF6FCFC1F0F3F75127EC43F015
:10274000166F0301F65127EC43F0176F1739F00BA2
:1027500016110301F16FF95127EC43F0166F0301D5
:10276000F85127EC43F0176F1739F00B16110301DE
:10277000F26FFB5127EC43F0166F0301FA5127EC7F
:1027800043F0176F1739F00B16110301F36FFD516A
:1027900027EC43F0166F0301FC5127EC43F0176F51
:1027A0001739F00B16110301F46FF56B1200E8CF27
:1027B00023F1DF07DF51220DF90EF324296F3F0EBD
:1027C000F4202A6F29C118F12AC119F190EC2EF0DA
:1027D000276F286BD89027351F6F2835206F23511E
:1027E0001F252B6F000E20212C6F2BC124F12B07EE
:1027F000D8A02C07D89027351F6F2835206FDF51C0
:10280000220D1F51F324216F2051F420226FF90E65
:102810002125296F3F0E22212A6F2ED029C118F1C0
:102820002AC119F190EC2EF01F6FFF0E2925186FA9
:10283000FF0E2A21196F90EC2EF0266F1F51256F85
:102840001E0E01012B25D96EDA6A050EDA222651F9
:10285000DF6E1F0E2B25D96EDA6A050EDA2225C12E
:10286000DFFF2707D8A02807FE0E2B27FF0E2C23FB
:10287000020E295F000E2A5B2851800A800F010E8C
:10288000D8B4275DCBE22451120004EE00F0D60E3E
:10289000EE6AE806FDE10DEE00F0F00EEE6AE806E5
:1028A000FDE10CEE00F0960EEE6AE806FDE10BEE9F
:1028B00000F0F00EEE6AE806FDE10AEE00F0F00E20
:1028C000EE6AE806FDE109EE00F0B40EEE6AE806F5
:1028D000FDE108EE00F0F20EEE6AE806FDE107EE1B
:1028E00000F0F50EEE6AE806FDE106EE00F0F90EE6
:1028F000EE6AE806FDE105EE00F010EEFFF0EE6A8C
:10290000E550E150FCE1E250FAE103EEA6F0590E89
:10291000EE6AE806FDE102EEA6F05A0EEE6AE8065F
:10292000FDE101EEC1F02A0EEE6AE806FDE100EEDF
:10293000E9F0170EEE6AE806FDE100EE01F01E0E6A
:10294000EE6AE806FDE100EE3FF0070EEE6AE806EB
:10295000FDE104EED6F0280EEE6AE806FDE1000186
:1029600014EF8EF0E8CF54F16EC615F10101545109
:1029700031EC40F002E2D89012000501D3510B0A6D
:10298000FAE126C550F1266B220E01014E6F050EAD
:102990004F6F4EC11BF14FC11CF1A2EC1AF01BC1CD
:1029A00052F11CC153F152C11FF153C120F1AFECE0
:1029B0003EF0E1E350C126F505011F0ED325D96E87
:1029C000DA6A050EDA22DF6A260E01014E6F050E65
:1029D0004F6F4EC11BF14FC11CF1A2EC1AF01BC18D
:1029E00052F11CC153F152C11EF153C11FF1A5ECAC
:1029F00042F001015439F00B516F300E406F5151CC
:102A000088ECF0F040C152F141C153F106016E5122
:102A100098EC44F002E2D8801200545169EC3DF089
:102A20000101516F52C139F153C13AF154C13BF127
:102A300051C13CF1030E3D6F56EC34F0ECD7E8CFBA
:102A400054F16EC615F10101545131EC40F002E22F
:102A5000D89012000501D3510B0AFAE126C550F1B6
:102A6000266B220E01014E6F050E4F6F4EC11BF1FA
:102A70004FC11CF1A2EC1AF01BC152F11CC153F161
:102A800052C11FF153C120F1AFEC3EF0E1E350C160
:102A900026F505011F0ED325D96EDA6A050EDA2256
:102AA000DF6A260E01014E6F050E4F6F4EC11BF1FE
:102AB0004FC11CF1A2EC1AF01BC152F11CC153F121
:102AC00052C11EF153C11FF139EC43F001015439D9
:102AD000F00B516F300E406F515188ECF0F040C157
:102AE00052F141C153F106016E5198EC44F002E2FB
:102AF000D8801200545169EC3DF00101516F52C170
:102B000039F153C13AF154C13BF151C13CF1030ECB
:102B10003D6F56EC34F0ECD70201B46BB56BB66B7D
:102B2000B76B0101086B2AD008510025D96E000E41
:102B30000121DA6EDF500201B427000EB523B45D27
:102B4000010EB55903E3B44BB52BB56BB429B511E0
:102B500002E1B46BB56BB451B627B551B723000E83
:102B6000B65D010EB75903E3B64BB72BB76BB62969
:102B7000B71102E1B66BB76B0101082BFE0E0225FF
:102B8000036F046BFF0E042308C105F1066B0651A9
:102B9000800A076F0351055D0451800A0759C4E399
:102BA00002511ED8FE0E12D8B45D0101086F0867ED
:102BB0000BD0025115D8FF0E09D8B65D0101086F80
:102BC000086702D0D8801200D89012000325D96E71
:102BD000FF0E0421DA6EDF50056F0551020112006D
:102BE0000025036FE86A02BFE8680121046F120044
:102BF00020EE01F01E51D9261F51DA22DF50206F3E
:102C000020C121F1226B213B223BF00E22172151E2
:102C10000F0B2213F00E2117236B0F0E2215246FBA
:102C200020EE02F01E51D9261F51DA22DF50231167
:102C3000256F2451266F25C115F126C116F1F4EC3C
:102C400024F015C127F116C128F11EC1D9FF1FC1FB
:102C5000DAFF10EE02F01E51E1261F51E222DFCF13
:102C6000E7FF20EE04F02751D9262851DA22DF5061
:102C7000206F20EE03F02751D9262851DA22DF50A9
:102C8000216F2139F00B20111EC1D9FF1FC1DAFFBE
:102C9000DF6E20EE01F01E51D9261F51DA2210EE10
:102CA00002F02751E1262851E222E750206F10EE72
:102CB00001F01E51E1261F51E222E750216F213918
:102CC000F00B2011DF6E1200F50E176F370E166F26
:102CD000010E4EEC32F04DD0C4ECE7F002A449D026
:102CE00002940201CE6701D044D0080E01011C6F8E
:102CF000A00E1B6FFD0E1E6F620E1D6F206B070E68
:102D00001F6F47EC27F01C511B1133E1080E2E6F8B
:102D100010D037D8DF620DD007D033D8DF6204D0AF
:102D20002EC12DF1320E2E6F01012E51800A4E0F51
:102D3000F4E301012E51800A4E0FEBE3A00E296F40
:102D4000080E2A6F2D512927000E2A2329C11BF1B5
:102D50002AC11CF1FCEC17F01BC12BF11CC12CF19A
:102D60002C51800A750FB80ED8B42B5D08E2D890AC
:102D70001200310E0301B25D750EB359ADE3D88078
:102D800012002E2B2E05296FA00E01012925D96EC8
:102D9000DA6A080EDA222C0CE8CF26F026500A0A4E
:102DA00057E10301DC6B0C010C0E206E000E1F6E50
:102DB000FD0E226E120E216E246A070E236ED7ECD2
:102DC00027F020501F1004E1020E0001FC6F020CDE
:102DD0000C010C0E206E000E1F6EFD0E226E6F0E8B
:102DE000216E246A020E236ED7EC27F020501F10AC
:102DF00004E1010E0001FC6F010C0C010C0E206EB1
:102E0000000E1F6EFF0E226E9C0E216E246A030EB2
:102E1000236ED7EC27F020501F1004E1030E0001B1
:102E2000FC6F030C0C010C0E206E000E1F6EFF0ECB
:102E3000226E240E216E246A040E236ED7EC27F036
:102E400020501F10D8A41200040E0001FC6F040CC7
:102E5000000E0301DC25D96EDA6A0C0EDA2226C0D8
:102E6000DFFFDC2B1200190E1F6E280EC26EC2800F
:102E70001F061F28FDE1C282320E1F6E1F061F288B
:102E800002E0C2B2FBD7C4CF20F0630E20600ED0A8
:102E90000301C96BC82B3B0EC86508D0C86BC76758
:102EA00005D0010EC76F169E169C188E0201D151D7
:102EB000205C09E30301C86BC92B3B0EC96503D035
:102EC000C96B18BEFF00C26A280E206007D003013C
:102ED000C32B020EC365020CFF00020C0301C65196
:102EE000205C11E3C46BC36BC52B770EC565770CF3
:102EF000C56B079C079AC76B189E000108A21200B9
:102F000008800892120020500201D15DD8A0120062
:102F10000301C56BC36BC42B3B0EC4653B0CC46B78
:102F2000078C0882000107BA1200078E078A120078
:102F3000325105EC38F015C137F116C138F137C1FF
:102F4000D9FF38C1DAFFDF50356F320502E1280EB4
:102F50000AD03251020AFBE03251030AF8E0325142
:102F6000040AF5E0020E366F3651355D2AE3F00EA5
:102F7000176F2E0E166F000E4EEC32F0880E010108
:102F8000296F130E2A6F000E2B6B2C6B2D6BF2EC3E
:102F90009FF032C118F1000E90EC27F0325105EC91
:102FA00038F015C137F116C138F137C1D9FF38C132
:102FB000DAFFDF50356F500E206FE00E1F6F57ECB9
:102FC00037F037C1D9FF38C1DAFFDF2A01013251AA
:102FD000AFEC37F015C133F116C134F13551020DA4
:102FE000F3503325D96E000E3421DA6E30C1DEFF86
:102FF00031C1DDFFD880120003D001011B4B1C2B17
:103000001BC1D9FF1CC1DAFFDF50200AF6E01BC14B
:10301000D9FF1CC1DAFFDF50090AEFE00101226B82
:10302000236B216B2D0E1BC1D9FF1CC1DAFFDF62A0
:1030300002D0212B07D02B0E1BC1D9FF1CC1DAFFF8
:10304000DF6222D01B4B1C2B1FD01BC1D9FF1CC120
:10305000DAFFDF501D6F1E6B1DBF1E0722C115F169
:1030600023C116F1186B0A0E176F16EC41F01D51B3
:1030700015251F6F1E511621206FD00E1F25226FA0
:10308000FF0E2021236FDED71BC1D9FF1CC1DAFF41
:10309000DF509FEC43F0D9E221510DE022C11DF138
:1030A00023C11EF11D1F1E1F1D4B1E2B1DC11BF119
:1030B0001EC11CF1120022C11BF123C11CF1120020
:1030C00002D0254A262A25C0D9FF26C0DAFFDF50C4
:1030D000200AF7E025C0D9FF26C0DAFFDF50090A31
:1030E000F0E02C6A2D6A2B6A2D0E25C0D9FF26C070
:1030F000DAFFDF6202D02B2A07D02B0E25C0D9FFC2
:1031000026C0DAFFDF6222D0254A262A1FD025C03A
:10311000D9FF26C0DAFFDF50276E286A27BE2806AF
:103120002CC01FF02DC020F0226A0A0E216E6EEC1A
:1031300041F027501F24296E285020202A6ED00EDF
:1031400029242C6EFF0E2A202D6EDED725C0D9FF34
:1031500026C0DAFFDF504AEC43F0D9E22B500DE0F5
:103160002CC027F02DC028F0271E281E274A282A09
:1031700027C025F028C026F012002CC025F02DC055
:1031800026F012001A5105EC38F015C11FF116C1D6
:1031900020F11FC1D9FF20C1DAFFDF50256F25675D
:1031A00001D012001A51AFEC37F015C121F116C150
:1031B00022F1236B44D02351020DF3502125D96E07
:1031C000000E2221DA6EDECF1BF1DDCF1CF11B5188
:1031D0001D6F030E1C151E6F191902E118511D19E0
:1031E0002DE11FC1D9FF20C1DAFFDF50DF06256FB7
:1031F00023C124F11ED0D89024351B6F1B512125EB
:103200001C6FE86A1BBFE86822211D6F020E1C2597
:10321000D96E000E1D21DA6E2451020DF3502125C6
:10322000E16E000E2221E26EDECFE6FFDDCFE5FF8C
:10323000242B2551245DD8B01200DDD7232B255136
:10324000235DD8B01200B7D7DACF0EF1F3CF0FF16C
:10325000F4CF10F1F6CF11F1F7CF12F1F8CF13F14F
:10326000F5CF14F18FEC44F0F2A801D001D006D0D4
:10327000F2A201D001D002D0DCEC41F0F0A801D0E4
:1032800001D00AD0F0A201D001D006D0F0AE01D01A
:1032900001D002D0AAEC44F0A3A601D001D00AD0FC
:1032A000A4A601D001D006D0A5A601D001D002D09D
:1032B000A1ECDCF0F2AA01D001D012D0F2A401D02E
:1032C00001D00ED0F1A401D001D00AD0000110AE7F
:1032D00001D001D003D0FFEC3AF002D0A1EC36F0DF
:1032E00014C1F5FF13C1F8FF12C1F7FF11C1F6FFBA
:1032F00010C1F4FF0FC1F3FF0EC1DAFF0DC1D9FFFA
:103300000CC1EAFF0BC1E9FF1100E8CF24F1276BE4
:1033100024072451330D8D0EF324286F130EF4204F
:10332000296F28C118F129C119F190EC2EF0256FF1
:10333000266B284B292B2651800A800F020ED8B409
:10334000255D07E32651800A800F180ED8B4255D4D
:1033500020E31F69206912002829186F000E292117
:10336000196F90EC2EF0216F28C118F129C119F1C5
:1033700090EC2EF0236F2151226F22513F0A23112E
:10338000D8B4272B2507D8A02607020E2827000E21
:1033900029232651800A800F010ED8B4255DDCE276
:1033A000020E276505D0F00E206F000E1F6F000C77
:1033B0002751020A04E12069000E1F6F000C270547
:1033C000C8E12069F00E1F6FF00C000118BE12005A
:1033D00014BE128814A21AD001011551220A161126
:1033E00010E01551260A16110CE015512A0A161183
:1033F00008E015512E0A161104E01551360A16116F
:1034000005E1098008BE8A8CD2C2CAF2130E0101FE
:10341000DA652BD0DA071C6B17D0D8901C35176FE4
:10342000020E01011725D96EDA6A060EDA221C5146
:10343000020D000EF324E16EE26A060EE222DECFF8
:10344000E6FFDDCFE5FF1C2BDAC117F1186B1CC1BD
:1034500019F11A6B19BF1A071A51800A1B6F1751FD
:10346000195D1851800A1B59D8E3DA51020D000E7C
:10347000F324D96EDA6A060EDA22010115C1DEFFE5
:1034800016C1DDFFDA2B12001E6B1CAF0AD01C1F09
:103490001B1F1A1F196D000E1A231B231C23010E5C
:1034A0001E6F18AF0AD0181F171F161F156D000EBC
:1034B000162317231823010E1E1B1F6B206B216B75
:1034C000226B1C5119111A111B1129E0010E1D6FDD
:1034D00006D0D89019371A371B371C371D2B1CAF55
:1034E000F8D7D8901F372037213722371951155D6B
:1034F0001A5116591B5117591C51185909E31951E2
:10350000155F1A51165B1B51175B1C51185B1F810D
:10351000D8901C331B331A3319331D2FE2D71E5199
:1035200008E0221F211F201F1F6D000E20232123D2
:1035300022231FC115F120C116F121C117F122C1AB
:1035400018F112001F6B206B216B02D01B4B1C2B40
:103550001BC1D9FF1CC1DAFFDF501AEC42F0F6E2C2
:103560002D0E1BC1D9FF1CC1DAFFDF6202D01F2B59
:1035700007D02B0E1BC1D9FF1CC1DAFFDF621FD0A1
:103580001B4B1C2B1CD022518EEC43F004E3225128
:10359000F9EC43F0226F22519FEC43F0D00ED8A0FB
:1035A000A90E2227203B213BF00E211720510F0BA3
:1035B0002113F00E201722512027000E21231BC1BA
:1035C000D9FF1CC1DAFF1B4B1C2BDF50226F0101FE
:1035D00022513DEC3EF0D7E21F510DE020C11DF11C
:1035E00021C11EF11D1F1E1F1D4B1E2B1DC11BF1D6
:1035F0001EC11CF1120020C11BF121C11CF11200DF
:10360000E8CF27F1000114B202D0D890120005C50E
:1036100015F10101275131EC40F0F7E30501D351D9
:10362000070AF3E11F0ED325D96EDA6A050EDA22F6
:10363000DF6A220E0101256F050E266F25C11BF1E1
:1036400026C11CF1A2EC1AF01BC128F11CC129F102
:1036500028C11FF129C120F1AFEC3EF0D6E30A9C4E
:103660000A9A0B9409900201CA6B08BE8A9C069ABA
:10367000468419A410D0020E0101166FDD0E156FDD
:10368000E5EC19F00101186B540E176F2F0E196F2E
:1036900050EC35F00FD0020E0101166FDD0E156FE4
:1036A000E5EC19F00101186B540E176F0F0E196F2E
:1036B00050EC35F000014694D8801200000118BE8D
:1036C000120014BE128814A219D01F50220A201012
:1036D00010E01F50260A20100CE01F502A0A20106C
:1036E00008E01F502E0A201004E01F50360A201058
:1036F00005E1098008BE8A8CD2C2CAF2130E01010C
:10370000DA652BD0DA07266A16D0D8902634216ED7
:10371000020E2124D96EDA6A060EDA222650020D34
:10372000000EF324E16EE26A060EE222DECFE6FF2F
:10373000DDCFE5FF262A0101DAC121F0226A26C089
:1037400023F0246A23BE24062450800A256E2150CB
:10375000235C2250800A2558D8E3DA51020D000E6E
:10376000F324D96EDA6A060EDA221FC0DEFF20C00B
:10377000DDFF0101DA2B1200000110B408D020EEA9
:1037800003F02050D9262150DA22030EDF1649D843
:1037900003E13FD8D8B41200020ED1EC3FF0000193
:1037A00010A40AD020EE08F02050D9262150DA22A9
:1037B000DF50D1EC3FF024D020EE05F02050D92688
:1037C0002150DA22DF3A20EE05F02050D926215090
:1037D000DA2210EE05F02050E1262150E222E750D7
:1037E000226ED8902232D8902230030BDF6E20EE6A
:1037F00005F02050D9262150DA22DF50D1EC3FF0DD
:1038000010D8D1EC3FF005D8D1EC3FF000010E8488
:10381000120020EE02F02050D9262150DA22DF508B
:10382000120020EE03F02050D9262150DA22DF507A
:103830001200F80E0101176FD40E166F010E4EEC38
:1038400032F02C0ECBEC42F0070170510FE0220E4B
:10385000CBEC42F0070E0101176F700E166F000ED1
:103860004EEC32F0220ECBEC42F006D0220ECBEC26
:1038700042F0220ECBEC42F02C0ECBEC42F0220EAA
:10388000CBEC42F00601DF5108E0060E0101176F94
:10389000DF0E166F000E4EEC32F0220ECBEC42F033
:1038A0002C0ECBEC42F0220ECBEC42F00601E8519C
:1038B00008E0060E0101176FE80E166F000E4EECC1
:1038C00032F0220ECBEC42F0EE0E0101176F0E0E1D
:1038D000166F000E4EEC32F00D0ECBEC42F0130ED4
:1038E00001012A6F880E296F2BEF37F00301C151B8
:1038F00027EC43F01F6F7F0E01014CD81E6F1EAFE7
:1039000012007F0E1F25D96EDA6A060EDA22DF2A30
:103910007F0E40D81E6F3F0E1E17030E1E5D02E382
:103920008F8013887F0E010135D83F0B050A09E10E
:10393000530E0301F16F300EF26F01011F5102ECC3
:1039400039F07F0E01011F25D96EDA6A0601060ED5
:10395000DA22DF503F0B3F0AD8A41200530E0301B6
:10396000F16F200EF26F01011F5102EC39F07F0E52
:1039700001011F25D96EDA6A060EDA22DF6A960E79
:103980001F25176F186B020E18237F0E03D8196FAF
:1039900050EF35F01F25D96EDA6A060EDA22DF50B5
:1039A0001200EF0E0101176FA50E166F010E4EECFF
:1039B00032F0070E0101176F700E166F000E4EECFD
:1039C00032F0220ECBEC42F00D0ECBEC42F0130E97
:1039D00001012A6F880E296F2BEC37F0ED0E0101E3
:1039E000176F430E166F010E4EEC32F0130E0101ED
:1039F0002A6F880E296F2BEC37F0ED0E0101176F3F
:103A00005B0E166F010E4EEC32F0130E01012A6FA1
:103A1000880E296F2BEC37F0EE0E0101176F500E58
:103A2000166F010E4EEC32F0130E01012A6F880E54
:103A3000296F2BEC37F0EE0E0101176F3B0E166F5E
:103A4000010E4EEC32F0130E01012A6F880E296F21
:103A50002BEC37F019EF1CF0E8CF53F102C515F14C
:103A60000101535131EC40F002E2D89012000501FF
:103A7000D351070AFAE11F0ED325D96EDA6A050E73
:103A8000DA22DF6A220E01014E6F050E4F6F4EC122
:103A90001BF14FC11CF1A2EC1AF01BC150F11CC16B
:103AA00051F150C11FF151C120F1AFEC3EF0DDE307
:103AB00000011EB402D000010E8C80ECF5F0010173
:103AC0005339F00B526F800E406F525188ECF0F07A
:103AD00040C150F141C151F10501025198EC44F04F
:103AE00002E2D8801200535169EC3DF00101526F9F
:103AF00050C139F151C13AF153C13BF152C13CF1CE
:103B0000030E3D6F56EC34F0ECD7E8CF2BF1FE0EF0
:103B10000101176F700E166F010E4EEC32F03D0E64
:103B2000CBEC42F001012BC115F1166BF4EC24F043
:103B300015C12DF116C12EF120EE03F02D51D9261D
:103B40002E51DA22DF505BEC43F0CBEC42F0010166
:103B500020EE04F02D51D9262E51DA22DF505BECF5
:103B600043F0CBEC42F00D0ECBEC42F01BEC45F0F9
:103B700001012C6B19D0EAEC44F016E317EC45F088
:103B800001012F6F0DD02F5100EC41F00DE3010129
:103B90002C2B0AD02F51BEEC40F0D8B0120004D02C
:103BA0002C51F1E0010AF6E0FFEC44F0D10E0101E6
:103BB000295D070E2A59D8B01200DDD73D6B50D8C9
:103BC0003D512225186F000E2321196F90EC2EF025
:103BD000DF6E46D8DF5004E03D2B100E3D65EFD779
:103BE0002A5107E02351020A410ED8B4221901E0FC
:103BF0001B8401013B6B2A512B0A03E1010E3B6F31
:103C00003D07DC5109E0DC513D5D3C6F3C51800AD1
:103C10007F0F02E33C513B272A0E266F010E276FD0
:103C20003B512627000E272326C11BF127C11CF17B
:103C30000E0E286F050E296F24512827000E292308
:103C400028C11DF129C11EF125C11FF1206B47ECD0
:103C500027F01C511B1102E1D8801200D8901200ED
:103C60002A0E3D25D96EDA6A010EDA22120020EE04
:103C700001F01E51D9261F51DA22DF50156F166B45
:103C8000F4EC24F015C124F116C125F120EE04F066
:103C90002451D9262551DA22DF50206F20EE03F07F
:103CA0002451D9262551DA22DF50216F2139F00B1A
:103CB0002011226F20EE02F01E51D9261F51DA2268
:103CC000DF50FEEC3BF0236F20EE02F01E51D926B0
:103CD0001F51DA2223C120F1203B0F0E20171EC1F5
:103CE000E1FF1FC1E2FFE750F00B2011DF6E20EE75
:103CF00001F01E51D9261F51DA2210EE02F0245194
:103D0000E1262551E222E750206F2339F00B2011E4
:103D1000DF6E1EC1D9FF1FC1DAFF22C1DFFF120013
:103D200020EE01F01E51D9261F51DA22DF50156F07
:103D3000166BF4EC24F015C124F116C125F120EE28
:103D400004F02451D9262551DA22DF50206F20EECD
:103D500003F02451D9262551DA22DF50216F213971
:103D6000F00B2011226F20EE02F01E51D9261F51B8
:103D7000DA22DF50236F20EE02F01E51D9261F51A8
:103D8000DA2223C120F1203B0F0E20171EC1E1FFD4
:103D90001FC1E2FFE750F00B2011DF6E20EE01F0B3
:103DA0001E51D9261F51DA2210EE02F02451E126CD
:103DB0002551E222E750206F2339F00B2011DF6EEE
:103DC0001EC1D9FF1FC1DAFF22C1DFFF1200E8CFF9
:103DD00053F103C515F10101535131EC40F002E2FA
:103DE000D89012000501D351070AFAE11F0ED3251E
:103DF000D96EDA6A050EDA22DF6A220E01014E6FF1
:103E0000050E4F6F4EC11BF14FC11CF1A2EC1AF011
:103E10001BC150F11CC151F150C11FF151C120F122
:103E2000AFEC3EF0DDE300010E8A80ECF5F001011D
:103E30005339F00B526F840E406F525188ECF0F002
:103E400040C150F141C151F10501035198EC44F0DA
:103E500002E2D8801200535169EC3DF00101526F2B
:103E600050C139F151C13AF153C13BF152C13CF15A
:103E7000030E3D6F56EC34F0ECD7FD0E0101176FC9
:103E8000800E166F010E4EEC32F0880E0101296F84
:103E9000130E2A6F000E2B6B2C6B2D6BF2EC9FF028
:103EA0000101306F06018F51800A500F04E38F51DA
:103EB000800A460F12E3010130510C0A0EE0305126
:103EC000090A0BE0880E296F130E2A6F2B6B2C6BDF
:103ED000010E2D6FF2EC9FF0E3D7010130510C0A77
:103EE00003E13051090A1DE0306B8F0E01013025CE
:103EF000D96EDA6A060EDA22280E3025E16EE26A01
:103F0000060EE222DFCFE7FF302B3051800A710F1F
:103F1000ECE3130E2A6F880E296F2BEC37F0D89044
:103F20001200D880120017C1D9FF18C1DAFFDF5084
:103F3000D95FD951D8B4120020EE01F01751D9261B
:103F40001851DA22000EDF6E32D017C1D9FF18C126
:103F5000DAFFDF5034D81AC1D9FF1BC1DAFF10EEE7
:103F600002F01751E1261851E222DFCFE7FF20EEE1
:103F700002F01751D9261851DA2210EE01F017512C
:103F8000E1261851E222E7501AD81AC1E1FF1BC1FD
:103F9000E2FFDFCFE7FF20EE01F01751D9261851DD
:103FA000DA22DF2A17C1D9FF18C1DAFFDF2A17C1C9
:103FB000D9FF18C1DAFF3F0EDF64C7D73F0C196F76
:103FC000195115251A6FE86A19BFE86816211B6F89
:103FD0001200E8CF53F15EC615F10101535131ECE7
:103FE00040F002E2D89012000501D351070AFAE12D
:103FF0001F0ED325D96EDA6A050EDA22DF6A220E89
:1040000001014E6F050E4F6F4EC11BF14FC11CF1E8
:10401000A2EC1AF01BC150F11CC151F150C11FF1AB
:1040200051C120F1AFEC3EF0DDE343EC36F080EC23
:10403000F5F001015339F00B526F150E406F5251DC
:1040400088ECF0F040C150F141C151F106015E51E0
:1040500098EC44F002E2D8801200535169EC3DF034
:104060000101526F50C139F151C13AF153C13BF1D5
:1040700052C13CF1030E3D6F56EC34F0ECD72FC12A
:1040800074F130C175F139D0C00E7425316FFF0E57
:104090007521326F3251800A800F010ED8B4315D24
:1040A00014E3766B2FD87651800A400FFBE333D8A8
:1040B000400E2A6FA8EC3CF0400E2D27000E2E2358
:1040C000C00E7427FF0E752318D0766B01D01AD856
:1040D00076C131F1326B31BF32073251800A336F12
:1040E0007451315D7551800A3359F1E314D874C1AC
:1040F0002AF1A8EC3CF0746B756B75517411D8B44F
:104100001200C2D7340E7625D96EDA6A010EDA2291
:10411000DF68762B12002DC126F12EC127F1010E8A
:10412000296F340E286F12000101186B196B0BD028
:1041300047D8240EDF6203D00101192B04D040D8E8
:10414000DF50181BF9D73CD8DF50F2E11F0E1925BC
:10415000D96EDA6A050EDA222A0EDF6E19C116F15F
:10416000176B16BF1707200E1625D96E050E1721DF
:10417000DA6E18390F0B18BFF0095BEC43F0DF6EF5
:1041800019C116F1176B16BF1707210E010116256D
:10419000D96E050E1721DA6E18510F0B5BEC43F048
:1041A000DF6E19C116F1176B16BF1707220E01013A
:1041B0001625D96E050E1721DA6E000EDF6E000C83
:1041C0001F0E01011925D96EDA6A050EDA221200D6
:1041D0000A0E236FA00E226F256B48D02307D36BE6
:1041E0009AEC41F0010122510CEC3DF00101D36742
:1041F0002FD018510CEC3DF0010117510CEC3DF0A3
:104200000101246B1DD024511925D96E000E1A21ED
:10421000DA6EDF500CEC3DF00101252BC00E1715B6
:10422000206F1851216F174B182BC00E17151C6FDC
:1042300018511D6F211902E120511C1904E1242B92
:104240001B51245DE0E36AEC3FF0010125511200AF
:10425000070E1F6FD00E1E6F01D000F001011E0768
:10426000D8A01F071E29D8B41F29F7E12351800ABF
:104270007F0FEBE3B3D70101706BD0390F0B506F99
:10428000516B50510F0B5BEC43F06B6F3ED8D0512C
:104290000F0B5BEC43F0DF6E38D8CF390F0B5BECC4
:1042A00043F0DF6E32D8CF510F0B5BEC43F0DF6E83
:1042B0002CD8DF6A010E226F520E216FFC0E246F84
:1042C0008F0E236F070E0101266FBB0E256F010EA7
:1042D000286F6B0E276F86ECCEF02151706F520E57
:1042E0007025D96EDA6A010EDA22DF6A2C6F520E5F
:1042F0002B6F000E2E6B2D6BACEC04F001E2000C6A
:10430000000109B4010C5EEF0DF0702B6B0E7025EF
:10431000D96EDA6A010EDA221200080E0401CB6FA0
:104320000401C5610CD0C5C4CBF40401BF0502E192
:10433000020EBF6F0401BF6702D0010EBF6F040100
:1043400004930491CBC405F40401CB510401C55D71
:10435000C56F040E0401CA6F280EC96F0401C4A101
:104360001DD022D0C2C4F6FFC3C4F7FF000EF86E02
:10437000C9C4D9FFCAC4DAFF0F0EF76403D008001E
:10438000F55005D0F6CFE9FFF7CFEAFFEF50DF6E2B
:104390000401C24BC32B0401C94BCA2B0401CB0738
:1043A000CB29D8B41200DED7C2C4C7F4C3C4C8F442
:1043B00064EC3CF0C7C4C2F4C8C4C3F41200080ED5
:1043C0000401CB6F0401C5610CD0C5C4CBF404015A
:1043D000BF0502E1020EBF6F0401BF6702D0010EEC
:1043E000BF6F040104930491CBC405F40401CB51C5
:1043F0000401C55DC56F040E0401CA6F280EC96FA4
:104400000401C4A11DD022D0C2C4F6FFC3C4F7FF6B
:10441000000EF86EC9C4D9FFCAC4DAFF0F0EF764E4
:1044200003D00800F55005D0F6CFE9FFF7CFEAFF3B
:10443000EF50DF6E0401C24BC32B0401C94BCA2BE2
:104440000401CB07CB29D8B41200DED7C2C4C7F40D
:10445000C3C4C8F420EC3CF0C7C4C2F4C8C4C3F45D
:1044600012000101E6511F0B02E0159801D01588DA
:104470000201C92BC9513E0A06E1C96B00014684FD
:10448000B1ECECF046940101D70507E10201EF67BA
:1044900002D07DEF43F0EF071200D751020A0EE180
:1044A0000201EF67F8D7EE2BEE51080AF2E1EE6B4E
:1044B00019988B9C960E0201EF6F960C00010BB4BD
:1044C000120006AA0BD00201EF67E5D7EE2BEE51E2
:1044D000060ADFE1EE6B19988B8CECD715A804D097
:1044E00000010C968B8C12000CA608D00201DF5143
:1044F00005E0EF67D0D7DF077DEF43F000010C96B2
:104500008B9C1200E8CF59F1000105BA02D0D89077
:10451000120061C615F10101595131EC40F0F7E389
:10452000040E0501D36101D0F2D725EED3F0050EBC
:10453000DF6401D0ECD780ECF5F001015939F00BC4
:10454000506F180E406F505188ECF0F0080E0101CA
:10455000516F0501D351040A09E1205127EC43F0C2
:10456000526F21C553F122C554F111D0215127ECCE
:1045700043F04E6F0501205127EC43F04F6F4F3948
:10458000F00B4E11526F22C553F123C554F1556BF8
:10459000566B576B586B010E176F510E166FD4EC9C
:1045A00040F0D8801200050E356F0301B151B011F3
:1045B00005E193EC3BF03FE3D8801200B0C333F148
:1045C000B1C334F101013151332732513423345115
:1045D000800A7D0FE90ED8B4335D2DE30301B06B83
:1045E000B16B61EC2DF023E3E7D764EC16F014E235
:1045F00093EC3BF0E1E22FC116F130C117F1000E50
:104600004EEC32F0010131510301B027010132516A
:104610000301B123D89012001BEC45F0FFEC44F0ED
:10462000890E0101295D130E2A59F8E335070101AE
:104630003567DBD7C1D72FC116F130C117F1000E96
:104640004EEC32F0DFD71B6B000EE6EC3EF01C6F39
:1046500019C115F11AC116F11CC117F168EC2AF045
:1046600002E301011B81040EE6EC3EF01C6F19C150
:1046700015F11AC116F11CC117F1A9EC2AF002E3D9
:1046800001011B83080EE6EC3EF01C6F19C115F109
:104690001AC116F11CC117F127EC2AF002E301013F
:1046A0001B850C0EE6EC3EF01C6F19C115F11AC10A
:1046B00016F11CC117F1A1EC28F002E301011B87E0
:1046C000100EE6EC3EF01C6F19C115F11AC116F17F
:1046D0001CC117F1E2EC28F002E301011B89010182
:1046E0001B511200000109B21200010E20C0D9FFB7
:1046F00021C0DAFFDF6204D0060ED1EC3FF003D018
:10470000070ED1EC3FF020EE02F033D820EE01F09E
:10471000205024D8D1EC3FF020EE05F02AD8223AE0
:104720000F0E2216221620EE03F0205017D8D1ECDF
:104730003FF020EE05F01DD82238F00B246E2450F7
:10474000D1EC3FF020EE04F02050D9262150DA229F
:10475000DF50D1EC3FF000010E841200D926215029
:10476000DA22DF50236E2338F00B2210246E2450FF
:1047700012002050D9262150DA22DF50226E12007A
:104780006598080E0401016F0401C4BF1BD0040129
:10479000C1510EE0020E0401C06F0401056BC80E8A
:1047A000046F040E036F280E026FC80E006FC80C52
:1047B000040E0401036F200E026F8C0E006F840E36
:1047C000046F840C0401C151D8A41200040120AF6D
:1047D000E1D70401C5510401265D000E2759D8A078
:1047E00026C4C5F48DEC21F0010E0401C06F040E47
:1047F0000401036F200E026F800E006F080E016F20
:10480000040E036F200E026F800E006F040E076F00
:10481000280E066FC80E046FC80CE8CF51F11BB408
:1048200009D00101515103E05151050A03E1010E84
:10483000516F128A51C615F10101515131EC40F00E
:1048400002E2D8901200000112AA0CD0129A0101C3
:104850002B6B010E2C6F050E33ECD4F0F2E3050E3A
:104860000101516F80ECF5F001015139F00B506FEF
:104870008D0E406F505188ECF0F040C14EF141C1B7
:104880004FF10601515198EC44F002E2D880120039
:10489000515169EC3DF00101506F4EC139F14FC1EA
:1048A0003AF151C13BF150C13CF1030E3D6F56EC62
:1048B00034F0ECD76598080E0401016F0401C4BF01
:1048C0001BD00401C1510EE0020E0401C06F0401AF
:1048D000056BC80E046F040E036F280E026FC80E1E
:1048E000006FC80C040E0401036F200E026F8C0EC3
:1048F000006F840E046F840C0401C151D8A412000F
:10490000040120AFE1D70401C5510401265D000E6A
:104910002759D8A026C4C5F4DFEC21F0010E04010C
:10492000C06F040E0401036F200E026F800E006F33
:10493000080E016F040E036F200E026F800E006FD1
:10494000040E076F280E066FC80E046FC80CE8CF60
:1049500027F01C9627B21C8600010BA408D027A2C2
:104960001200000119A612000001078812000001C0
:1049700006AA120000010ABC120000010AAA13D004
:1049800000F027A208D0206A260E1F6E5EEC1BF0F6
:1049900000011C841200206A280E1F6E5EEC1BF0C2
:1049A00000011C94120027A212000A8C19A404D042
:1049B0000401D6C2DEF403D00401D5C2DEF4DF6BFD
:1049C000DE3BDF3BF00EDF17DE510F0BDF13F00E87
:1049D000DE17DF51DE11D8A412000A9C0A8A206A71
:1049E000260E1F6E5EEF1BF00101010E186F190EEF
:1049F000176F196B1A6B1B6B1C6B1D6B100E155D03
:104A0000270E16590AE3192B100E155F270E165B99
:104A1000100E155D270E1659F6E2E80E155D030E11
:104A200016590AE31A2BE80E155F030E165BE80E03
:104A3000155D030E1659F6E2640E155D000E16594B
:104A40000AE31B2B640E155F000E165B640E155DEA
:104A5000000E1659F6E20A0E155D000E16590AE30D
:104A60001C2B0A0E155F000E165B0A0E155D000E5C
:104A70001659F6E215C11DF117C115F118C116F14D
:104A80001200040120511F0B0101156F1505D8A458
:104A9000120004012039E832030B0101156F1505DE
:104AA000D8A41200040124512AE02405D8A412003D
:104AB00026D0040E0401C36FB50EC26F080EC56F79
:104AC000C4810401C48F1200040E0401C36FB50E2B
:104AD000C26FF7D7010E0401C16F010C040E04016F
:104AE000C36FCE0EC26F070EC56F810EC46F810CEF
:104AF00022C4CCF40401CC8F0401C48F1200040141
:104B00002151D7E0010AE0E0210AE4E0010AE6E0F1
:104B1000030AD8A41200ECD7040120511F0B010195
:104B2000006F0005D8A4120004012039E832030BFD
:104B30000101006F0005D8A41200040124512AE0ED
:104B40002405D8A4120026D0040E0401C36FB50EAC
:104B5000C26F080EC56FC4810401C48F1200040E19
:104B60000401C36FB50EC26FF7D7010E0401C16F08
:104B7000010C040E0401C36FCE0EC26F070EC56F89
:104B8000810EC46F810C22C4CCF40401CC8F0401CB
:104B9000C48F120004012151D7E0010AE0E0210A8C
:104BA000E4E0010AE6E0030AD8A41200ECD704010D
:104BB0002039E832030BD8A412002ED00401C48F90
:104BC000080E0401CD6F080C8DEF3AF0E3EF31F0E1
:104BD000040E0401C36FBD0EC26F0401C481010E37
:104BE000C56FC48F010C60EF28F0E8EF0EF0BE0E29
:104BF0000101036F040E046F040124510101032716
:104C0000000E042303C1C2F404C1C3F4E6D70401B7
:104C1000C48F22C4BEF4120004012151E4E0010A51
:104C2000E4E0020AE2E0060AC9E0030ACDE00E0A67
:104C3000CFE0010ACBE0030ADAE0010AD8A41200AF
:104C4000E6D73DD022C11BF123C11CF124C11DF1C7
:104C500025C11EF124C115F125C116F1CFEC36F0A6
:104C600015C11FF116C120F147EC27F01C511B1193
:104C700005E122C122F123C123F112002229156F7F
:104C8000000E2321166F24C1F6FF25C1F7FF000E89
:104C9000F86E0F0EF76403D00800F55005D0F6CF7C
:104CA000E9FFF7CFEAFFEF500101176F186B17BF4D
:104CB0001807A7EC40F015C122F116C123F12351CA
:104CC000221106E022C1D9FF23C1DAFFDF50BAE189
:104CD000226B236B120004012039E832030BD8A4A5
:104CE00012002ED00401C48F080E0401CD6F080CF1
:104CF00041EF3AF077EF31F0040E0401C36FBD0EBF
:104D0000C26F0401C481010EC56FC48F010C1DEF79
:104D100028F08AEF12F0BE0E0101186F040E196F11
:104D20000401245101011827000E192318C1C2F4EF
:104D300019C1C3F4E6D70401C48F22C4BEF4120023
:104D400004012151E4E0010AE4E0020AE2E0060A7B
:104D5000C9E0030ACDE00E0ACFE0010ACBE0030A66
:104D6000DAE0010AD8A41200E6D70401E86BE96B87
:104D7000FC0E0101176FB20E166F010E4EEC32F0F1
:104D8000880E0101296F130E2A6F000E2B6B2C6BFE
:104D90002D6BF2EC9FF00101306F880E296F130E1E
:104DA0002A6F2B6B2C6B010E2D6FF2EC9FF0010123
:104DB0003051180AD8B412003051160AD8B4120073
:104DC00030511A0AD8B4120030511B0AD8B412005C
:104DD0003051170AD8B412001BEC45F0FFEC44F038
:104DE000D10E0101295D070E2A59F8E3780E04015E
:104DF000E85D000EE959D8B01200BAD7256A000E56
:104E000049EC40F0266E23C01FF024C020F026C0DD
:104E100021F0E8EC2BF0D8B02580040E49EC40F0EE
:104E2000266E23C01FF024C020F026C021F027ECFE
:104E30002CF0D8B02582080E49EC40F0266E23C035
:104E40001FF024C020F026C021F0A9EC2BF0D8B030
:104E500025840C0E49EC40F0266E23C01FF024C0C0
:104E600020F026C021F0A5EC2CF0D8B02586100E3D
:104E700049EC40F0266E23C01FF024C020F026C06D
:104E800021F066EC2CF0D8B025882550120035D0E2
:104E90001BC1D9FF1CC1DAFFDF5013E039D8F7641A
:104EA00003D00800F55005D0F6CFE9FFF7CFEAFFB1
:104EB000EF500101216F1BC1D9FF1CC1DAFFDF18C0
:104EC00018E01BC1D9FF1CC1DAFFDF50216F20D8C9
:104ED000F76403D00800F55005D0F6CFE9FFF7CF0F
:104EE000EAFFEF500101215D1B6F1C6BD8A01C076E
:104EF00012001B4B1C2B1D4B1E2B1F07D8A020077D
:104F000001011F29D8B42029C3E11B6B1C6B1200BF
:104F10001DC1F6FF1EC1F7FF000EF86E0F0E120046
:104F2000E8CF1CF10101185105EC38F015C11DF155
:104F300016C11EF11DC1D9FF1EC1DAFFDF50216F5E
:104F4000216701D012001851AFEC37F015C11FF1E5
:104F500016C120F11DC1D9FF1EC1DAFFDF50DF06E7
:104F6000216F1CC122F11ED0D8902235196F195122
:104F70001F251A6FE86A19BFE86820211B6F020E0F
:104F80001A25D96E000E1B21DA6E2251020DF35044
:104F90001F25E16E000E2021E26EDECFE6FFDDCFA1
:104FA000E5FF222B2151225DD8B01200DDD733D08E
:104FB0001FC0D9FF20C0DAFFDF5012E036D8F764F7
:104FC00003D00800F55005D0F6CFE9FFF7CFEAFF90
:104FD000EF50256E1FC0D9FF20C0DAFFDF1817E0A1
:104FE0001FC0D9FF20C0DAFFDF50256E1ED8F7643E
:104FF00003D00800F55005D0F6CFE9FFF7CFEAFF60
:10500000EF50255C1F6E206AD8A0200612001F4AB0
:10501000202A214A222A2306D8A024062328D8B4ED
:105020002428C6E11F6A206A120021C0F6FF22C0B0
:10503000F7FF000EF86E0F0E12000401286B296BAB
:1050400024D00401C48F040128810401C65125E045
:105050000401288322D00401C48F1FD00401C48F0F
:105060006AEC42F025D8F76403D00800F55005D06B
:10507000F6CFE9FFF7CFEAFFEF500101156F15A555
:105080000CD0010E0401286F08D0040120511F0B21
:10509000D8E0010AE0E0030AE1E00401C4AF120035
:1050A000040EC36F280EC26FC481020EC56F020CBE
:1050B000C7C4F6FFC8C4F7FF000EF86E0F0E12004B
:1050C0000401286B296B2AD00401C48F04012881B4
:1050D0000401C6512BE00401288328D00401C48FA9
:1050E00025D00401C48F06EC42F0C7C4F6FFC8C443
:1050F000F7FF000EF86E0F0EF76403D00800F550AE
:1051000005D0F6CFE9FFF7CFEAFFEF500101006FBE
:1051100000A50CD0010E0401286F08D00401205115
:105120001F0BD2E0010ADAE0030ADBE00401C4AF9E
:105130001200040EC36F280EC26FC481020EC56F29
:10514000020C14B20AAE24D0180E0101176503D068
:105150003C0E176502D0018C01D0019C29D824E0B7
:105160000201AE4BAF2B010115510201AE5D0101F1
:1051700016510201AF590AE30001019E01BC018EE4
:1051800001BE02D0D8901200D88012000001F8D7DA
:105190003E0E0101176102D0019C04D04C0E176530
:1051A00001D0018C05D8DCE10201AE6BAF6BEED70C
:1051B000010E01AC000E0101186F010E01AE000ED0
:1051C000181B120014B20AAE24D0180E0101176584
:1051D00003D03C0E176502D0028001D0029029D87E
:1051E00024E00201B04BB12B010115510201B05D69
:1051F000010116510201B1590AE30001029202B005
:10520000028202B202D0D8901200D88012000001AF
:10521000F8D73E0E0101176102D0029004D04C0E67
:10522000176501D0028005D8DCE10201B06BB16BDB
:10523000EED7010E02A0000E0101186F010E02A2AE
:10524000000E181B1200E8CF27F0E1670AD027A054
:1052500003D0206A220E02D0206A240E1F6E5EEF59
:105260001BF0E10522E10AAC03D01C9027B01C80A2
:1052700000010ABC120019A403D000011CB21200E4
:10528000000106AA120027A008D0206A220E1F6E75
:105290005EEC1BF000011B8E1200206A240E1F6EB4
:1052A0005EEC1BF000011B9E1200E151020AD8A423
:1052B000120019A403D000011CB21200000106AABA
:1052C000120027B0E2D7E9D7E8CF27F0E2670AD08B
:1052D00027A403D0206A2A0E02D0206A2C0E1F6E4B
:1052E0005EEF1BF0E20522E10AAC03D01C9A27B462
:1052F0001C8A00010ABC120019A403D000011CBCC6
:105300001200000106AA120027A408D0206A2A0E63
:105310001F6E5EEC1BF000011C881200206A2C0E30
:105320001F6E5EEC1BF000011C981200E251020A95
:10533000D8A4120019A403D000011CBC1200000163
:1053400006AA120027B4E2D7E9D7E8CF27F0E4672E
:105350000AD027A803D0206A360E02D0206A380E61
:105360001F6E5EEF1BF0E40522E10AAC03D01D9630
:1053700027B81D8600010ABC120019A403D0000141
:105380001DB81200000106AA120027A808D0206A42
:10539000360E1F6E5EEC1BF000011D841200206AA9
:1053A000380E1F6E5EEC1BF000011D941200E451DC
:1053B000020AD8A4120019A403D000011DB81200DB
:1053C000000106AA120027B8E2D7E9D7E8CF27F0F4
:1053D000E3670AD027A603D0206A2E0E02D0206AE7
:1053E000300E1F6E5EEF1BF0E30522E10AAC03D026
:1053F0001D9027B61D8000010ABC120019A403D01D
:1054000000011DB21200000106AA120027A608D052
:10541000206A2E0E1F6E5EEC1BF000011C8E120027
:10542000206A300E1F6E5EEC1BF000011C9E120005
:10543000E351020AD8A4120019A403D000011DB23E
:105440001200000106AA120027B6E2D7E9D714B26B
:105450000AAE24D0180E0101176503D03C0E176563
:1054600002D0018801D0019829D824E00201AC4B78
:10547000AD2B010115510201AC5D01011651020174
:10548000AD590AE30001019A01B8018A01BA02D0BC
:10549000D8901200D88012000001F8D73E0E01010A
:1054A000176102D0019804D04C0E176501D0018815
:1054B00005D8DCE10201AC6BAD6BEED7010E01A8A3
:1054C000000E0101186F010E01AA000E181B120038
:1054D00014B20AAE24D0180E0101176503D03C0E99
:1054E000176502D0018001D0019029D824E0020183
:1054F000A84BA92B010115510201A85D010116510C
:105500000201A9590AE30001019201B0018201B22E
:1055100002D0D8901200D88012000001F8D73E0EB9
:105520000101176102D0019004D04C0E176501D023
:10553000018005D8DCE10201A86BA96BEED7010E52
:1055400001A0000E0101186F010E01A2000E181B30
:10555000120014B20AAE24D0180E0101176503D050
:105560003C0E176502D0018401D0019429D824E0B3
:105570000201AA4BAB2B010115510201AA5D0101E9
:1055800016510201AB590AE30001019601B40186EC
:1055900001B602D0D8901200D88012000001F8D7CE
:1055A0003E0E0101176102D0019404D04C0E176524
:1055B00001D0018405D8DCE10201AA6BAB6BEED708
:1055C000010E01A4000E0101186F010E01A6000ECC
:1055D000181B120033D024C11BF125C11CF126C1B8
:1055E0001DF127C11EF126C115F127C116F1CFEC1F
:1055F00036F015C11FF116C120F1B8EC32F01C5184
:105600001B1105E124C124F125C125F11200242933
:10561000166F000E2521176F26C1F6FF27C1F7FF71
:10562000000EF86E0800F550186F196B18BF1907B7
:10563000EBEC3CF016C124F117C125F125512411E2
:1056400006E024C1D9FF25C1DAFFDF50C4E1246B95
:10565000256B1200F80E0101176FBC0E166F010EBC
:105660004EEC32F00201E32B1BEC45F0FFEC44F072
:10567000E90E0101295D030E2A59F8E3020E020129
:10568000E365020CE36BFB0E0101176F1A0E166F38
:10569000010E4EEC32F0010E01012A6FF40E296F5B
:1056A0002BEC37F01BEC45F0FFEC44F0E90E010168
:1056B000295D030E2A59F8E38E9C8D981BEC45F06A
:1056C000FFEC44F0E90E0101295D030E2A59F8E3CD
:1056D000ACEFC1F0E8CF17F101011751FE0F166FC3
:1056E0000001FA6B0101186B0DD0EE0E01011825B7
:1056F000D96EDA6A0301030EDA22DF5006EC45F0B8
:105700000101182B1651185DF0E30001FA390F0B57
:105710005BEC43F0186FEC0E01011725D96EDA6AC5
:10572000030EDA22DF50181902E0D89012000001AF
:10573000FA510F0B5BEC43F0186FED0E01011725CA
:10574000D96EDA6A030EDA22DF501819EEE1D8803A
:10575000120014B20AAE26D0180E216403D03C0EFB
:10576000216402D0018801D00198010E01A8000E29
:10577000226E010E01AA000E221A26E00201AC4B95
:10578000AD2B1F50AC5D2050AD590AE30001019ACA
:1057900001B8018A01BA02D0D8901200D880120054
:1057A0000001F8D73E0E216002D0019804D04C0EC3
:1057B000216401D00188010E01A8000E226E010EA5
:1057C00001AA000E221ADAE10201AC6BAD6BE8D738
:1057D00014B20AAE26D0180E216403D03C0E216408
:1057E00002D0018001D00190010E01A0000E226EB6
:1057F000010E01A2000E221A26E00201A84BA92BDD
:105800001F50A85D2050A9590AE30001019201B080
:10581000018201B202D0D8901200D880120000019B
:10582000F8D73E0E216002D0019004D04C0E2164C6
:1058300001D00180010E01A0000E226E010E01A216
:10584000000E221ADAE10201A86BA96BE8D714B2A4
:105850000AAE26D0180E216403D03C0E216402D07B
:10586000018401D00194010E01A4000E226E010EEC
:1058700001A6000E221A26E00201AA4BAB2B1F50F4
:10588000AA5D2050AB590AE30001019601B40186DC
:1058900001B602D0D8901200D88012000001F8D7CB
:1058A0003E0E216002D0019404D04C0E216401D040
:1058B0000184010E01A4000E226E010E01A6000E4D
:1058C000221ADAE10201AA6BAB6BE8D714B20AAE76
:1058D00026D0180E216403D03C0E216402D0028031
:1058E00001D00290010E02A0000E226E010E02A253
:1058F000000E221A26E00201B04BB12B1F50B05D02
:105900002050B1590AE30001029202B0028202B2B1
:1059100002D0D8901200D88012000001F8D73E0EB5
:10592000216002D0029004D04C0E216401D002808C
:10593000010E02A0000E226E010E02A2000E221A1B
:10594000DAE10201B06BB16BE8D714B20AAE26D02F
:10595000180E216403D03C0E216402D0018C01D0CA
:10596000019C010E01AC000E226E010E01AE000E74
:10597000221A26E00201AE4BAF2B1F50AE5D205025
:10598000AF590AE30001019E01BC018E01BE02D0A5
:10599000D8901200D88012000001F8D73E0E216086
:1059A00002D0019C04D04C0E216401D0018C010E68
:1059B00001AC000E226E010E01AE000E221ADAE1D9
:1059C0000201AE6BAF6BE8D7FC0E176FA10E166F1E
:1059D000010E4EEC32F0300E0101296F750E2A6F68
:1059E000000E2B6B2C6B2D6BF2EC9FF00101306FD6
:1059F00030510C0A03E03051090A01E1000C30C1BA
:105A000031F1300E296F750E2A6F2B6B2C6B010E46
:105A10002D6FF2EC9FF0080AF1E1010131510B0A00
:105A20000AE11BEC45F0FFEC44F0890E0101295D11
:105A3000130E2A59F8E331510A0A03E031510B0AD7
:105A4000DDE131511200010E05EC38F015C118F1FD
:105A500016C119F118C1D9FF19C1DAFFDF6A020EA8
:105A600005EC38F015C118F116C119F118C1D9FFAC
:105A700019C1DAFFDF6A030E05EC38F015C118F121
:105A800016C119F118C1D9FF19C1DAFFDF6A040E76
:105A900005EC38F015C118F116C119F118C1D9FF7C
:105AA00019C1DAFFDF6A050E05EC38F015C118F1EF
:105AB00016C119F118C1D9FF19C1DAFF000EDF6E46
:105AC000000C1A0ECBEC42F00301B26BB36B0294E4
:105AD0002FD0C4ECE7F002A42BD002940201CE67D1
:105AE00001D026D0080E01011C6FA00E1B6FFD0E09
:105AF0001E6F6A0E1D6F206B070E1F6F47EC27F09D
:105B00001C511B1102E1D8901200080E01011C6FFC
:105B1000A00E1B6FFB0E1E6F380E1D6F206B090E43
:105B20001F6F47EC27F01C511B1102E1D8801200B7
:105B3000310E0301B25D750EB359F8E2CAD7E8CF52
:105B400021F1196B580E186F90EC2EF0226F1F0583
:105B500007E1186B580E176F2251FE0B21110CD064
:105B60001F51020A0CE1186B580E176FD89021359F
:105B7000206F2251FD0B15D0196F50EF35F01F51DA
:105B8000030A05E1186B0FD82251FB0B0AD01F51F5
:105B9000040AD8A41200186B06D8D89020372251D6
:105BA000F70B2011E9D7580E176F21C120F1D890BB
:105BB0002037D8902037580C15C1D9FF16C1DAFF0D
:105BC00010EE06F028D810EE05F01551E12616511A
:105BD000E222DFCFE7FF20EE04F01551D92616515F
:105BE000DA2215C1E1FF16C1E2FFDFCFE7FF20EEA9
:105BF00002F01551D9261651DA2210EE04F00BD816
:105C0000D051DF6E20EE02F01551D9261651DA225E
:105C1000CFC1DFFF12001551E1261651E222DFCF7E
:105C2000E7FF20EE01F01551D9261651DA221200B5
:105C3000E8CF51F152C615F10101515131EC40F05C
:105C400002E2D890120000010CAAFBD78A8C040152
:105C5000DA6BDB6B00011A8C80ECF5F00101513935
:105C6000F00B506F030E406F505188ECF0F040C1C4
:105C70004EF141C14FF10601525198EC44F002E25D
:105C8000D8801200515169EC3DF00101506F4EC1B6
:105C900039F14FC13AF151C13BF150C13CF1030E12
:105CA0003D6F56EC34F0ECD71A6B18AF06D0176D79
:105CB000181FD8B0182B010E1A6F16AF06D0156D2D
:105CC000161FD8B0162B010E1A1B1B6B1C6B18511C
:105CD00017111BE0010E196F04D0D8901737183731
:105CE000192B18AFFAD7D8901B371C371751155DF1
:105CF0001851165905E31751155F1851165B1B8192
:105D0000D89018331733192FEED71A5104E01B6DB2
:105D10001C1FD8B01C2B1BC115F11CC116F11200A1
:105D20000A0E01011D6FA00E1E6F30D01D07D36B30
:105D30009AEC41F001011E510CEC3DF00101D367DA
:105D400017D019510CEC3DF0010118510CEC3DF04D
:105D50009AEC41F001011E811E510CEC3DF0000E49
:105D6000C6EC3DF01C6F6AEC3FF001011C511200C3
:105D7000070E1B6FD00E1A6F01D000F001011A0739
:105D8000D8A01B071A29D8B41B29F7E11D51800A96
:105D90007F0FCCE2000CE8CF22F0216A22C020F075
:105DA000010E20161F50010B2018D8A4218022C0FC
:105DB00020F0020E20161F50020B2018D8A42182BA
:105DC00022C020F0040E20161F50040B2018D8A467
:105DD000218422C020F0080E20161F50080B201826
:105DE000D8A4218622C020F0100E20161F50100BC0
:105DF0002018D8A4218822C020F0200E20161F5081
:105E0000200B2018D8A4218A21501200E8CF51F18C
:105E100067C615F10101515131EC40F002E2D89012
:105E2000120080ECF5F001015139F00B506F010EBA
:105E30002B6F2C6B030E33ECD4F0F1E3240E010135
:105E4000406F505188ECF0F040C14EF141C14FF12C
:105E50000601675198EC44F002E2D88012005151DB
:105E600069EC3DF00101506F4EC139F14FC13AF17B
:105E700051C13BF150C13CF1030E3D6F56EC34F083
:105E8000ECD7E8CF51F168C615F10101515131EC61
:105E900040F002E2D890120080ECF5F00101513997
:105EA000F00B506F010E2B6F2C6B040E33ECD4F003
:105EB000F1E3250E0101406F505188ECF0F040C134
:105EC0004EF141C14FF10601685198EC44F002E2F5
:105ED000D8801200515169EC3DF00101506F4EC164
:105EE00039F14FC13AF151C13BF150C13CF1030EC0
:105EF0003D6F56EC34F0ECD7E8CF51F166C615F1A2
:105F00000101515131EC40F002E2D890120080ECD6
:105F1000F5F001015139F00B506F010E2B6F2C6B16
:105F2000020E33ECD4F0F1E3230E0101406F505127
:105F300088ECF0F040C14EF141C14FF106016651CD
:105F400098EC44F002E2D8801200515169EC3DF027
:105F50000101506F4EC139F14FC13AF151C13BF1CE
:105F600050C13CF1030E3D6F56EC34F0ECD7080EF7
:105F7000236F33D00E0E256F1F25216F000E2021B9
:105F8000226F12D02507C10E01012525D96EDA6ACC
:105F9000010EDA222107D8A0220721C118F122C15F
:105FA00019F190EC2EF0DF6E2567ECD7246B256B92
:105FB000C10E2525D96EDA6A010EDA22DF50241BC4
:105FC000252B2551800A730FF3E3245121EECEF0E7
:105FD000DF6202D0D880120023072367CBD7D89086
:105FE00012000401E86BE96BF90E0101176F010E55
:105FF000166F010E4EEC32F0880E0101296F130E60
:106000002A6F000E2B6B2C6B2D6BF2EC9FF00101B5
:10601000306F30512D0A06E1130E2A6F880E296F5A
:106020002BEF37F0130E2A6F880E296F2BEC37F009
:106030001BEC45F0FFEC44F0D10E0101295D070E89
:106040002A59F8E3B40E0401E85D000EE959CCE3E7
:10605000FF00CAD7E8CF51F153C615F101015151E4
:1060600031EC40F002E2D89012008A9C0401DA6B15
:10607000DB6B00011A9C80ECF5F001015139F00B4B
:10608000506F040E406F505188ECF0F040C14EF15B
:1060900041C14FF10601535198EC44F002E2D8801F
:1060A0001200515169EC3DF00101506F4EC139F1C0
:1060B0004FC13AF151C13BF150C13CF1030E3D6F6C
:1060C00056EC34F0ECD720EE02F01551D9261651DB
:1060D000DA22DF50196F20EE02F024D8E750176F54
:1060E00010EE02F01551E1261651E222E750186F2A
:1060F00018390F0B1711DF6E20EE01F013D8DFCF28
:10610000E7FF20EE01F01551D9261651DA22DF6A99
:1061100020EE01F01551D9261651DA221939F00B6B
:10612000DF6E12001551D9261651DA2215C1E1FF92
:1061300016C1E2FF1200E8CF9DF2000108BA050C7B
:10614000000115B2050C9CC29EF21DD09D6704D0C3
:1061500083EC37F002019F6F9F5119E09E6701D0D9
:1061600016D09F51040A03E09F51020AD8B42AECCA
:106170002BF01BEC45F0FFEC44F0990E0101295D7A
:106180003A0E2A59F8E302019E079E29DFE19F514A
:10619000040A03E09F51020AD8B42AEC2BF0020152
:1061A0009F511200E8CF51F155C615F1010151512F
:1061B00031EC40F002E2D890120000010CACFBD7A9
:1061C0008A8E80ECF5F001015139F00B506F060E0C
:1061D000406F505188ECF0F040C14EF141C14FF199
:1061E0000601555198EC44F002E2D880120051515A
:1061F00069EC3DF00101506F4EC139F14FC13AF1E8
:1062000051C13BF150C13CF1030E3D6F56EC34F0EF
:10621000ECD7E8CF25F12507DF5127EC43F01F6FBE
:10622000DE5127EC43F0206F2039F00B1F11236F54
:106230002551220DF80EF324186F3F0EF420196F2C
:1062400090EC2EF0246F2451231902E0D890120014
:106250002551220DF90EF324216F3F0EF420226FF9
:1062600021C118F122C119F190EC2EF0266F010E18
:106270002665ECD7100E266501D0E8D7D88012002D
:10628000FC0E176FC20E166F010E4EEC32F0880E28
:106290000101296F130E2A6F000E2B6B2C6B2D6BD7
:1062A000F2EC9FF00101306F30513A0AD8A412008D
:1062B000070E306F8F0E01013025D96EDA6A060E97
:1062C000DA22350E3025E16EE26A070EE222DFCFD8
:1062D000E7FF302B3051800A660FECE307014F6B6C
:1062E000130E01012A6F880E296F2BEF37F004017E
:1062F000C48F0F014D6B4E6B0401BE6B22C4BDF405
:106300000401226704D0100E0401CD6F100C200E82
:106310000401CD6F0401CE6B4B0ECF6FD06BD16BF0
:10632000D26BD36B080ED46F010ED56F0401CC6B0A
:10633000CC8F0401B16B0401B06B1A0E0F014E6FCC
:106340000401148D149F1E0E0F014F6F04011C8D4C
:106350001C9F188D189F13EF44F0E8CF31F13DECEE
:106360001FF0D8B03DEC1FF0D8B012000101326B25
:10637000316712D06A0E3225176F186B130E18236F
:10638000280E01013225D96EDA6A060EDA22DF50B4
:10639000196F50EC35F011D0790E3225176F186B4C
:1063A000130E1823280E01013225D96EDA6A060E63
:1063B000DA22DF50196F50EC35F00101322B0E0E4E
:1063C0003265D6D70E0C0401C48F0F014D6B4E6B96
:1063D0000401BE6B22C4BDF40401226704D0100E78
:1063E0000401CD6F100C200E0401CD6F0401CE6BA3
:1063F0004B0ECF6FD06BD16BD26BD36B080ED46FBB
:10640000010ED56F0401CC6BCC8F0401B16B04017C
:10641000B06B1A0E0F014E6F0401148D149F1E0EE7
:106420000F014F6F04011C8D1C9F188D189F06EFE4
:1064300044F0E8CF27F16DC615F10101275131EC89
:1064400040F002E2D89012000501D351080AFAE1A7
:106450001F0ED325D96EDA6A050EDA22DF6A230E03
:106460000101256F050E266F25C11BF126C11CF108
:10647000A2EC1AF01BC128F11CC129F128C11FF19F
:1064800029C120F1AFEC3EF0DDE3500E206FD20EBB
:106490001F6F57EC37F0FF00D8801200E8CF18F1DB
:1064A0000101185118E0410ECBEC42F0540ECBEC38
:1064B00042F011D001011FD8F76403D00800F55055
:1064C00005D0F6CFE9FFF7CFEAFFEF50CBEC42F073
:1064D0000101164B172B01010ED8F76403D00800F9
:1064E000F55005D0F6CFE9FFF7CFEAFFEF500009EE
:1064F000D8B41200DFD716C1F6FF17C1F7FF000EA0
:10650000F86E0F0E1200E8CF27F127C115F1166BB8
:10651000270E186F100E176F16EC41F01C51640D0A
:10652000F3CF1FF1F4CF20F11D510A0DF3501F25B9
:10653000216FF4502021226F15512125236F165110
:106540002221246F1BC115F1166B030E186FE80E84
:10655000176F16EC41F015512325256F1651242194
:10656000266F1E5125251B6F000E26211C6F120061
:1065700029D01DC1F6FF1EC1F7FF000EF86E0800FE
:10658000F55020EC44F0216F1BC1D9FF1CC1DAFF8C
:10659000DF5020EC44F0226F2151225D236F010176
:1065A000236706D01BC1D9FF1CC1DAFFDF5006E10B
:1065B00023511B6F1C6B1BBF1C0712001B4B1C2B9A
:1065C0001D4B1E2B1F07D8A0200701011F29D8B47F
:1065D0002029CFE11B6B1C6B1200049C9CA29CB475
:1065E000048CAACFF9F004AC05D09C989C880001DB
:1065F0000592120005820CAE0AD0000E0201DD25C4
:10660000D96EDA6A090EDA22F9C0DFFFDD2B0BAA98
:1066100004D00001F951CCEF16F000011EB4D4EC07
:10662000F4F0000113BC02D0000117B250EC10F0DE
:1066300005A404D00001F9511AEC3AF00001F95117
:1066400078EFCAF01A6B16AF06D0156D161FD8B0CA
:10665000162B010E1A6F18AF04D0176D181FD8B083
:10666000182B1851171117E0010E196F04D0D8908C
:1066700017371837192B18AFFAD71751155D18515E
:10668000165904E31751155F1851165BD89018334B
:106690001733192FF2D71A5104E0156D161FD8B011
:1066A000162B15C115F116C116F11200E8CF51F1E4
:1066B00056C615F10101515131EC40F002E2D8907B
:1066C00012008A9E80ECF5F001015139F00B506FF9
:1066D000070E406F505188ECF0F040C14EF141C1BF
:1066E0004FF10601565198EC44F002E2D8801200B6
:1066F000515169EC3DF00101506F4EC139F14FC16C
:106700003AF151C13BF150C13CF1030E3D6F56ECE3
:1067100034F0ECD7E8CF51F164C615F101015151C5
:1067200031EC40F002E2D890120080ECF5F001016B
:106730005139F00B506F210E406F505188ECF0F042
:1067400040C14EF141C14FF10601645198EC44F053
:1067500002E2D8801200515169EC3DF00101506F06
:106760004EC139F14FC13AF151C13BF150C13CF139
:10677000030E3D6F56EC34F0ECD7E8CF51F163C611
:1067800015F10101515131EC40F002E2D8901200B4
:1067900080ECF5F001015139F00B506F200E406F85
:1067A000505188ECF0F040C14EF141C14FF106016B
:1067B000635198EC44F002E2D8801200515169EC28
:1067C0003DF00101506F4EC139F14FC13AF151C155
:1067D0003BF150C13CF1030E3D6F56EC34F0ECD769
:1067E000E8CF51F162C615F10101515131EC40F091
:1067F00002E2D890120080ECF5F001015139F00B63
:10680000506F190E406F505188ECF0F040C14EF1BE
:1068100041C14FF10601625198EC44F002E2D88088
:106820001200515169EC3DF00101506F4EC139F138
:106830004FC13AF151C13BF150C13CF1030E3D6FE4
:1068400056EC34F0ECD7E8CF51F165C615F10101F3
:10685000515131EC40F002E2D890120080ECF5F09A
:1068600001015139F00B506F220E406F505188ECEE
:10687000F0F040C14EF141C14FF10601655198EC75
:1068800044F002E2D8801200515169EC3DF0010160
:10689000506F4EC139F14FC13AF151C13BF150C176
:1068A0003CF1030E3D6F56EC34F0ECD739513E6F9E
:1068B000030E3A153F6F3DC140F1416B0D0ED8906C
:1068C00040374137E82EFBD73BC142F1436B0A0EFC
:1068D000D89042374337E82EFBD740514211446FDE
:1068E00041514311456F3E514411466F3F5145118F
:1068F000476F3C51D8A4478F46C130F147C131F1B1
:106900003BC132F198EC17F002E3D8801200D89026
:106910001200E8CF56F150C615F10101565131EC85
:1069200040F002E2D8901200565169EC3DF00101AE
:10693000556F56C11FF15551010A9FEC2DF080ECA7
:10694000F5F001015639F00B556F010E406F5551AE
:1069500088ECF0F00601505198EC44F002E2D88047
:106960001200565169EC3DF00101556F55C14EF1D1
:10697000565113ECE6F0F3D7416A0301EE0502E04D
:10698000D89012000101016BEE0E01010125D96EB4
:10699000DA6A0301030EDA22DF50F66F0101006BA1
:1069A0000301F6514118F76F0301F73302E3180EA4
:1069B000411A00F0000141330301F633D890010180
:1069C000002B070E0065ECD7012B060E0165DCD706
:1069D0000301F5514118D4E1D88012000101326B56
:1069E000E4EC2CF00101336F33510B0A03E172EC3C
:1069F00036F020D8335102E032511AE01BEC45F05A
:106A0000FFEC44F0990E0101295D3A0E2A59F8E392
:106A1000326BE4EC2CF00101336F33510B0A03E1CC
:106A200072EC36F007D8335102E0325101E0010C2C
:106A300079EFF3F0010ED8A0000E326F12000001C2
:106A40000DAC000C01011C6B15D0000E01011C25C2
:106A5000D96EDA6A0A0EDA221CC117F1186B17BF59
:106A6000180717511525E16E18511621E26EDFCF78
:106A7000E7FF1C2BE4C217F10101186B1CC119F1CF
:106A80001A6B19BF1A071A51800A1B6F1751195D2B
:106A90001851800A1B59D9E30D9C0201E4511200E0
:106AA0000A0E1D6FA00E1C6F26D01D07D36B9AEC2B
:106AB00041F001011C510CEC3DF00101D3670DD0F8
:106AC00018510CEC3DF0010117510CEC3DF00101A7
:106AD00019510CEC3DF06AEF3FF0070E1B6FD00E22
:106AE0001A6F01D000F001011A07D8A01B071A295C
:106AF000D8B41B29F7E11D51800A7F0FD8A01200DE
:106B0000D4D7E8CF51F10101510502E0D89012002D
:106B100080ECF5F001015139F00B506F010E2B6F35
:106B20002C6B33ECD4F0F2E3230E0101406F505193
:106B300088ECF0F0010140C14EF141C14FF15151DB
:106B400069EC3DF00101506F4EC139F14FC13AF18E
:106B500051C13BF150C13CF1030E3D6F56EC34F096
:106B6000D88012002DC127F12EC128F12FC129F1A3
:106B700030C12AF188EC3DF00201D05122E003013E
:106B8000AA4BAB2BD890AA350101316F280E3125C5
:106B9000D96EDA6A080EDA22F8C4DEFFF9C4DDFF26
:106BA0000301D890AA350101316F000E3125D96E4D
:106BB000DA6A0801080EDA22000EDE6EDD6ED88079
:106BC000000CD8901200E8CF4EF180ECF5F00201F5
:106BD000F039F00B0101516F10D0820E406F51510E
:106BE00088ECF0F005D0810E406F515188ECF0F048
:106BF00040C14FF141C150F104D04E51EEE0010AC5
:106C0000F2E00201F05169EC3DF00101516F4FC11A
:106C100039F150C13AF1F0C23BF151C13CF1030EE0
:106C20003D6F56EF34F01FC1F8F21B9813D00101ED
:106C3000200507E11DC115F11EC116F136EC3FF02C
:106C400006D01DC115F11EC116F11FEC35F0020171
:106C5000D46FF76B0201D46702D0F867E8D7F86702
:106C600003D000011B88000CD407F75101011D253A
:106C7000D96E000E1E21DA6EDF50216F0201F72B54
:106C800001012151120046840101186B520E176F49
:106C9000E7C119F150EC35F00101196B520E186F74
:106CA00090EC2EF00201F96F0101E56BB8C319F108
:106CB000B9C31AF123EC23F0E76F14B20AAE06D081
:106CC0000201F951E00B0101E71905D00101E7517B
:106CD0000201F9190101E56FE5C1ECF3148E000121
:106CE00046941200FB0E176F2E0E166F010E4EEC1F
:106CF00032F0E80E0101296FFD0E2A6F000E2B6B9A
:106D00002C6B2D6BF2EC9FF00101306F30510C0AAF
:106D100011E03051090A0EE03051080A0BE0E80E8C
:106D2000296FFD0E2A6F2B6B2C6B010E2D6FF2EC71
:106D30009FF0EAD73051080A02E1D8901200D880BB
:106D40001200F2943F6602D07CEF44F03F0402E16F
:106D500067EF44F03F50020A02E172EF44F03F5007
:106D6000030A02E120EF3EF03F50040A02E130EF57
:106D700038F03F50050A02E115EF43F03F50060A94
:106D800002E103EF43F03F50070A02E101EF3FF059
:106D90003F50080A02E17CEF39F03F6A120015C14A
:106DA00019F116C11AF101011951176F1A51186F13
:106DB000194B1A2B17C1F6FF18C1F7FF000EF86E1A
:106DC0000F0EF76403D00800F55005D0F6CFE9FFA9
:106DD000F7CFEAFFEF500009E6E1010119C117F111
:106DE0001AC118F11551175F1651185BFF0E1725C0
:106DF000156FFF0E1821166F120037C12BF138C125
:106E00002CF139C12DF13AC12EF1ACEC04F002E2C3
:106E1000D890120000010D9C1BEC45F013D000012E
:106E20000DAC10D00A0E0101256F000E246F37C182
:106E300026F138C127F160EC08F002E3D880120097
:106E400000010D9CFFEC44F0E90E0101295DFD0EEF
:106E50002A59DEE2E4D70301B66BB76B01012B6B55
:106E60001BD0C4ECE7F0EAEC44F016E317EC45F075
:106E700001012C6F0DD02C5100EC41F00DE301010C
:106E80002B2B0AD02C51BEEC40F006E3D880120028
:106E90002B51F1E0010AF6E00301B6510101295D31
:106EA0000301B75101012A59DCE2D89012001F29D1
:106EB000186F000E2021196F90EC2EF0216F1FC16A
:106EC00018F120C119F190EC2EF0236F2151226F9F
:106ED000224B232B2229D8B4232902E1226B236BD6
:106EE0001FC117F120C118F12351196F50EC35F073
:106EF000010E01011F25176F000E2021186F22C1FE
:106F000019F150EF35F0EEEC34F0BF6FBF5102E0F5
:106F1000BF5112001EA408D00301CD6B138C19823F
:106F200016800001039E000C000117823BEC21F04B
:106F30000101BF6F1792BF0503E0BF51030A0EE1C5
:106F40000301CD6B138C19821680039E0101BF5182
:106F5000030AE9E1010E0CECC4F0000C020CE8CFCE
:106F600017F1170506E1080E0101166F500E156F97
:106F700012001751020A06E1090E0101166F640E94
:106F8000156F12001751030A06E10A0E0101166F70
:106F9000A00E156F12001751040A06E10B0E010135
:106FA000166FA00E156F1200060E0101166FF10E7E
:106FB000156F120061EC40F0186F20EE03F01651CF
:106FC000D9261751DA2218C1DFFF61EC40F0186FA3
:106FD00020EE02F01651D9261751DA2218C1DFFF30
:106FE00061EC40F016C1D9FF17C1DAFFDF6E61EC2A
:106FF00040F0186F20EE01F01651D9261751DA2211
:1070000018C1DFFF000109921200E8CF17F101015A
:10701000170505E1020E166FFB0E156F12001751D2
:10702000020A06E1020E0101166FFC0E156F120036
:107030001751030A06E1020E0101166FFD0E156FCE
:1070400012001751040A06E1020E0101166FFE0E2E
:10705000156F1200020E0101166FFF0E156F120060
:10706000416609D02F0E0101016F100E006FDBEC9D
:107070003BF03F6A12004106010E0101016F690EEB
:10708000006FDBEC3BF086A6120000F086A6120033
:1070900000F086A6120011A206D0010E0401D76FDF
:1070A000F40ED66FE6D7330E0301EE6F080E406E76
:1070B0003F2A15EF43F0040E0101196F030E186FFC
:1070C00090EC2EF0216F040E196F020E186F90ECE9
:1070D0002EF0236F2151226FFF0E225D000E2359E7
:1070E00004E2040E206F1F6F040C040E196F010ED2
:1070F000186F90EC2EF0216F040E196F000E186BB4
:1071000090EC2EF0206F21511F6F1200E8CF1BF181
:107110001A6B1C6B0AD0E90E01011C25D96EDA6AC4
:10712000000EDA22DF501A1B1C2B1BC115F1166B47
:107130001CC117F1186B17BF18071851800A196F77
:107140001551175D1651800A1959E5E3E90E010141
:107150001B25D96EDA6A000EDA221AC1DFFF12008F
:107160009E940201EB6B000116BE12000301E69132
:1071700082ACE681080EE72BE76103D0D890E637B2
:10718000080CE76BF80E0201EA25D96EDA6A030EE5
:10719000DA22E6C3DFFFEA2B060EEA65060CEA6B8D
:1071A000829C949C829C168E168C8F800001138882
:1071B00012000251040A02E0D890120000C1D9FF67
:1071C00001C1DAFFDF504E0AF7E120EE01F0005175
:1071D000D9260151DA22DF50100AEEE120EE02F04A
:1071E0000051D9260151DA22DF505E0AE5E120EE96
:1071F00003F00051D9260151DA22DF50AC0ADCE15C
:10720000D8801200E8CF1AF1060E0301EE6F0101DB
:10721000D0510301EF6FCFC1F0F3F36B7F0E01018B
:107220001A25D96EDA6A060EDA22DF50196F19AD07
:1072300005D01A510F0B0301F21304D01A39F00BC9
:107240000301F313F46BF56B030E0101176FEE0EE0
:10725000166FD4EF40F07F0E010120D8DB8E18AC02
:1072600003D07F0E1BD8DB8C960E0101D625176F3D
:10727000186B020E18237F0ED625D96EDA6A060E19
:10728000DA22DF50196F50EC35F0530E0301F16F25
:10729000100EF26F0101D65102EF39F0D625D96EEA
:1072A000DA6A060EDA22000C010E01012A6FF40ED2
:1072B000296F2BEC37F0F60E0101176F640E166F75
:1072C000010E4EEC32F0030E01012A6FE80E296F19
:1072D0002BEC37F0F60E0101176F580E166F010EEA
:1072E0004EEC32F0030E01012A6FE80E296F2BECF1
:1072F00037F00001199C1200402E13D0BCEC34F082
:107300000DE31182010E0401D76FF40ED66F1196B2
:107310001B923C0E0201CD6F010E456E3F6A7CEF61
:1073200044F00301F5330301F4330301F3330301A4
:10733000F2330301F1330301F0330301EF330301AF
:10734000EE333F0601EF3FF0E8CF56F151C615F19D
:107350000101565131EC40F002E2D890120080EC6D
:10736000F5F001015639F00B556F020E406F555183
:1073700088ECF0F00601515198EC44F002E2D8801C
:107380001200565169EC3DF00101556F55C14EF1A7
:10739000565113ECE6F0F3D7E8CF21F12107215144
:1073A000330D890EF324226F130EF420236F246B08
:1073B000F50E01012425D96EDA6A0601060EDA22DD
:1073C00022C118F123C119F190EC2EF0DF6E224B8F
:1073D000232B242B030E2465EBD7060E0101206F0F
:1073E000F50E1F6F1200DE6BDF6BC12903E1390E52
:1073F000DE6FDF6FC151030A0BE1C6390F0B5BEC87
:1074000043F0DE6FC6510F0B5BEC43F0DF6F1200F1
:10741000C151060A04E0C151070AD8A41200C5519F
:107420000F0B5BEC43F0DE6FC6390F0B5BEC43F0E8
:10743000DF6F1200E8CF1FF01F502B0A03E102019B
:10744000C66B12001E0E0201C625D96EDA6A070E3F
:10745000DA221FC0DFFFC62BC651160AD8A41200BD
:1074600007011E51430A0AE11F51470A07E1205153
:10747000530A04E121514E0AD8B4120000010594C8
:10748000120004012051800AD8A41200800E0401C9
:10749000C46F13D0EB0E0401C36FD50EC26F120E72
:1074A000C56F120CEB0E0401C36F920EC26F430E38
:1074B000C56F430C0401C46B120004012351010A7F
:1074C000E9E0030AEFE0010AD8A41200F3D715C1DE
:1074D0001BF116C11CF102D01B4B1C2B1BC1D9FF89
:1074E0001CC1DAFFDF50F8E11751196F18511A6FFC
:1074F000174B182B19C1F6FF1AC1F7FF000EF86ED3
:107500001BC1D9FF1CC1DAFF1B4B1C2B0800F5CF98
:10751000DFFFDF50D8B41200E7D704012051800A02
:10752000D8A41200800E0401C46F13D0EB0E040126
:10753000C36FD50EC26F120EC56F120CEB0E040195
:10754000C36F920EC26F430EC56F430C0401C46B30
:10755000120004012351010AE9E0030AEFE0010AE5
:10756000D8A41200F3D7C76A300EC66E0101166B9D
:10757000176B186B196B550E1A6F7EEC42F0166B79
:10758000010E176F186B196BAA0E1A6F7EEC42F082
:10759000000E166B176B186B196BEAEC40F0550A6E
:1075A000D8A41200166B010E176F186B196BEAEF57
:1075B00040F0E8CF5DF104C515F101015D5131ECFA
:1075C00040F002E2D890120080ECF5F001015D3944
:1075D000F00B5C6F790E406F5C5188ECF0F00001AD
:1075E000118CF8EC44F02AEC2BF01B901682010170
:1075F000DD5103E0DD050201E66FD8801200F29450
:10760000EB0E0101016F500E006FDBEC3BF000014F
:1076100011B00ED086B602D0416A1200412A415004
:10762000330AD8A41200416A1180000111821200AD
:1076300086B6F2D7412A4150330AD8A41200416AD3
:1076400011900001118212001A6B1B6B1851171157
:107650001BE0010E196F04D0D89017371837192B7B
:1076600018AFFAD7D8901A371B371751155D185134
:10767000165905E31751155F1851165B1A81D890FA
:1076800018331733192FEED71AC115F11BC116F194
:1076900012001DC115F11EC116F11FC117F120C145
:1076A00018F154EC2EF015C123F116C124F11DC1BF
:1076B00015F11EC116F11FC117F120C118F122ECFE
:1076C00033F015C121F116C122F121C11DF122C1F2
:1076D0001EF123C11FF124C120F112007F0E010110
:1076E000D625D96EDA6A060EDA22C00EDF167F0EB4
:1076F000D62512D81EAF2BEF39F07F0ED6250CD829
:107700001EAD05D0000118BC12002BEF39F00001AE
:1077100018AC12002BEF39F0D96EDA6A060EDA22B5
:10772000DF501E6F1200F90E0101176FFE0E166F6B
:10773000010E4EEC32F01BEC45F00CD0EAEC44F0BC
:1077400009E317EC45F001012B6F2B513E0A02E1D2
:10775000D8901200FFEC44F0890E0101295D130E50
:107760002A59ECE31B0ECBEC42F0D8801200040146
:10777000FF51D8A41200000112B012001F6A0101CB
:10778000E6A102D006841F2A0101E6A302D00684E6
:107790001F2A0101E6A502D006841F2A1F6601D018
:1077A000069407BC02D014AC03D000010888120074
:1077B000000108981200D59E0051026F0151036F1D
:1077C000046B056B02510008066F000E0355076F2E
:1077D000010E0455086F000E0555096F07C106F12B
:1077E00008C107F109C108F1096B08BF0969065111
:1077F000D76E00510008D66ED58E1200E8CF15F175
:10780000150501E1010C1551020A01E1020C1551A7
:10781000040A01E1030C1551080A01E1040C155199
:10782000100A01E1050C1551200A01E1060C155161
:10783000400A01E1070C1551800A01E1080C000C17
:107840001BD0C7C4F6FFC8C4F7FF000EF86EC9C44A
:10785000D9FFCAC4DAFF0F0EF76403D00800F55051
:1078600005D0F6CFE9FFF7CFEAFFEF50DF6E040156
:10787000C74BC82BC94BCA2B0401CB07CB29D8B4A3
:107880001200DFD7456602D0B0EF43F0450402E1B5
:107890002DEF44F04550020A02E1B3EF44F04550A9
:1078A000030AF6E04550040AF8E04550050AF0E006
:1078B0004550060A02E151EF44F04550070A02E143
:1078C00045EF44F0456A12001BD0C7C4F6FFC8C498
:1078D000F7FF000EF86EC9C4D9FFCAC4DAFF0F0E55
:1078E000F76403D00800F55005D0F6CFE9FFF7CFD5
:1078F000EAFFEF50DF6E0401C74BC82BC94BCA2B00
:107900000401CB07CB29D8B41200DFD786EC44F0B2
:10791000000112805BEC38F00201E56B149A010162
:10792000010E226F3A0E216FF90E246FB10E236FF4
:10793000130E266FFA0E256F86ECCEF021514B6F99
:10794000010E166F3A0E156F4BC117F1DDEF43F0C4
:107950002AC12BF11CD026C117F127C118F128C16B
:1079600019F129C11AF12BC11BF1E8EC20F02C6FA1
:10797000D351D8A412002C512627000E27232C51B6
:10798000010DF3502827000E29232C512B5F2B6764
:10799000E2D71200040E0101186F176B196F50EC3B
:1079A00035F0040E0101186F010E176F040E196FE8
:1079B00050EC35F0040E0101186F020E176F000E27
:1079C000196B50EC35F0040E0101186F030E176FA0
:1079D000196B50EF35F0185120EC44F0186F196B0B
:1079E00018BF190710D016C1D9FF17C1DAFFDF5031
:1079F00020EC44F0181905E116C116F117C117F172
:107A00001200164B172B16C1D9FF17C1DAFFDF5032
:107A1000EAE1166B176B1200E8CF15F1166B15AF84
:107A200003D00001038802D00001039877EC3EF0F8
:107A30000101D8901537162B1651800A780FEFE305
:107A400056EC42F0000103A612000101D3671200B8
:107A5000030ED36F030C000109B2120020C0D9FF3E
:107A600021C0DAFFDF50D1EC3FF020EE01F02050D2
:107A7000D9262150DA22DF50D1EC3FF020EE02F07F
:107A80002050D9262150DA22DF50D1EC3FF00001FE
:107A90000E8412001F511E1117E0010E206F04D03A
:107AA000D8901E371F37202B1FAFFAD71E511C5DF1
:107AB0001F511D5904E31E511C5F1F511D5BD890BF
:107AC0001F331E33202FF2D71CC11CF11DC11DF125
:107AD0001200E8CF22F10101196B580E186F90ECDB
:107AE0002EF0216F2251030A03E100011EB8010CA0
:107AF00022C11FF1FF0E01011F2721C120F11F2B01
:107B000002D0D89020331F2FFCD72051010B120038
:107B100027C122F128C123F129C124F12AC125F16D
:107B2000A7EC3DF02B6F2B39F00B2C6F27C122F106
:107B300028C123F129C124F12AC125F1A7EC3DF088
:107B40002C272C510201D02701012C51120022C1F7
:107B50001DF123C11EF124C11FF125C120F113EC39
:107B600036F00101266F0BAA04D026C1A9FFA8A2F6
:107B7000FED70101266701D0000C400E266503D018
:107B80002651C90F12002651D00F1200E8CF15F16F
:107B90000101176B166B56EC42F00101D8901737B4
:107BA000179103B61781162B1651800A780FF3E34D
:107BB000155107E00001039877EC3EF001011751E1
:107BC000120000010388F8D7636A626A9F0E0F01F2
:107BD0005D6F5E6B4D6B4E6BFB0E5C6F658C0401D5
:107BE000C46B0401C16B0401BD6B0401CD6B659CCA
:107BF000160E0F014C6F02D06296040062B6FCD7DD
:107C0000659812001F4B202B226BEF0E01012225DD
:107C1000D96EDA6A030EDA22DF50216F1F51186F16
:107C20002051196F1F4B202B90EC2EF0211902E0F0
:107C3000D8901200222B050E2265E7D7D880050CBC
:107C400086B611D000F086B60ED000F086B60BD006
:107C5000010E0101016F690E006FDBEC3BF03F2A62
:107C6000050E416E050C2F0E0101016F100E006F05
:107C7000DBEC3BF0010E3F6E010CE8CF1AF1010E78
:107C8000196F1A51800A190F04E21A51800A1F0F46
:107C90000DE21A51800A390F04E21A51800A3F0F8F
:107CA00005E21A519FEC43F0D8A0196B19C118F1E5
:107CB00018311200636A626A9F0E5D6F5E6B4D6BD6
:107CC0004E6BFB0E5C6F658C0401C46B0401C16BD1
:107CD0000401BD6B0401CD6B659C160E0F014C6F4A
:107CE00002D06296040062B6FCD7659812009692A4
:107CF0009690000103A809D0848284B209D00101C2
:107D0000D36706D0020ED36F03D0000103A884927C
:107D10008D8000F08DB005D00101D36702D0010E37
:107D2000D36F8D9012001B6B61EC40F0186F1B51EC
:107D30001625196FE86A1BBFE86817211A6F19C169
:107D4000D9FF1AC1DAFF18C1DFFF1B2B1B51800AB4
:107D5000790FEAE361EC40F00001099212004F0E46
:107D6000196FD40E186F90EC2EF0216F4F0E196F13
:107D7000D50E186F90EC2EF0226F2151246F2251F6
:107D8000236F2051241902E11F51231902E1D880E9
:107D90001200D890120000C1D9FF01C1DAFFDF50F4
:107DA000060A02E0D890120020EE01F00051D92618
:107DB0000151DA22180EDF6205D002510C0A02E1ED
:107DC000D880120002510A0AFBE0ECD7E8CF15F187
:107DD00015C1C2FFC280190E0101166F16070101FD
:107DE0001629FCE1C282320E166FC2A204D0160719
:107DF00001011629FAE1C450FC0B166FC26A165134
:107E0000120086969896080E416E412EFED79886EF
:107E1000280E416E412EFED786A603D00301F58FB2
:107E200002D00301F59F010E0101016FA50E006F45
:107E3000DBEC3BF03F2A12001B6B61EC40F0186F4B
:107E40001B511625196FE86A1BBFE86817211A6FC6
:107E500019C1D9FF1AC1DAFF18C1DFFF1B2B1B5153
:107E6000800A7D0FEAE3000109921200B8EC42F0AB
:107E70000101176F175111E0A098040E0401C86F9B
:107E8000300EC76F15C1C9F416C1CAF417C1CBF4BF
:107E900064EC3CF0A08813EC44F00101175112008F
:107EA0001B6B61EC40F0186F1B511625196FE86AC7
:107EB0001BBFE86817211A6F19C1D9FF1AC1DAFF71
:107EC00018C1DFFF1B2B1B51800A7B0FEAE3000167
:107ED00009921200849296928D80969000F000F0A4
:107EE0008DB005D00101D36702D0010ED36F84821B
:107EF00000F000F084B205D00101D36702D0040E77
:107F0000D36F8D9000F0120017C118F1196B155145
:107F1000010B181BD8901633153318A104D0010E8D
:107F2000151BA00E161BD8901833192B070E1965B8
:107F3000EED715C115F116C116F1070C1B6B61ECDC
:107F400040F0186F1B511625196FE86A1BBFE868CF
:107F500017211A6F19C1D9FF1AC1DAFF18C1DFFF43
:107F60001B2B1B51800A7E0FEAE3000109921200CD
:107F70000101206B1EC117F11FC118F1EE0E0101A6
:107F80002025D96EDA6A030EDA22DF50196F50EC21
:107F900035F001011E4B1F2B202B060E2065EAD762
:107FA000060CE8CF1FF0000E4224D96EDA6A0D0EDF
:107FB000DA221FC0DFFF422A4250F00AD8B4426AD8
:107FC0000001FB2BFB51F00AD8A41200000109822A
:107FD0001200E8CF15F1000E4224D96EDA6A0D0EB8
:107FE000DA2215C1DFFF422A4250F00AD8B4426AB1
:107FF0000001FB2BFB51F00AD8A4120000010982FA
:108000001200010E01011F6F7F0E01011F25D96EA5
:10801000DA6A060EDA22960E1F25186F196B020E09
:10802000192390EC2EF0DF6E1F2B0F0E1F65ECD77F
:108030000F0C02510E0A02E0D890120000C1D9FFC5
:1080400001C1DAFF070EDF6401D0F6D720EE01F0A0
:108050000051D9260151DA22010EDF62EDD7D88016
:10806000010CE8CF18F10101185103E01851050A7D
:1080700002E1D890120018C116F1FF0E162715C1A3
:1080800017F1162B02D0D8901733162FFCD71731C3
:108090001200E8CF1FF01FC0C2FFC280190E206E71
:1080A00020062028FDE1C282320E206EC2A203D03B
:1080B00020062028FBE1C450FC0B206EC26A205031
:1080C0001200000E0201D325D96EDA6A0D0EDA22F3
:1080D000DF500101156F0201D32BD351F00AD8B440
:1080E000D36B0001FB07FB6701D00E940101155112
:1080F000120002510D0A02E0D890120000C1D9FF0F
:1081000001C1DAFFDF504E0AF7E120EE01F0005125
:10811000D9260151DA22DF50620AEEE1D88012003E
:1081200002510B0A02E0D890120000C1D9FF01C130
:10813000DAFFDF504E0AF7E120EE01F00051D926B8
:108140000151DA22DF50610AEEE1D88012001751A6
:1081500015C1D9FF16C1DAFFDF6205D015C115F1CF
:1081600016C116F1120015C1D9FF16C1DAFF154B61
:10817000162BDF50ECE1156B166B1200E8CF15F1F2
:1081800015510D0A04E115C1C4F2D8901200155121
:108190000A0A07E10201C4510D0A03E1C46BD88049
:1081A00012000201C46BF1D7000109B212000101F3
:1081B000186B18511625D96E000E1721DA6EDF5094
:1081C000E9EC3FF00101182B070E1865F2D700010A
:1081D0000E84070C8B92030ECCEC44F00101185175
:1081E000CCEC44F001011751CCEC44F01651CCEC2E
:1081F00044F0000ECCEC44F01A6F8B821A5112003E
:10820000E8CF15F115514F0A04E115C1C5F2D89018
:10821000120015514B0A07E10201C5514F0A03E153
:10822000C56BD88012000201C56BF1D7196B1A6BB0
:1082300015A104D01751192718511A23D8901737B0
:108240001837D8901633153316511511F1E119C1AD
:1082500015F11AC116F11200E8CF1AF11851AFEC5E
:1082600037F015C11BF116C11CF11A51020DF35064
:108270001B25D96E000E1C21DA6EDECF18F1DDCF82
:1082800019F11200E8CF37F10101370508E1FB0EC3
:10829000166FC00E156F080E176FDDEF43F0FB0E63
:1082A0002C6FC00E2B6F2E6B080E2D6FACEF04F0F1
:1082B000E8CF37F10101370508E1F90E166FA60E78
:1082C000156F0A0E176FDDEF43F0F90E2C6FA60E37
:1082D0002B6F2E6B0A0E2D6FACEF04F0236A246A0D
:1082E0001FA004D02150232622502422D8902136CA
:1082F0002236D89020321F3220501F10F1E123C0C7
:108300001FF024C020F01200000109B2120020C0AA
:10831000D9FF21C0DAFFDF50D1EC3FF020EE01F0B1
:108320002050D9262150DA22DF50D1EC3FF0000155
:108330000E8412008D9096908482969200F08D802B
:1083400000F000F08DB005D00101D36702D0010E1E
:10835000D36F849200F000F000F08D9000F01200D6
:10836000E8CF37F10101370508E1FA0E166FB60EB6
:10837000156F090E176FDDEF43F0FA0E2C6FB60E76
:108380002B6F2E6B090E2D6FACEF04F0E8CF37F199
:108390000101370508E1F90E166F9B0E156F0A0EE5
:1083A000176FDDEF43F0F90E2C6F9B0E2B6F2E6BCA
:1083B0000A0E2D6FACEF04F0F29210A003D01090D3
:1083C000F19C8A8210A206D01092F19C000110BA92
:1083D0008A8212008A92010E0101D86F00010F8A71
:1083E000010C0101D76706D0010ED76F0A88020180
:1083F000EF6B1200D70506E1020ED76F0201EF6B9B
:10840000EE6B1200D76B00010B86120004012451A1
:108410000F0B080D000EF3240401C76FC86B040E88
:10842000C823040124AF1200040E0401C727000E64
:10843000C823000CE8CF17F1010E166F1751200A60
:1084400009E01751800A720F04E21751800A770F72
:10845000D8A0166B16C115F11531120000010BA43E
:108460000CD00201DA51D8A4DA07DA671200A1ECC5
:1084700044F0320EDA6FD82B320CFDECF5F002012D
:10848000D86B1200000108BA050C000115B2050CEA
:10849000FF0E01012C6FE00E2B6F000E2E6B2D6B6B
:1084A000ACEC04F001E2000C5EEF0DF096829690C9
:1084B000000103968D8000F08DB005D00101D367D7
:1084C00002D0010ED36F00F084A202D00001038617
:1084D0008D901200040124510F0B080D000EF3249F
:1084E0000401C76FC86B040EC823040124AF120037
:1084F000040E0401C727000EC823000C8B92020E45
:10850000CCEC44F001011851CCEC44F001011751BE
:10851000CCEC44F01651CCEC44F01A51CCEC44F0C5
:108520008B821200E8CF21F0206A090E216405D069
:10853000202A0A0E215E2160FBD721C01FF00F0EFA
:108540001F162038F00B1F1012001EC1CFF11FC1E3
:10855000D0F1186B590E176F1F51196F50EC35F091
:108560000101186B5A0E176F1EC119F150EF35F04B
:10857000040118BF000C200E0401CD6101D0000CD5
:10858000A0A8000C0401196703D013EC44F0000C00
:10859000040119511200E8CF15F10301A86BA96B72
:1085A000000EA76F0A0EA66F00011D9AA4B803D093
:1085B00000011DAAFBD715C1A9FF1200E8CF15F1D4
:1085C0000301A86BA96B000EA76F0A0EA66F00012E
:1085D0001D9A9EB803D000011DAAFBD715C1AEFF9E
:1085E0001200040118BF1200200E0401CD6101D059
:1085F000200CA0A812000401196702D006EF44F075
:108600000401195112009886080E416E412EFED7C2
:10861000402E05D0400E406E3F2A01EF3FF003018F
:10862000D890EE333F0615EF43F086969896080EE5
:10863000416E412EFED70301EEB19886010E010175
:10864000016F870E006FDBEC3BF03F2A1200E8CF92
:1086500015F1600E0101156503D01551A90F120027
:10866000400E156503D01551C90F12001551D00FDA
:1086700012004F0E186FD40E176F1F51196F50EC68
:1086800035F04F0E0101186FD50E176F1EC119F18D
:1086900050EF35F0E8CF21F0206A2150800A460FD4
:1086A00006E22150800A500F02E3010E206E20C026
:1086B0001FF01F301200E8CF15F10F0E0101151742
:1086C0000A0E156104D0300E152715511200370E11
:1086D0001527010115511200DA2F1200FDECF5F0FB
:1086E000230E0301AC5D000EAD59320ED8B0FA0E68
:1086F0000201DA6F010ED86F010C19A80CD019987D
:108700008B9C0CA604D0320E0201EF6F320C0F0EC0
:108710000201EF6F0F0C19888B8CF3D7E8CF17F19C
:10872000166B1751800A250F06E21751800A3F0F7A
:1087300002E3010E166F16C115F115311200E8CFD4
:1087400017F1166B1751800A460F06E21751800A7F
:10875000500F02E3010E166F16C115F1153112000C
:108760000201D86702D0C4EF44F0D80502E12EEF31
:1087700042F0D851020A02E16CEF43F0D86B1200CC
:10878000FB0E0101176F8A0E166F010E4EEC32F0D0
:10879000130E01012A6F880E296F2BEF37F0F8ECCA
:1087A00044F02AEC2BF041ECB0F019EC1CF04BEC4F
:1087B000DFF0168200011B8012000DEC45F000096D
:1087C000FCE115C1B3F416C1B4F417C1B2F4010E43
:1087D0000401B16F010CE8CF5CF1000113AC07D0CC
:1087E00001015C0504E1CFEC43F0D8801200D89081
:1087F0001200E8CF15F11551800A250F05E2155139
:10880000800A3F0FD8B0158B15511200400E04019D
:10881000181B040E1B6F300E1A6F400E196F1817BD
:10882000880E1813880C400E0401181B040E1B6FD1
:10883000300E1A6F400E196F1817880E1813880C17
:10884000E8CF15F11551800A050F05E21551800A90
:108850001F0FD8B0159B155112000001FF51D8A46D
:10886000FF07FF671200A1EC44F0452A120EFF6FCC
:10887000120CE8CF27F027AA03D0206A900E02D06E
:10888000206A920E1F6E5EEF1BF00001FF51D8A40C
:10889000FF07FF671200A1EC44F04506640EFF6F6E
:1088A000640C0001FF2FB0EF43F0FDECF5F0456ADA
:1088B0000201D76BB0EF43F00201D76702D0D4EFCB
:1088C00044F0D70502E1BCEF44F0D76B1200869666
:1088D00098960B0E0101016FC40E006FDBEC3BF0AC
:1088E0003F2A12009886010E0101016F870E006F6A
:1088F000DBEC3BF03F2A120098862F0E0101016F3E
:10890000100E006FDBEC3BF03F2A12000401D56B28
:108910000401CC9FA288E4EC3DF077EFEDF0A0B825
:10892000A1A81200E8ECEBF0F1EC42F0A1981200E3
:10893000E8CF15F1010115A902D0D8801200D89016
:108940001200AA0ECB6E550EBC6ECC6ACA843F0EC6
:10895000BB6E3F0CF0925E0E776E786AA496A3868B
:108960000001168412000001FF2F1200FDECF5F04B
:10897000452A090EFF6F090C00010ABC1200FDEC2C
:10898000F5F00201D76B12000BA45CEF44F0320E3D
:108990000201DA6FD82B320CE8CF15F115C1C9FFEF
:1089A000C7A0FED7C950120000010AAC1200A1EC0A
:1089B00044F00201D72B1200400E04011C1B1C17AF
:1089C000880E1C13880C400E04011C1B1C17880EFB
:1089D0001C13880C000105B202D0D8901200D88078
:1089E000120017C1F8FF16C1F7FF15C1F6FF1200FC
:1089F000139C1B900301CF6B00011A9A1200C4EC68
:108A0000E7F0AEC329F1AFC32AF11200E8CF15F1A8
:108A1000010115510001FA1B1200A0A8010C04016C
:108A2000B1511200E8CF15F115C1F5F01200059211
:108A30000001F95112000301AE6BAF6B1200FFFF92
:108A4000FFFFFFFFFFFFFFFFFFFFFFFFFFFFFFFF36
:108A5000FFFFFFFFFFFFFFFFFFFFFFFFFFFFFFFF26
:108A6000FFFFFFFFFFFFFFFFFFFFFFFFFFFFFFFF16
:108A7000FFFFFFFFFFFFFFFFFFFFFFFFFFFFFFFF06
:10EAC00030352F30312F30312C30303A30303A3031
:10EAD000300051495552433A2022636C6F7365648C
:10EAE0002200434D53204552524F523A2031393380
:10EAF00000434D53204552524F523A203531350094
:10EB0000434D45204552524F523A20313300434D38
:10EB100045204552524F523A203131005149555209
:10EB2000433A2022726563762200434F4E4E45439E
:10EB300054204641494C0051534D54505055543A7D
:10EB4000202D0001000A006400E803102743535100
:10EB50003A20302C30004352494E473A2000434D72
:10EB600054493A2000435245473A2000434C4F5302
:10EB7000454400735F6C6F636B002B43504252003F
:10EB80002B43504257002B434D4752002241434BE9
:10EB9000220009024300020100C0640904000001D0
:10EBA00002020000052400100104240202052406CC
:10EBB0000001052401000107058203080002090481
:10EBC0000100020A000000070503024000010705DA
:10EBD00083024000011201100102000008D8040A5B
:10EBE000000100000000012B514654504346473DB0
:10EBF000226163636F756E74222C22636F72746579
:10EC000078757064617465222C224264746724668E
:10EC100064764B220D00432F25642E466C61736889
:10EC2000696E672120446F6E277420706F7765725C
:10EC3000206F6666210D0A002B514654504F5045F7
:10EC40004E3D227570646174652E636F72746578D1
:10EC50002E6C76222C32310D002B514655504C3DF6
:10EC6000227570646174652E686578222C333635A0
:10EC70003030302C350D002B515552434346473D23
:10EC800022757263706F7274222C227561727431F6
:10EC9000220D00446F776E6C6F616465642073753C
:10ECA000636365737366756C6C792E0D0A002E684C
:10ECB0006578222C225546533A7570646174652E2E
:10ECC000686578222C300D00436F6D6D616E642095
:10ECD0006E6F7420617661696C61626C652E0D0ADD
:10ECE00000557067726164696E672E2E2E506C65D8
:10ECF00061736520776169742E002B51534D545018
:10ED00004346473D22736D74707365727665722257
:10ED10002C22002B514346473D226E777363616E70
:10ED20006D6F6465222C302C310D002B51465450F0
:10ED30004346473D22636F6E746578746964222C84
:10ED4000320D002B51494346473D227064702F72AB
:10ED500065747279222C302C310D002B51494346B9
:10ED6000473D227064702F7265747279222C312CA9
:10ED7000310D002B51534D54504346473D22636F94
:10ED80006E746578746964222C3100465450206496
:10ED900069726563746F7279206572726F722E0D7D
:10EDA0000A00556E706C7567207468652055534273
:10EDB000206361626C650D0A002B43504D533D2268
:10EDC000534D222C22534D222C22534D220D0055FF
:10EDD0005047524144453A4845582053495A4520E6
:10EDE0004552523B002B51534D54504346473D2210
:10EDF0006163636F756E74222C22002B51534D5446
:10EE0000504346473D2273736C74797065222C30F1
:10EE100000446F776E6C6F6164696E672065727213
:10EE20006F722E0D0A002B514644454C3D227570E1
:10EE3000646174652E686578220D002B4347514D3F
:10EE4000494E3D312C302C302C302C302C300D00E4
:10EE50002B4347515245513D312C302C302C302C16
:10EE6000302C300D002B51534D54504346473D221A
:10EE700073656E646572222C22002B51494F5045F8
:10EE80004E3D312C312C22544350222C220046542A
:10EE90005020736572766572206572726F722E0DE6
:10EEA0000A0023343A3032303030303032303030B3
:10EEB0003046430D0A00495320414C5245414459C4
:10EEC000204C4F434B45440D0A002B51494F5045B0
:10EED0004E3D312C302C22544350222C22004469C8
:10EEE000726563746F7279206572726F722E0D0A8B
:10EEF000002B51495552433A202272656376222CE9
:10EF0000302C0051495552433A20227265637622D3
:10EF10002C312C330023343A303030303030303123
:10EF200046460D0A0D0A004D6F64656D20657272CC
:10EF30006F7220302E2E0D0A004D6F64656D2065B6
:10EF400072726F7220312E2E0D0A004D6F64656D46
:10EF5000206572726F7220322E2E0D0A004D6F6482
:10EF6000656D206572726F7220332E2E0D0A00556A
:10EF70005047524144453A48455820455252313B4A
:10EF800000555047524144453A4845582045525251
:10EF9000333B00555047524144453A54494D452D65
:10EFA0004F55543B002B434744434F4E543D312C67
:10EFB000224950222C22002B434E4D493D322C3108
:10EFC0002C302C302C300D002B43434C4B3D223049
:10EFD000302F30312F30312C0053544154453A20DA
:10EFE000434F4E4E45435445440057616974206673
:10EFF0006F72206865782E2E0D0A0046696E616C6E
:10F000002076657273696F6E2E0D0A002B5146547F
:10F01000504357443D2247503531220D002B514675
:10F0200054504745543D2247505F46353100554EB8
:10F0300053454E545F4255465F46554C4C0D00516A
:10F04000495552433A202272656376222C30005192
:10F05000495552433A202272656376222C3100438F
:10F0600050494E3A204E4F5420494E53455200438A
:10F0700050494E3A204E4F54205245414459005376
:10F08000494D5320554E4C4F434B45440D0A002BE0
:10F09000514654504745543D2247505F3531005545
:10F0A0005047524144453A4353204552523B003069
:10F0B000362C25732C383430393930302564003003
:10F0C000372C25732C3834303939303025640030F2
:10F0D000362C25732C3834313939303025640030E2
:10F0E000372C25732C3834313939303025640030D1
:10F0F000362C25732C383538393930302564002BBF
:10F1000051534D54504453543D312C312C22004323
:10F110004D45204552524F523A203130300048453B
:10F12000582053495A45204552520D0A002B51464A
:10F1300054504E4C53543D222E220D00546573748E
:10F1400054696D653A2025642C200030362C2573D7
:10F150002C38353039393030300030372C25732C8D
:10F1600038353039393030300030362C25732C3872
:10F17000303139393030300030362C25732C38326C
:10F180003139393030300030362C25732C3832325A
:10F1900039393030300030372C25732C3832323941
:10F1A000393030300030362C25732C383233393931
:10F1B0003030300030362C25732C3830343939302B
:10F1C00030300030362C25732C3832343939303019
:10F1D000300030372C25732C383038393930303006
:10F1E0000030362C25732C38323939393030300024
:10F1F00030372C25732C38323939393030300030E3
:10F20000362C25732C3833333939303230003037CF
:10F210002C25732C38333339393032300030362CCA
:10F2200025732C38333039393030310030372C25C4
:10F23000732C38333039393030310030362C257367
:10F240002C38303239393030310030372C25732C9E
:10F2500038303239393030310030362C25732C3883
:10F26000353439393030310030362C25732C38356F
:10F270003539393030310030372C25732C3835355D
:10F2800039393030310030362C25732C3833303951
:10F29000393030320030372C25732C38333039393F
:10F2A0003030320030362C25732C3830323939303A
:10F2B00030320030372C25732C3830323939303029
:10F2C000320030362C25732C383534393930303211
:10F2D0000030362C25732C38353539393030320032
:10F2E00030372C25732C38353539393030320030F1
:10F2F000362C25732C3833303939303033003037E1
:10F300002C25732C38333039393030330030362CDB
:10F3100025732C38353439393030330030362C25CC
:10F32000732C38333039393030340030372C257372
:10F330002C38333039393030340030362C25732CAA
:10F3400038353439393030340030362C25732C3888
:10F35000333039393030350030372C25732C383381
:10F360003039393030350030362C25732C38333075
:10F3700039393030360030372C25732C383330395A
:10F38000393030360030362C25732C38343039394A
:10F390003025640030372C25732C3834303939301F
:10F3A00025640030362C25732C383431393930251A
:10F3B000640030372C25732C3834313939302564CA
:10F3C0000030362C25732C38353839393025640017
:10F3D0002B51464C44533D22554653220D00514675
:10F3E00054504F50454E3A20302C300051534D541C
:10F3F000505055543A20302C3000434D4520455252
:10F40000524F523A203130004350494E3A2053492E
:10F410004D2050494E0049705254696D653A25643B
:10F420006D2C20004155544F2055504752414445C2
:10F430003A002B5149444E534346473D312C22005C
:10F440002B435343533D22495241220D0051534D0A
:10F450005450424F44593A202D0051465450434C89
:10F460004F53453A20300051534D5450424F445968
:10F470003A203100434F4E4E454354204641494CBB
:10F4800000762E25645F6D6F6465300D0A00762E60
:10F4900025645F6D6F6465310D0A0048455820573B
:10F4A00052204552520D0A005349412049503A4FCB
:10F4B00046462C2000477072734174743A25642CC0
:10F4C00020004F4E2C282564206461797329003078
:10F4D000362C2530336439393030300030372C2524
:10F4E00030336439393030300030362C38343039EC
:10F4F00039303025640030372C38343039393030E9
:10F5000025640030362C38343139393030256400E8
:10F5100030372C3834313939303025640030362CCE
:10F5200038353839393030256400222C22382E38CD
:10F530002E382E38220D002B514953454E443D3074
:10F540002C300D002B4950523D31393230300D00F6
:10F550002B434F50533D342C302C22002B51494328
:10F560004C4F53453D310D00313630302039392074
:10F5700030303000313330312039392030303000F4
:10F5800033333031203939203030300031333032AC
:10F5900020393920303030003333303220393920AF
:10F5A00030303000313630322039392030303000C0
:10F5B0003133393320393920303030003131343073
:10F5C000203939203030310033313430203939207E
:10F5D0003030310031313430203939203030320090
:10F5E0003331343020393920303032003131343049
:10F5F000203939203030330033313430203939204C
:10F600003030330051494F50454E3A20302C3000B5
:10F6100051494F50454E3A20312C300051494E4906
:10F62000535441543A20320051494F50454E3A20EC
:10F63000302C350051494E49535441543A2037003B
:10F640004350494E3A205245414459004953204CB9
:10F650004F434B45440D0A002B5149444541435407
:10F660003D320D002B51465450434C4F53450D0035
:10F670005374617941282564292C20005349412085
:10F6800049503A4F4E2C20005154696D653A25641B
:10F69000732C20004E6F20557067726164652E00D8
:10F6A00030362C38353039393030300030372C385E
:10F6B000353039393030300030362C383031393946
:10F6C0003030300030362C3832313939303030007B
:10F6D00030362C38323239393030300030372C382F
:10F6E000323239393030300030362C383233393913
:10F6F0003030300030362C3830343939303030004A
:10F7000030362C38323439393030300030372C38FC
:10F71000303839393030300030362C3832393939D8
:10F720003030300030372C38323939393030300011
:10F7300030362C38333339393032300030372C38CA
:10F74000333339393032300030362C3833303939B0
:10F750003030310030372C383330393930303100E7
:10F7600030362C38303239393030310030372C389F
:10F77000303239393030310030362C38353439397F
:10F780003030310030362C383535393930303100B1
:10F7900030372C38353539393030310030362C3867
:10F7A000333039393030320030372C383330393952
:10F7B0003030320030362C38303239393030320087
:10F7C00030372C38303239393030320030362C383E
:10F7D000353439393030320030362C383535393916
:10F7E0003030320030372C3835353939303032004E
:10F7F00030362C38333039393030330030372C380C
:10F80000333039393030330030362C3835343939EB
:10F810003030330030362C38333039393030340022
:10F8200030372C38333039393030340030362C38DA
:10F83000353439393030340030362C3833303939BA
:10F840003030350030372C383330393930303500EE
:10F8500030362C38333039393030360030372C38A8
:10F860003330393930303600555047524144453AEB
:10F870004F4B3B0030362C3834303939302564005A
:10F8800030372C38343039393025640030362C3854
:10F89000343139393025640030372C383431393936
:10F8A0003025640030362C3835383939302564003D
:10F8B000466F7263654F66663A2564002B51494472
:10F8C000454143543D310D002B5149444E5343466D
:10F8D000473D22002B5149435347503D312C3300C3
:10F8E0002B4346554E203D20310D002B51494353AB
:10F8F00047503D310D002B4356455253494F4E0D55
:10F90000002B51494E49535441540D0051534D540D
:10F91000505055543A2000514654504357443A20D1
:10F920003000514654504745543A20300043475226
:10F9300045473A20312C300043475245473A203161
:10F940002C310043475245473A20312C320043477F
:10F950005245473A20312C330043475245473A201D
:10F96000312C340043475245473A20312C3500436F
:10F970004F4E4E454354204F4B004845582045526A
:10F9800052310D0A0048455820455252330D0A00A5
:10F9900049532057524F4E470D0A00434F444520CC
:10F9A0004552520D0A0053544154204552520D0AFB
:10F9B000000D0A4743207625640D0A002B5146545A
:10F9C000504745543D2200504F5254313A25732C34
:10F9D0002000504F5254323A25732C2000504F5281
:10F9E00054333A25732C20007374616E6461727411
:10F9F0002C200064696769706C65782C20002B519D
:10FA00004953454E443D300D002B51534D54504306
:10FA10004C520D002B514953454E443D302C002B88
:10FA2000514953454E443D312C002B4347524547E5
:10FA30003D310D002B514E57494E464F0D0022418E
:10FA4000444D2D4349442200514453494D3A2030FE
:10FA50002C00514453494D3A20312C004352454724
:10FA60003A20312C3000435245473A20312C3100A6
:10FA7000435245473A20312C3200435245473A2001
:10FA8000312C3300435245473A20312C3400435245
:10FA900045473A20312C3500514654504E4C535472
:10FAA0003A00434D45204552524F5200434D53209A
:10FAB0004552524F5200434F4445204F4B0D0A00D0
:10FAC000484558204552520D0A00526573746172C0
:10FAD000740D0A002B51494143543D320D004745F6
:10FAE0004E4552414C2C2000554E4B4E4F574E2CFC
:10FAF0002000424154204C4F572C20006D61676517
:10FB00006C616E2C2000756E6B6E6F776E2C200012
:10FB100053656375726974793A002B51504F57449D
:10FB20003D310D002B51494143543D310D002B43D4
:10FB3000474154543D310D0053454E442046414900
:10FB40004C002B435344483D300D002B434F505342
:10FB50003D300D002B434D45453D310D002B4352AB
:10FB600045473D310D002B434C49503D310D002B95
:10FB700043545A553D330D002B43475245473F0DE3
:10FB8000002B434D47463D300D002B434D47463D2E
:10FB9000310D002B5149535441540D0043474154FA
:10FBA000543A20300043475245473A2031004347FA
:10FBB0004154543A2031004445414354204F4B00B6
:10FBC0004545204552520D0A004353204552520DDF
:10FBD0000A002B4346554E3D300D002A2373696DB4
:10FBE0005F673000454646364630384600667470DA
:10FBF0005F6C6F6164004C4E723A25642C20005398
:10FC0000413A2025732C2000534D3A2025732C2097
:10FC100000534E3A2025732C200053503A20257370
:10FC20002C20004950313A25732C20004950323A9B
:10FC300025732C20004950333A25732C2000415065
:10FC40004E3A25732C2000444E533A25732C200045
:10FC50005757573A25732C20006573707269742CBE
:10FC6000200028435245472564200043475245471A
:10FC7000256420004E6F5F43617264290053696DF3
:10FC80004C6F636B3A0050616E537461743A00615B
:10FC900025732C25730D0A002B514453494D3F0DFC
:10FCA000002B43474154543F0D002B4352433D31F9
:10FCB0000D002B435245473F0D002B434F50533F00
:10FCC0000D002B51434349440D002B4350494E3DF9
:10FCD00022002B43434C4B3D2200302E302E302E41
:10FCE00030003A757064617465002B43434C4B3FA0
:10FCF0000D002B434D47533D22000A303030303049
:10FD00003000435041533A2030004346554E3A208C
:10FD10003100434F4E4E454354004552522564290D
:10FD2000200044282564292C200070616E656C2C0D
:10FD300020004C3A2025732C20004F6E6C696E65B4
:10FD40003A0047454E4552414C00554E4B4E4F5799
:10FD50004E002B4350494E3F0D002B4346554E3F1E
:10FD60000D00514953454E443A0053454E44204FEF
:10FD70004B00286E756C6C29002B435355420D00C7
:10FD80002B43494D490D002B4347534E0D002B513A
:10FD900047534E0D002B43474D520D002B51474DFD
:10FDA000520D002B435042523D002B434D47533DD3
:10FDB00000434C49503A2000435042523A200043FD
:10FDC0004F50533A2000432F25640D0A0044283138
:10FDD000292C200053494D312C2000647363312CB1
:10FDE0002000647363322C200042454C4C2C2000D0
:10FDF000475052532C2000414F66662C20004D4F37
:10FE000066662C20004C3A25732C2000503A25734E
:10FE10002C2000616275732C2000563A25643B202B
:10FE200000434D4525642000434D53256420005375
:10FE3000494D313A280028636F6465290055736580
:10FE400072733A00414354495645003030303130E6
:10FE500030002B4353510D002B3038220D007570AC
:10FE60006F6666002C3134352C002C3132392C0071
:10FE70002B434D474400224E414B22004353513AFD
:10FE8000200043434C4B3A00434D47533A00514303
:10FE90004349440053494D31200053494D3220001D
:10FEA00023343A3130006D6F646530006D6F6465E6
:10FEB00031006D6F64653F006E636F64650072654D
:10FEC0006465660073696D5F6C00736669726D00CE
:10FED0002825642920002F256429200047534D2C14
:10FEE0002000414F6E2C20004D4F6E2C20002874B6
:10FEF0007874290053494D313A004F5554313A0036
:10FF00004F5554323A004D6F64653A005245434FA5
:10FF10004E0053494D455200534D534552004D3A02
:10FF2000202573002B434D450075706F6E005147BF
:10FF3000534E0033334343006C7461620073746149
:10FF40006200252E3264006C636667007363666727
:10FF5000006C6C6F67006C746D70006C747874006A
:10FF600073747874006E782C200025733B20002F6A
:10FF7000256429004F55543A002573293B004E4F04
:10FF80004E45004750525300444159530047525385
:10FF900054004D5253540030303038005244590010
:10FFA00045310D004F4E2F00495031002055310092
:10FFB000495032002055320020553300205534007E
:10FFC000494E3A004F4646004255460047534D00C1
:10FFD00045525200444E5300282564002F256400EA
:10FFE000510D0A00480D005530004C3000222C0005
:10FFF00039310041310023005B007C003E000000ED
:020000040001F9
:100000000101976B5F51156F030E6015166F186B2A
:100010000E0E176F16EC41F0040E15259A6F040EA4
:1000200016219B6F6051996F9941E8423F0B070B76
:10003000996F9AC11FF19BC120F1B7EC2FF001E23B
:10004000000C13AC03D0010199051FE01EA804D0D9
:1000500001019951030A19E00101995154ECD9F0B9
:10006000EFE31EC597F19E6B0BD0FAEC8DF0650E99
:100070009E25E16EE26A010EE222DFCFE7FF9E2BB2
:1000800005011E5101019E5DF0E3C1054EE160AF27
:1000900034D00501A6EC8DF092EC8DF0310EDF6EC0
:1000A0009E2B1F0E6DEC8DF054EC8DF0616F61395D
:1000B0000F0B5BEC43F0DF6E9E2B54EC8DF00F0BBF
:1000C0005BEC43F0DCEC8DF09D65EED71F0E63EC2E
:1000D0008DF01F0E9E2578EC8DF05BEC43F086ECE6
:1000E0008DF05BEC43F0DF6E9E2B9E51C6ECEFF083
:1000F000D2EC8DF094EC20F015D00501D48117A43A
:1001000009D0010E01011E6F000EC6EC0BF010ECC1
:100110008EF002D001019E6B9E5157ECE3F002E29B
:100120000101996B010199511200C151020A4FE17D
:1001300060AF3AD00501A6EC8DF092EC8DF0320E56
:10014000DF6E9E2B1F0E6DEC8DF054EC8DF0616F09
:1001500061390F0B5BEC43F0DF6E9E2B54EC8DF09E
:100160000F0B5BEC43F0DCEC8DF09D65EED71F0EC2
:1001700063EC8DF0030E9D6F54EC8DF0616F61396F
:100180000F0B5BEC43F0DF6E9E2B54EC8DF00F0BEE
:100190005BEC43F0DF6E9E2B9D2B040E9D65ECD730
:1001A0009E51C6ECEFF0A4D70501D48117A409D065
:1001B000010E01011E6F000EC6EC0BF010EC8EF06C
:1001C00002D001019E6B9E5157ECE3F0A8D7C151BC
:1001D000030A4FE160AF3AD00501A6EC8DF092EC36
:1001E0008DF0330EDF6E9E2B1F0E6DEC8DF054ECF8
:1001F0008DF0616F61390F0B5BEC43F0DF6E9E2B6E
:1002000054EC8DF00F0B5BEC43F0DCEC8DF09D6556
:10021000EED71F0E63EC8DF0030E9D6F54EC8DF046
:10022000616F61390F0B5BEC43F0DF6E9E2B54EC7A
:100230008DF00F0B5BEC43F0DF6E9E2B9D2B050EBC
:100240009D65ECD79E51C6ECEFF052D70501D481E5
:1002500017A409D0010E01011E6F000EC6EC0BF0B1
:1002600010EC8EF002D001019E6B9E5157ECE3F032
:1002700056D7C151060A03E0C151070A5CE160AFDD
:1002800047D00501D46B01019E6BC1390F0B5BECAC
:1002900043F005011F6F010192EC8DF0C1510F0B6E
:1002A0005BEC43F0DF6E9E2B1F0E63EC8DF0010EB6
:1002B0009D6F54EC8DF0616F61390F0B5BEC43F077
:1002C000DF6E9E2B54EC8DF00F0B5BEC43F0DCECFF
:1002D0008DF09D65EED71F0E63EC8DF0030E9D6FC4
:1002E00054EC8DF0616F61390F0B5BEC43F0DF6E06
:1002F0009E2B54EC8DF00F0B5BEC43F0DF6E9E2BCE
:100300009D2B060E9D65ECD79E51C6ECEFF0F0D606
:100310000501D48117A409D0010E01011E6F000E42
:10032000C6EC0BF010EC8EF002D001019E6B9E51DA
:1003300057ECE3F0F4D6C12901E082D6C4C1DBF169
:10034000C451190A09E0C451200A06E0C451210A27
:1003500003E0C451220A30E10501D46B010E010112
:100360009D6FC451200A02E1020E9D6FC451210A03
:1003700002E1030E9D6FC451220A02E1040E9D6F3B
:100380009D5154ECD9F001E25BD69E6B07D0FAEC9C
:100390008DF01F0E9E25C5EC0DF09E2B05011E5104
:1003A00001019E5DF4E31F0E9E25D96EDA6A050EEB
:1003B000DA22DF6A2CEF8DF0C451810A0AE10501CF
:1003C000AEEC8DF0EC0E246FE10E236F86ECCEF0D8
:1003D0000CD0C451820A0DE10501AEEC8DF0F60E91
:1003E000246F940E236F86ECCEF021519D6F2CEF7D
:1003F0008DF0C4518A0A01E00DD10501D46B050EC0
:1004000001019AEC8DF086ECCEF021519D6F9DC1DB
:100410009EF11DBC23D001019C6B7FEC8DF0CD0EB5
:100420009C25186F196B000E192390EC2EF0DF6ECF
:100430007FEC8DF0DF5004E09C2B0F0E9C65EDD718
:100440001F0E47EC8DF0FC0E246F230E236F010E60
:10045000266F770E256F86ECCEF01ED01F0E47EC70
:100460008DF0FC0E246F500E236F070E266F500E7A
:10047000256F86ECCEF021519D6F9D519E271F0E5A
:1004800047EC8DF0FC0E246F470E236F070E266F8E
:10049000AB0E256F86ECCEF04EEC8DF07FEC8DF040
:1004A000C80E9C25186F196B000E192390EC2EF0C6
:1004B000DF6E7FEC8DF0DF5004E09C2B040E9C651A
:1004C000EDD71F0E47EC8DF0F90E246FC70E236F8A
:1004D000010E266F770E256F86ECCEF04EEC8DF078
:1004E0007FEC8DF08A0E9C25186F196B010E192375
:1004F00090EC2EF0DF6E7FEC8DF0DF5004E09C2B53
:100500000F0E9C65EDD71F0E47EC8DF0FC0E246F8F
:100510002C0E236F010E266F770E256F86ECCEF022
:100520004EEC8DF07FEC8DF0850E9C25186F196BCD
:10053000010E192390EC2EF0DF6E7FEC8DF0DF5072
:1005400004E09C2B040E9C65EDD71F0E47EC8DF04C
:10055000F90E246FD20E236F010E266F770E256FD2
:1005600086ECCEF04EEC8DF07FEC8DF009EC8EF049
:1005700090EC2EF0DF6E7FEC8DF0DF5004E09C2BD2
:100580000F0E9C65F1D71F0E47EC8DF0FC0E246F0B
:10059000350E236F010E266F770E256F86ECCEF099
:1005A0004EEC8DF07FEC8DF002EC8EF090EC2EF0A6
:1005B000DF6E7FEC8DF0DF5004E09C2B040E9C6519
:1005C000F1D71F0E47EC8DF0F90E246FDD0E236F6F
:1005D000010E266F770E256F86ECCEF021519D6FB0
:1005E0009D519E27196B750E186F90EC2EF09D6F24
:1005F000D8909D33030E9D171F0E47EC8DF0F80E1B
:10060000246FB00E236F9DC125F1266B86ECCEF0D2
:100610002CEF8DF0C4518B0A01E011D10501D46B90
:1006200001019E6B050E9AEC8DF086ECCEF0215107
:100630009D6F9D519E271F0E47EC8DF0F10E246F8C
:100640003C0E236FF2C225F1266B86ECCEF02151D1
:100650009D6F9D519E271F0E47EC8DF0F60E246F67
:10066000880E236FE1C225F1266B86ECCEF0215176
:100670009D6F9D519E271F0E47EC8DF0F40E246F49
:10068000180E236FDDC125F1266B86ECCEF02151CB
:100690009D6F9D519E271F0E47EC8DF0F40E246F29
:1006A000160E236FDEC225F1266B86ECCEF02151AB
:1006B0009D6F9D519E271F0E47EC8DF0F40E246F09
:1006C000B50E236FD7C325F1266B86ECCEF02151F2
:1006D0009D6F9D519E271EA40AD01F0E47EC8DF0E2
:1006E000F60E246F7C0E236F86ECCEF009D01F0E21
:1006F00047EC8DF0F40E246FA80E236F86ECCEF03D
:1007000021519D6F9D519E271F0E47EC8DF0FB0ED2
:10071000246FF60E236FDCC125F1266B86ECCEF03C
:1007200021519D6F9D519E271F0E47EC8DF0FE0EAF
:10073000246FFA0E236F86ECCEF021519D6F9D51F0
:100740009E270CAA0ED01F0E47EC8DF0FA0E246FD8
:10075000DE0E236F86ECCEF021519D6F9D519E27BA
:100760002ED00DAE0AD01F0E47EC8DF0FE0E246F7A
:10077000DC0E236F86ECCEF0EFD70DA40AD01F0E4F
:1007800047EC8DF0FD0E246FF00E236F86ECCEF05B
:10079000E3D708AE0AD01F0E47EC8DF0FD0E246F94
:1007A000E90E236F86ECCEF0D7D71F0E47EC8DF005
:1007B000FA0E246FE80E236F86ECCEF0CDD71F0E15
:1007C00047EC8DF0FF0E246F000E236F86ECCEF009
:1007D00021519D6F9D519E270CAC0FD01F0E47ECF1
:1007E0008DF0FD0E246F420E236F86ECCEF021516A
:1007F0009D6F9D519E272CEF8DF00EA00AD01F0EED
:1008000047EC8DF0FF0E246FCC0E236F86ECCEF0FC
:10081000EED70DA60AD01F0E47EC8DF0FF0E246F09
:10082000830E236F86ECCEF0E2D71F0E47EC8DF0DF
:10083000FD0E246F4A0E236F86ECCEF0D8D7C4513C
:100840008C0A01E06AD10501D46B050E01019AEC16
:100850008DF086ECCEF021519D6F9DC19EF1500E22
:10086000196FEA0E186F90EC2EF0550A17E11F0E63
:1008700047EC8DF0F80E246F680E236F86ECCEF0F7
:1008800021519D6F500E186FEA0E176F000E196BF5
:1008900050EC35F001019D519E275AD0500E196F32
:1008A000EA0E186F90EC2EF0430A0AE11F0E47EC97
:1008B0008DF0F00E246F9F0E236F86ECCEF0E0D704
:1008C000500E196FEA0E186F90EC2EF0470A0AE1ED
:1008D0001F0E47EC8DF0EF0E246F6F0E236F86EC2A
:1008E000CEF0CED7500E196FEA0E186F90EC2EF0A6
:1008F000410A0AE11F0E47EC8DF0EF0E246F810EC6
:10090000236F86ECCEF0BCD7500E196FEA0E186F2D
:1009100090EC2EF0530A0AE11F0E47EC8DF0ED0E1D
:10092000246FCF0E236F86ECCEF0AAD7500E196F2E
:10093000EA0E186F90EC2EF0540A0AE11F0E47ECF5
:100940008DF0EF0E246F930E236F86ECCEF098D7C8
:100950001F0E47EC8DF0FF0E246F6A0E236F070EFB
:10096000266F9B0E256F86ECCEF021519D6F9D5119
:100970009E271F0E47EC8DF0FF0E246F6A0E236F2B
:10098000080E266FD20E256F86ECCEF021519D6F9A
:100990009D519E271F0E47EC8DF0FF0E246F6A0EAF
:1009A000236F070E266F8B0E256F86ECCEF021513C
:1009B0009D6F9D519E271F0E47EC8DF0FE0E246FFC
:1009C0002F0E236F86ECCEF04EEC8DF07FEC8DF089
:1009D000ED0E9C25186F196B000E192390EC2EF06C
:1009E000DF6E7FEC8DF0DF5004E09C2B080E9C65E1
:1009F000EDD71F0E47EC8DF0FE0E246F050E236F12
:100A0000010E266F770E256F86ECCEF04EEC8DF042
:100A10007FEC8DF0F60E9C25186F196B000E1923D4
:100A200090EC2EF0DF6E7FEC8DF0DF5004E09C2B1D
:100A3000080E9C65EDD71F0E47EC8DF0FE0E246F5F
:100A40000C0E236F010E266F770E256F86ECCEF00D
:100A50004EEC8DF07FEC8DF0980E9C25186F196B85
:100A6000000E192390EC2EF0DF6E7FEC8DF0DF503E
:100A700004E09C2B1A0E9C65EDD71F0E47EC8DF001
:100A8000FC0E246F3E0E236F010E266F770E256F2E
:100A900086ECCEF04EEC8DF03C0E01019C25D96E1B
:100AA000DA6A070EDA22770E9C25E16EE26A010E01
:100AB000E222DFCFE7FF7FEC8DF0DF5004E09C2BDC
:100AC000130E9C65E9D71F0E47EC8DF0FF0E246FC7
:100AD000790E236F010E266F770E256F86ECCEF010
:100AE00021519D6F010E1C6F770E1B6FFA0E1E6F4A
:100AF000A60E1D6F206B050E1F6F47EC27F01C51D3
:100B00001B1101E076D61F0E47EC8DF0FC0E246F12
:100B1000740E236F86ECCEF06AD6C4518D0A01E0C4
:100B2000C1D30501D46B050E01019AEC8DF086EC62
:100B3000CEF021519D6F9DC19EF11F0E47EC8DF0AF
:100B4000FF0E246F060E236F86ECCEF021519D6FB1
:100B50009D519E27E0670AD01F0E47EC8DF0F90EDD
:100B6000246FE80E236F86ECCEF070D0E051080AB7
:100B70000AE11F0E47EC8DF0FE0E246F130E236F5B
:100B800086ECCEF063D0E051040A0AE11F0E47EC78
:100B90008DF0FC0E246F590E236F86ECCEF056D0EC
:100BA000E051060A0AE11F0E47EC8DF0FA0E246FA1
:100BB000FC0E236F86ECCEF049D0E0510C0A0AE11E
:100BC0001F0E47EC8DF0FD0E246FDB0E236F86ECBD
:100BD000CEF03CD0E051020A0AE11F0E47EC8DF046
:100BE000FD0E246F2A0E236F86ECCEF02FD0E0513D
:100BF0000A0A0AE11F0E47EC8DF0FD0E246FE20E8B
:100C0000236F86ECCEF022D0E0510E0A0AE11F0ECF
:100C100047EC8DF0F90E246FF30E236F86ECCEF0C7
:100C200015D0E0050AE11F0E47EC8DF0FF0E246F92
:100C3000650E236F86ECCEF009D01F0E47EC8DF0C9
:100C4000FB0E246F060E236F86ECCEF021519D6FB4
:100C50009D519E271F0E47EC8DF0FE0E246FF40E63
:100C6000236F86ECCEF021519D6F9D519E2712ACD3
:100C70000ED01F0E47EC8DF0FF0E246F7E0E236FFB
:100C800086ECCEF021519D6F9D519E2716D018A461
:100C90000AD01F0E47EC8DF0FF0E246FD00E236F8D
:100CA00086ECCEF0EFD71F0E47EC8DF0FE0E246FD2
:100CB000440E236F86ECCEF0E5D71F0E47EC8DF087
:100CC000FD0E246FD10E236F86ECCEF021519D6F67
:100CD0009D519E271F0E47EC8DF0F40E246F240EBD
:100CE000236F86ECCEF021519D6F9D519E2707A466
:100CF00035D00301BC510101616F0301BD510101F8
:100D0000626F636B646B6151C008156FA80E62550A
:100D1000166F000E6355176F000E6455186FA00E06
:100D2000196F050E1A6F000E1B6B1C6B44EC1AF04A
:100D300015C175F116C176F11F0E47EC8DF0F40E5A
:100D4000246FC20E236F75C125F176C126F186ECA2
:100D5000CEF021519D6F9D519E270AD01F0E47EC6A
:100D60008DF0FF0E246FC40E236F86ECCEF0F1D70A
:100D70001F0E47EC8DF0FD0E246FD10E236F86EC15
:100D8000CEF021519D6F9D519E271F0E47EC8DF097
:100D9000FF0E246FC00E236F86ECCEF021519D6FA5
:100DA0009D519E27E6A10DD01F0E47EC8DF0FB0E46
:100DB000246FAC0E236F86ECCEF021519D6F9D51B8
:100DC0009E27E6A30DD01F0E47EC8DF0F60E246F84
:100DD000260E236F86ECCEF021519D6F9D519E27EC
:100DE000E6A50DD01F0E47EC8DF0FA0E246F820E93
:100DF000236F86ECCEF021519D6F9D519E27E6A773
:100E00000DD01F0E47EC8DF0FA0E246F8C0E236F61
:100E100086ECCEF021519D6F9D519E27E6A90DD005
:100E20001F0E47EC8DF0F60E246F320E236F86EC0A
:100E3000CEF021519D6F9D519E271F0E47EC8DF0E6
:100E4000FD0E246FD10E236F86ECCEF021519D6FE5
:100E50009D519E2707AC0DD01F0E47EC8DF0FA0E6A
:100E6000246FF20E236F86ECCEF021519D6F9D51C1
:100E70009E271F0E47EC8DF0FF0E246F740E236F1C
:100E800086ECCEF021519D6F9D519E278AAE0DD0EC
:100E90001F0E47EC8DF0F60E246F260E236F86ECA6
:100EA000CEF021519D6F9D519E278AAC0DD01F0E13
:100EB00047EC8DF0FB0E246FAC0E236F86ECCEF06A
:100EC00021519D6F9D519E271F0E47EC8DF0FD0E09
:100ED000246FD10E236F86ECCEF021519D6F9D5172
:100EE0009E2714A26BD01F0E47EC8DF0FC0E246FD2
:100EF000860E236F86ECCEF021519D6F9D519E276B
:100F000009A00DD01F0E47EC8DF0FD0E246FE90EE9
:100F1000236F86ECCEF021519D6F9D519E270101DC
:100F2000196B540E186F90EC2EF0986F9851F00BCF
:100F30000BE11F0E47EC8DF0FD0E246F220EB5EC79
:100F40008DF086ECCEF036D09851F00B100A0BE104
:100F50001F0E47EC8DF0F60E246F740EB5EC8DF07D
:100F600086ECCEF027D09851F00B200A0BE11F0E33
:100F700047EC8DF0FD0E246F220EB5EC8DF086EC63
:100F8000CEF018D09851F00B300A0BE11F0E47EC51
:100F90008DF0F60E246F700EB5EC8DF086ECCEF071
:100FA00009D01F0E47EC8DF0FD0E246FCD0E236F80
:100FB00086ECCEF021519D6F9D519E271F0E47EC70
:100FC0008DF0FE0E246F3D0E236F86ECCEF0215186
:100FD0009D6F9D519E27010E54ECD9F029E31F0E01
:100FE00047EC8DF0FF0E246FAC0E236F86ECCEF035
:100FF00021519D6F9D519E27010E69EC3DF0000926
:101000000AE11F0E47EC8DF0FE0E246FEE0E236FEB
:1010100086ECCEF009D01F0E47EC8DF0FE0E246F4B
:10102000360E236F86ECCEF021519D6F9D519E2789
:10103000020E54ECD9F029E31F0E47EC8DF0FF0EA1
:10104000246FB40E236F86ECCEF021519D6F9D511D
:101050009E27020E69EC3DF000090AE11F0E47ECE5
:101060008DF0FE0E246FEE0E236F86ECCEF009D0CD
:101070001F0E47EC8DF0FE0E246F360E236F86ECAC
:10108000CEF021519D6F9D519E27030E54ECD9F057
:1010900029E31F0E47EC8DF0FF0E246FB80E236F6F
:1010A00086ECCEF021519D6F9D519E27030E69EC79
:1010B0003DF000090AE11F0E47EC8DF0FE0E246F93
:1010C000EE0E236F86ECCEF009D01F0E47EC8DF0AC
:1010D000FE0E246F360E236F86ECCEF021519D6FED
:1010E0009D519E27040E54ECD9F029E31F0E47ECC6
:1010F0008DF0FF0E246FBC0E236F86ECCEF02151D5
:101100009D6F9D519E27040E69EC3DF000090AE198
:101110001F0E47EC8DF0FE0E246FEE0E236F86EC53
:10112000CEF009D01F0E47EC8DF0FE0E246F360E68
:10113000236F86ECCEF021519D6F9D519E271F0E8F
:1011400047EC8DF0FD0E246FD10E236F86ECCEF0B0
:1011500021519D6F9D519E271F0E47EC8DF0FB0E78
:10116000246F100E236F86ECCEF021519D6F9D51A0
:101170009E274F0E196FD30E186F90EC2EF0616FF3
:1011800061AD0AD01F0E47EC8DF0F60E246F830E72
:10119000236F86ECCEF009D01F0E47EC8DF0F40ED5
:1011A000246FAF0E236F86ECCEF04EEC8DF01F0E49
:1011B00047EC8DF0FC0E246F7D0E236F86ECCEF095
:1011C00021519D6F9D519E27000E2CEC07F00009C8
:1011D0000FE01F0E47EC8DF0FD0E246FD40E236F31
:1011E00086ECCEF021519D6F010E9C6F9D519E2784
:1011F00001019C6710D01F0E9E25216F226B050EEA
:101200002223F40E246FAF0E236F86ECCEF0215113
:101210009D6F9D519E271F0E47EC8DF0FD0E246F94
:101220003A0E236F86ECCEF021519D6F9D519E2783
:1012300013AC23D01F0E47EC8DF0FF0E246FA40ECD
:10124000236F86ECCEF021519D6F9D519E2709A6FC
:101250000AD01F0E47EC8DF0FF0E246FB00E236FE7
:1012600086ECCEF0F9D31F0E47EC8DF0FF0E246F05
:10127000A80E236F86ECCEF0EFD316A00AD01F0E77
:1012800047EC8DF0FF0E246F0C0E236F86ECCEF032
:10129000E3D31F0EFCDBFF0E246FC40E236F86EC1E
:1012A000CEF0DAD3C4518E0A01E0E4D00501D46B4C
:1012B0001EA80CD0050E0101226F1F0E216FFE0E1D
:1012C000246FE80E236F86ECCEF00BD0050E0101E3
:1012D000226F1F0E216FFD0E246FFE0E236F86EC12
:1012E000CEF021519D6F9DC19EF19C6B7FEC8DF0E6
:1012F00009EC8EF090EC2EF0DF6E7FEC8DF0DF507D
:1013000004E09C2B1F0E9C65F1D71F0EC0DBFB0E6B
:10131000246FFF0E236F010E266F770E256F86EC6C
:10132000CEF0BCDBECDB02EC8EF090EC2EF0DF6E4E
:10133000E6DBDF5004E09C2B050E9C65F3D71F0E07
:10134000A6DBFC0E246F1A0E236F010E266F770E9C
:10135000256F86ECCEF0A2DBD2DBC00E9C25186F89
:10136000196B010E192390EC2EF0DF6EC8DBDF50F5
:1013700004E09C2B1F0E9C65EFD71F0E88DBFD0E33
:10138000246F320E236F010E266F770E256F86ECC9
:10139000CEF021519D6F9D519E271EA609D01F0E94
:1013A00076DBFE0E246FE20E236F86ECCEF008D0C3
:1013B0001F0E6DDBFD0E246FF70E236F86ECCEF053
:1013C0006DDB9DDBF10E9C25186F196B010E192347
:1013D00090EC2EF0DF6E93DBDF5004E09C2B0F0EC1
:1013E0009C65EFD71F0E53DBFC0E246F110E236F8D
:1013F000010E266F770E256F86ECCEF04FDB7FDB7C
:101400009C29186F196B020E192390EC2EF0DF6ED9
:1014100076DBDF5004E09C2B1F0E9C65F0D71F0E7F
:1014200036DBFC0E246F080E236F010E266F770E3D
:10143000256F86ECCEF032DB62DB210E9C25186F27
:10144000196B020E192390EC2EF0DF6E58DBDF5083
:1014500004E09C2B1F0E9C65EFD71F0E18DBFF0EC0
:10146000246F1E0E236F010E266F770E256F86ECFC
:10147000CEF0F2D2C4518F0A01E069D20501D46BDB
:1014800001019E6B050E226F1F0E216FFF0E246F50
:10149000880E236F86ECCEF021519D6F9D519E27C3
:1014A000500E196FBF0E186F90EC2EF0616F500E3A
:1014B000196FBE0E186F90EC2EF09B6F61519A6FF2
:1014C0001F0EE5DA5DDB86ECCEF021519D6F9D515C
:1014D0009E27500E196FC10E186F90EC2EF0616FA1
:1014E000500E196FC00E186F90EC2EF09B6F61516B
:1014F0009A6F1F0ECCDA4DDB86ECCEF021519D6F3A
:101500009D519E271F0EC3DAFF0E246FA80E236F76
:1015100086ECCEF021519D6F9D519E27500E196F84
:10152000C50E186F90EC2EF0616F500E196FC40E3F
:10153000186F90EC2EF09B6F61519A6F1F0EA7DA17
:101540001FDB86ECCEF021519D6F9D519E27500EE2
:10155000196FC30E186F90EC2EF0616F500E196F5B
:10156000C20E186F90EC2EF09B6F61519A6F1F0E98
:101570008EDA26DB86ECCEF021519D6F9D519E27A1
:10158000500E196FCB0E186F90EC2EF0616F500E4D
:10159000196FCA0E186F90EC2EF09B6F61519A6F05
:1015A0001F0E75DAF6DA86ECCEF021519D6F9D5153
:1015B0009E271F0E6CDAFF0E246FB00E236F86EC91
:1015C000CEF021519D6F9D519E27500E196FC90E6F
:1015D000186F90EC2EF0616F500E196FC80E186FD7
:1015E00090EC2EF09B6F61519A6F1F0E50DAC8DAA3
:1015F00086ECCEF021519D6F9D519E27500E196FA4
:10160000C70E186F90EC2EF0616F500E196FC60E5A
:10161000186F90EC2EF09B6F61519A6F1F0E37DAA6
:10162000CFDA86ECCEF021519D6F9D519E27500E52
:10163000196FCD0E186F90EC2EF0616F500E196F70
:10164000CC0E186F90EC2EF09B6F61519A6F1F0EAD
:101650001EDA9FDA86ECCEF021519D6F9D519E27B8
:101660001F0E15DAFF0E246F120E236F86ECCEF0DC
:1016700021519D6F9D519E27500E196FCF0E186FEF
:1016800090EC2EF0616F500E196FCE0E186F90EC2B
:101690002EF09B6F61519A6F1F0EF9D971DA86ECAB
:1016A000CEF021519D6F9D519E27500E196FD10E86
:1016B000186F90EC2EF0616F500E196FD00E186FEE
:1016C00090EC2EF09B6F61519A6F1F0EE0D961DA9A
:1016D00086ECCEF021519D6F9D519E271F0ED7D9CC
:1016E000FF0E246F180E236F86ECCEF021519D6FF4
:1016F0009D519E27500E196FE30E186F90EC2EF03F
:10170000616F500E196FE20E186F90EC2EF09B6F08
:1017100061519A6F1F0EBBD95CDA86ECCEF0215175
:101720009D6F9D519E271F0EB2D9FF0E246FC80ECC
:10173000236F86ECCEF021519D6F9D519E27500E58
:10174000196FE10E186F90EC2EF0616F500E196F4B
:10175000E00E186F90EC2EF09B6F61519A6F1F0E88
:1017600096D937DA86ECCEF021519D6F9D519E2798
:101770001F0E8DD9FF0E246F8D0E236F86ECCEF0D9
:1017800021519D6F9D519E27500E196FDB0E186FD2
:1017900090EC2EF0616F500E196FDA0E186F90EC0E
:1017A0002EF09B6F61519A6F1F0E71D9FC0E246F42
:1017B000620E236F9AC125F19BC126F186ECCEF013
:1017C00021519D6F9D519E27500E196FDD0E186F90
:1017D00090EC2EF0616F500E196FDC0E186F90ECCC
:1017E0002EF09B6F61519A6F1F0E51D9FC0E246F22
:1017F0006B0E236F9AC125F19BC126F186ECCEF0CA
:1018000021519D6F9D519E27500E196FD70E186F55
:1018100090EC2EF0616F500E196FD60E186F90EC91
:101820002EF09B6F61519A6F1F0E31D9FE0E246FFF
:10183000210E236F9AC125F19BC126F186ECCEF0D3
:1018400021519D6F9D519E27500E196FD90E186F13
:1018500090EC2EF0616F500E196FD80E186F90EC4F
:101860002EF09B6F61519A6F1F0E11D9FE0E246FDF
:10187000280E236F9AC125F19BC126F186ECCEF08C
:1018800021519D6F9D519E27500E196FDF0E186FCD
:1018900090EC2EF0616F500E196FDE0E186F90EC09
:1018A0002EF09B6F61519A6F1F0EF1D8FD0E246FC1
:1018B0001A0E236F9AC125F19BC126F186ECCEF05A
:1018C00021519D6F9D519E271F0EE1D8FF0E246F61
:1018D000920E236F86ECCEF021519D6F9D519E2775
:1018E000500E196FD30E186F90EC2EF0616F500EE2
:1018F000196FD20E186F90EC2EF09B6F61519A6F9A
:101900001F0EC5D83DD986ECCEF021519D6F9D515B
:101910009E27500E196FD50E186F90EC2EF0616F48
:10192000500E196FD40E186F90EC2EF09B6F615112
:101930009A6F1F0EACD8FF0E246F6F0E236F9AC1E3
:1019400025F19BC126F186ECCEF0F7EF83F0020182
:10195000F55127E00101C451260A09E0C451270AC4
:1019600006E0C451280A03E0C451290A75E10201C6
:10197000F50506E1050E010135D986ECCEF00ED055
:10198000F551020A0BE1050E0101226F1F0E216FB6
:10199000FA0E246FA60E236F86ECCEF00201F56BD3
:1019A0005BD00101C451300AD8B460BF05D0050E28
:1019B00019D986ECCEF050D060AF37D00501D46B8A
:1019C00000011EA42ED001019E6B660E05011F6F43
:1019D0000101A8D8660EDF6E9E2B1F0E7ED864D83C
:1019E000616F61390F0B5BEC43F0DF6E9E2B5CD8AF
:1019F0000F0B5BEC43F0E0D89D65F1D71F0E63D869
:101A00001F0E9E2575D85BEC43F080D85BEC43F04D
:101A1000DF6E9E2B9E51C6ECEFF0C4D894EC20F004
:101A20001BD0000E47ECB8F017D00501D48117A4E5
:101A300008D0010E01011E6F000EC6EC0BF0F0D8AD
:101A400002D001019E6B9E5147ECB8F09E5157ECBD
:101A5000E3F002E20101996B97C11EF501019E6B53
:101A600010D0650E9E25D96EDA6A010EDA220E0EAE
:101A700001019E25E16EE26A050EE222DFCFE7FF5B
:101A80009E2B97519E5D02E392EF80F0EAD7010111
:101A90009E25216F226B050E2223120021519D6F7E
:101AA0009D519E279C6B12001F0E01019E25D96E31
:101AB000DA6A050EDA22C10E9D25E16EE26A010E98
:101AC000E222E750120001019E25D96EDA6A050E66
:101AD000DA222C0EDF6E9E2B2C0C9E25D96EDA6A34
:101AE000050EDA222C0EDF6E9E2B010E9D6F010C6F
:101AF000D96EDA6A050EDA22C4390F0B1200770E9E
:101B00009C25D96EDA6A010EDA221200DF6E9E2B56
:101B10001F0E01019E25D96EDA6A050EDA22C45124
:101B20000F0B12009E2B1F0E9E25D96EDA6A050E32
:101B3000DA221200226F1F0E216FFE0E246F1A0E82
:101B4000236F130E266FFA0E256FFA0CD46B01016A
:101B50009E6B300E05011F6F0101300CD46B050E1A
:101B60000101226F1F0E216F1200236F98C161F1D6
:101B70000F0E61176129256F266B000E2623000CBE
:101B8000FF0E246FD80E236F9AC125F19BC126F159
:101B90001200FE0E246FD60E236F9AC125F19BC151
:101BA00026F112002D0E01019E25D96EDA6A05017B
:101BB000050EDA22DF6A000CDF6E9E2B9D2B020CD5
:101BC000FF0E246FDC0E236F9AC125F19BC126F115
:101BD0001200FE0E246FD00E236F9AC125F19BC117
:101BE00026F11200226F1F0E216FFD0E246F6F0E63
:101BF000236F12000E0E01019E25D96EDA6A050EC2
:101C0000DA221200BA0E9C25186F196B010E1923E7
:101C1000010C9A0E9C25186F196B010E1923010CEB
:101C2000090E01019E6F090C330E0301FF6F4686FA
:101C30000401FE69468246804684060EFF6FDAEC98
:101C40000FF0E96B1AD083500F0BE06F270ED26FA5
:101C5000100ED16F01D004000101D107D8A0D20726
:101C6000D129D8B4D229F7E183500F0BE01904E051
:101C7000E95103E0E90701D0E92BE9510A0AE3E160
:101C80000F0EE01BE06705D01780949C829C948423
:101C900050D0E051040A10E10B82949C9484AD94DE
:101CA0007E86090E7F6EC20EB06EAC8EAC88AD8A99
:101CB0009E9A9F9A9D8A3DD0E051060A02E11188C2
:101CC0002DD0E0510E0A08E1098A949C9484AD94C9
:101CD0007E867F6A340EE8D7E00508E11382F1883A
:101CE000F092F08EF088060E766E23D0E0510A0A4C
:101CF00003E0E0510C0A0AE10F8E0101E0510A0AEB
:101D000001E11084F19CF292F28813D0E051080AAC
:101D10000DE10001058A01EC40F09896949C9484B2
:101D2000AD947E86010E7F6E370EBED7E051020A5B
:101D3000ABE0080E0101E96F8D968D948A988A9622
:101D40008D9C8D9A8D8C8D8A8D868D848A888A86CD
:101D50008F808F808C8AEA0ED26F600ED16F01D097
:101D600004000101D107D8A0D207D129D8B4D229C3
:101D7000F7E18D9C8D9A8D968D948A988A968F9096
:101D80008F908C9AEA0ED26F600ED16F01D0040052
:101D90000101D107D8A0D207D129D8B4D229F7E1BF
:101DA000E92FD0D7D08EF28EF28C196BFF0E186906
:101DB00090EC2EF00301FF1916E00101196BFF0EE4
:101DC000186990EC2EF00301FF190DE02BECDEF00A
:101DD0000101186BFF0E1769FFC319F150EC35F0C4
:101DE000010E0101E96F41ECB0F0420E0101196FE3
:101DF0003B0E186F90EC2EF00601F96FF929D8B45C
:101E00008F80130E0101196F890E186F90EC2EF060
:101E10000601F96FF929D8B48F800501D55113E077
:101E2000050E01011C6FD50E1B6FFC0E1E6FDA0E26
:101E30001D6F206B070E1F6F47EC27F01C511B1105
:101E400002E01EA40E8C0701AB5102E01EA40E8C12
:101E5000B8C3D1F1B9C3D2F10301B96B020EB86FA7
:101E6000000146941BEC45F0FFEC44F03D0E0101EF
:101E7000295D000E2A59F8E3D1C1B8F3D2C1B9F3F4
:101E800023EC2DF0DA6B148E1580048E0580000192
:101E9000189EB3EC3AF086CFE8F1E8A916D0270EE9
:101EA000D26F100ED16FD107D8A0D2070101D1296E
:101EB000D8B4D229F8E186CFE8F1E8A906D000012C
:101EC0000F82000E86EC3CF03FD0ACECC1F013B0BA
:101ED0003BD01A8A169E1584500E0101186FC00E51
:101EE000176F000E196B50EC35F0500E0101186F92
:101EF000C10E176F000E196B50EC35F034ECE5F0A5
:101F000018A622D08D8C8D8AEA0E0101D26F600E48
:101F1000D16F01D000F00101D107D8A0D207D1299B
:101F2000D8B4D229F7E18D9C8D9AEA0ED26F600E5B
:101F3000D16F01D000F00101D107D8A0D207D1297B
:101F4000D8B4D229DFE0F6D712B014AA01D00E8699
:101F500012A005D000010EA602D0FF00FFD700019D
:101F600012A005D08D8C8D9A010E5EECB4F012B0EB
:101F70000FA215D086CFE8F10101E8B910D0270EE5
:101F8000D26F100ED16FD107D8A0D2070101D1298D
:101F9000D8B4D229F8E186CFE8F1E8A9FF0012B061
:101FA0001BD086CFE8F10101E8A916D0270ED26F29
:101FB000100ED16FD107D8A0D2070101D129D8B412
:101FC000D229F8E186CFE8F1E8A906D000010F8216
:101FD000010E86EC3CF0B8D704B015A40BD01594D4
:101FE0008D9C158A17A006D0040EBB6E9E949F94FC
:101FF0009D84948C000112B009D0F4EC05F003012B
:10200000EA6FEA5103E0EA510CECC4F013AE06D0DB
:102010000301DF6703D02AEC2BF0139E040E0301AB
:10202000D5650AD0D56B500E0101206FDE0E1F6FF3
:1020300057EC37F0ACECC1F003A403D003940301D8
:10204000CD2B040E0301CD650AD0CD6B500E0101DE
:10205000206FDE0E1F6F57EC37F0ACECC1F002AA18
:1020600009D0500E0101206FD60E1F6F57EC37F0CC
:10207000ACECC1F002A809D0500E0101206FD60EC1
:102080001F6F57EC37F0ACECC1F002AC10D0029CE3
:102090000301CB2B010ECB650AD0CB6B500E010197
:1020A000206FD80E1F6F57EC37F0ACECC1F002AECA
:1020B00010D0029E0301CC2B010ECC650AD0CC6B54
:1020C000500E0101206FD80E1F6F57EC37F0ACECAB
:1020D000C1F003AC04D00001039C4BECDFF009A875
:1020E0000FD00998500E0101206FBE0E1F6F57ECE4
:1020F00037F0500E0101206FC00E1F6F57EC37F004
:1021000012A00EA471D016BE6FD00BA217D0030E72
:102110000101176FF80E166F9EEC3FF0030E0101E0
:10212000276FF80E266FF9ECD5F05EE2030E010181
:10213000166FF80E156FDCEC2DF054D011A80FD0EF
:10214000030E0101176FF80E166F1CEC3FF0030E23
:102150000101206FF80E1F6F6CECD2F0E7D709AACF
:102160000FD0030E0101176FF80E166F1CEC3FF035
:10217000030E01012A6FF80E296FA7ECD7F0D5D70F
:102180000FAE0FD0030E0101176FF80E166FDAECC9
:1021900037F0030E0101276FF80E266F1AECBFF01F
:1021A000C4D713A20FD0030E0101176FF80E166FDC
:1021B00050EC3FF0030E01011F6FF80E1E6F91EC03
:1021C00006F010D005BA05B60FD0030E0101176F47
:1021D000F80E166F93EC3EF00301F851080A02E185
:1021E000058602D0168E168C12A00FAE3ED041503E
:1021F000080A25E110B406D00301EE51EB0A1FE1F5
:102200000C841DD00101D5B51AD0D5A30FD0030180
:10221000EE51A50A14E0020E0101D5170301EE519B
:10222000EB0A0DE1040E0101D56F09D00301EE5157
:10223000A50A05E10101D5B1E3D7D581D5831AB44B
:102240000BD01AA203D01A920301E96B0301E9A78C
:102250000CD01A84148609D00C841AA206D01A92C3
:102260000301E96B1A9410AA148812A005AA90D051
:1022700016BA29D00101D8678BD005A611D00588E0
:10228000FBC316F1F9C317F1010E186F0301FA51E0
:10229000FAEC12F0168A059CF00E0101D86F78D086
:1022A0000301C02B450E0101166FC0C317F1186B57
:1022B000540EFAEC12F00301C0510F0AEBE1C06BAF
:1022C0008F801388E7D70101D8670AD0169A0001DA
:1022D00005B803D076EC1CF05BD00598059658D075
:1022E00005AC56D005A802D005980596059C169A0F
:1022F0000301EE51240A06E0EE515E0A03E0EE51BE
:10230000260A2FE1EE51240A02E1189C04D0EE5176
:102310005E0A03E1188C059E02D0189C058E03010D
:10232000C15123EEEFF0DF621CD04050120A03E0EF
:102330004050060A16E140506AEC2BF012E303010C
:10234000EF5127EC43F0D66F4050120A1EE109A26C
:102350000BD0150E0101166FC0C317F1186BFAEC04
:1023600012F076EC1CF098D7060E0101166FC0C370
:1023700017F1186BFAEC12F069EC13F0030E01017F
:10238000176FEE0E166FD4EC40F06EEC3BF084D776
:1023900012A013A213D013A608D013960301E96B61
:1023A0001AA40CD01A94148809D00301E9A306D00A
:1023B000E96B1AB403D01A8414860C8412B004D0CA
:1023C000000114B2C4ECE7F012A01BBA00D118A8A7
:1023D000FED0189818A417AC78D012BE76D00001A1
:1023E00013AC08D0F8EC44F02AEC2BF01682010E66
:1023F0000101E96F310ED7EC0CF0E86FE8511AECEF
:1024000012F00DE2000118B023D01880178E500E84
:102410000101206FD00E1F6F57EC37F019D000016B
:1024200004901BEC45F009D0000104A006D018A0D0
:102430000CD0189018820E9208D0FFEC44F0410E98
:102440000101295D9C0E2A59EFE3000104A0DAD7AF
:10245000300ED7EC0CF0E86FEA6BE8511AEC12F092
:102460000EE2010E0101EA6F17B821D01788178616
:10247000500E206FCE0E1F6F57EC37F018D00001B2
:1024800004901BEC45F009D0000104A006D017A869
:102490000CD01798178A0E9208D0FFEC44F0410E2A
:1024A0000101295D9C0E2A59EFE304A0DAD701014E
:1024B000EA5103E0ACECC1F002D0F1EC2FF00101E5
:1024C000E95101E184D01B8082D018B412BC7FD0C6
:1024D000000113AC08D0F8EC44F02AEC2BF0168283
:1024E000010E0101E96F300ED7EC0CF0E86FEA6BDA
:1024F000E8511AEC12F00EE2010E0101EA6F17B872
:1025000028D017881786500E206FCE0E1F6F57ECFD
:1025100037F01FD0000104901BEC45F009D00001FA
:1025200004A006D017A80CD01798178A0E9208D0CE
:10253000FFEC44F0410E0101295D9C0E2A59EFE3A6
:1025400004B007D0010E0101EA6F17B802D0178856
:1025500017860101EA5137E0310ED7EC0CF0E86F35
:10256000EA6BE8511AEC12F00EE2010E0101EA6F7B
:1025700018B021D01880178E500E206FD00E1F6F0C
:1025800057EC37F018D0000104901BEC45F009D04F
:10259000000104A006D018A00CD0189018820E924A
:1025A00008D0FFEC44F0410E0101295D9C0E2A5930
:1025B000EFE304A0DAD70101EA5103E0ACECC1F08B
:1025C00002D0F1EC2FF00101E95101E07CD712A01B
:1025D0001AAACED11A9AF10E0101176F3A0E166F90
:1025E000010E4EEC32F0130E01012A6F880E296F96
:1025F0002BEC37F00101E96B18A402D0010EE96F52
:102600000101E9512CEC07F0020A07E10301E82B74
:10261000E851020A04E1FF0002D00301E86BFA0E60
:102620000101176F340E166F010E4EEC32F0880E5A
:102630000101296F130E2A6F000E2B6B2C6B2D6B73
:10264000F2EC9FF00101E86FF80E176FEB0E166FBA
:10265000010E4EEC32F0880E0101296F130E2A6F25
:10266000000E2B6B2C6B2D6BF2EC9FF00101E86FD1
:10267000030EE96F0301D12B18D0FE0E176F520E17
:10268000166F010E4EEC32F0880E0101296F130E09
:102690002A6F000E2B6B2C6B2D6BF2EC9FF001015F
:1026A000E86FE851230A04E0E9070101E967E5D78B
:1026B000E9512BE00301D16B0101EA6B8F0E01019F
:1026C000EA25D96EDA6A060EDA229B0EEA25E16E59
:1026D000E26A070EE222DFCFE7FF8F0EEA25D96E0E
:1026E000DA6A060EDA22DF5004E0EA2B0F0EEA6502
:1026F000E5D7880E0101296F130E2A6F2B6B2C6B07
:10270000010E2D6FF2EC9FF007D0020E0301D16590
:1027100003D0D16BACECC1F0030E0101E96F0301F2
:10272000CE2B69D0FC0E176FBA0E166F010E4EEC51
:1027300032F0880E0101296F130E2A6F000E2B6BE9
:102740002C6B2D6BF2EC9FF00101E86FC06BEA6B14
:102750008F0E0101EA25D96EDA6A060EDA22D20E50
:10276000EA25E16EE26A080EE222DFCFE7FFC05100
:10277000030A0BE18F0EEA25D96EDA6A060EDA2219
:10278000370EDF6202D08C8A0ED00101C051030ADD
:102790000AE18F0EEA25D96EDA6A060EDA22300EC9
:1027A000DF6201D08C9A8F0E0101EA25D96EDA6AB8
:1027B000060EDA222C0EDF6201D0C02B8F0E010133
:1027C000EA25D96EDA6A060EDA22DF5004E0EA2B37
:1027D0001F0EEA65BDD7880E0101296F130E2A6FFF
:1027E0002B6B2C6B010E2D6FF2EC9FF00101E85169
:1027F000130A04E0E9070101E96794D7E95103E00E
:102800000301CE6B07D0020E0301CE6503D0CE6B61
:10281000ACECC1F062EC0FF017E2500E0101206F3A
:10282000DA0E1F6F57EC37F0ACECC1F017B812AEF0
:1028300001D00E8218B012AC01D00E8217B818A0C9
:1028400001D00E8216B01B80030E0101E96F030157
:10285000CA2B4FD0FB0E176F780E166F010E4EEC81
:1028600032F0880E0101296F130E2A6F000E2B6BB8
:102870002C6B2D6BF2EC9FF00101E86FEA6B8F0E71
:102880000101EA25D96EDA6A060EDA228B0EEA25F4
:10289000E16EE26A070EE222DFCFE7FF8F0EEA2544
:1028A000D96EDA6A060EDA22DF5004E0EA2B0F0E48
:1028B000EA65E5D7880E0101296F130E2A6F2B6B8D
:1028C0002C6B010E2D6FF2EC9FF00101E8511C0AF8
:1028D00013E0E8511D0A10E0E8511E0A0DE0E8512E
:1028E0001F0A0AE0E851200A07E0E851210A04E043
:1028F000E9070101E967AED7E9510CE0E851200A88
:1029000009E0E8511E0A06E0E8511F0A03E003014E
:10291000CA6B0ED0040E0301CA650AD0CA6B500EF2
:102920000101206FDC0E1F6F57EC37F0ACECC1F0EB
:10293000A00E0601F96F070EFA6FF9C61BF1FAC671
:102940001CF1FCEC17F01B51E86FE851630A03E13E
:102950000301D86B0DD00B0EE86102D0010E06D03A
:10296000100EE86102D0020E01D0030E0301D86FF1
:1029700012B0A1D21AB014AC01D0158214BC1AA0A6
:10298000159219BE07AC01D0088A07BC19AE089A87
:1029900013BC07A609D0050E0101536F1F0E526F1D
:1029A000000E546B35ECA6F012A405D00301BF5104
:1029B000BE11D8B4FF0012A604D000011296ACECF0
:1029C000C1F013BC03AE1DD0039EF80E0101176FBA
:1029D000BC0E166F010E4EEC32F0F8EC44F016828D
:1029E00009B608D0500E0101206FC20E1F6F57ECC0
:1029F00037F007D0500E0101206FC60E1F6F57EC45
:102A000037F01AAE0ED01A9E13AC0BD0000109A6F7
:102A100008D0F8EC44F02AEC2BF0069809961B80BD
:102A20000B881BA0F3D013AC16A0EBD004B008BAEF
:102A3000E8D015B2E6D016B28AD006B843D001016C
:102A4000E96BD50E0101E925D96EDA6A050EDA22A5
:102A5000CD0EE925186F196B000E192390EC2EF09E
:102A6000DF6ED50E0101E925D96EDA6A050EDA228C
:102A7000DF5004E0E92B0F0EE965E3D70101E96BB4
:102A8000F50E0101E925D96EDA6A050EDA22C80EC3
:102A9000E925186F196B000E192390EC2EF0DF6EEC
:102AA000F50E0101E925D96EDA6A050EDA22DF504A
:102AB00004E0E92B040EE965E3D70FB806880001AE
:102AC000099647D000010FA844D00101E96BD50E4B
:102AD0000101E925D96EDA6A050EDA228A0EE925A6
:102AE000186F196B010E192390EC2EF0DF6ED50EC6
:102AF0000101E925D96EDA6A050EDA22DF5004E019
:102B0000E92B0F0EE965E3D70101E96BF50E010131
:102B1000E925D96EDA6A050EDA22850EE925186FE5
:102B2000196B010E192390EC2EF0DF6EF50E0101EA
:102B3000E925D96EDA6A050EDA22DF5004E0E92BC6
:102B4000040EE965E3D706980001098602D000016A
:102B5000169262EC0FF015AE0AD0020E02019C6FC5
:102B6000000E9BEC30F00101E96F159E08D0010EBC
:102B700002019C6F000E9BEC30F00101E96F010136
:102B8000E90506E0E951020A03E0E951040A20E1FF
:102B900009B608D0500E0101206FCA0E1F6F57EC06
:102BA00037F007D0500E0101206FCC0E1F6F57EC8D
:102BB00037F00FA80BD009B603D00301DA8102D099
:102BC0000301DA83DA51030A19E1DA6B0D8A16D0B0
:102BD000E96714D00301DA6B0D9A09B608D0500EDC
:102BE0000101206FC40E1F6F57EC37F007D0500E55
:102BF0000101206FC80E1F6F57EC37F00301DB6B2C
:102C00001A9E0BA802D00B9801D01B9013BC15A6DE
:102C100054D00001159642EC42F00101E96F030126
:102C2000EA5104E0EA6BEA510CECC4F00101E967F7
:102C300001D0168203AE17D009B608D0500E01019C
:102C4000206FC20E1F6F57EC37F007D0500E0101F6
:102C5000206FC60E1F6F57EC37F00001039EF8EC93
:102C600044F016822AD00101E95103E0E951050A36
:102C700016E109B608D0500E0101206FC20E1F6F79
:102C800057EC37F007D0500E0101206FC60E1F6FB2
:102C900057EC37F0F8EC44F02AEC2BF00ED0E95169
:102CA000030A04E1010E0CECC4F007D0E951040A58
:102CB00004E1010E0CECC4F015860EAA0BD0139C97
:102CC0000E9A0E9C16900301CF6B00011A9A2AEC03
:102CD0002BF0F1D00EACEFD00E9C13BCECD01680D4
:102CE0000101E96BD50E0101E925D96EDA6A050EFD
:102CF000DA22CD0EE925186F196B000E192390EC1E
:102D00002EF0DF6ED50E0101E925D96EDA6A050EC7
:102D1000DA22DF5004E0E92B0F0EE965E3D7010169
:102D2000E96BF50E0101E925D96EDA6A050EDA22A2
:102D3000C80EE925186F196B000E192390EC2EF0C0
:102D4000DF6EF50E0101E925D96EDA6A050EDA2289
:102D5000DF5004E0E92B040EE965E3D709960698F5
:102D600000010FA802D00001068862EC0FF0D7C363
:102D70009CF2000E9BEC30F00101E96F159EE90515
:102D800005E118B402D00D8801D00D820101E9518E
:102D9000020A03E0E951040A55E10F800FA852D05E
:102DA0000101E96BD50E0101E925D96EDA6A050E3C
:102DB000DA228A0EE925186F196B010E192390EC9F
:102DC0002EF0DF6ED50E0101E925D96EDA6A050E07
:102DD000DA22DF5004E0E92B0F0EE965E3D70101A9
:102DE000E96BF50E0101E925D96EDA6A050EDA22E2
:102DF000850EE925186F196B010E192390EC2EF042
:102E0000DF6EF50E0101E925D96EDA6A050EDA22C8
:102E1000DF5004E0E92B040EE965E3D709860001E1
:102E2000069862EC0FF0D7C39CF2000E9BEC30F0DA
:102E30000101E96F159EE951020A03E0E951040A14
:102E400001E10E8E0101E951050A01E1088C010141
:102E5000E90506E0E951020A03E0E951040A13E139
:102E600009B608D0500E0101206FCA0E1F6F57EC33
:102E700037F007D0500E0101206FCC0E1F6F57ECBA
:102E800037F00D8A14D0E96712D00D9A09B608D030
:102E9000500E0101206FC40E1F6F57EC37F007D0A2
:102EA000500E0101206FC80E1F6F57EC37F01B90BA
:102EB0000301DB6B1A9E12B023D00FA402D00F9433
:102EC0001B8C46840101DA511AE080ECF5F0010117
:102ED000E96B11D0E951020D000EF324D96EDA6AC4
:102EE000060EDA220101DECF4EF1DDCF4FF101EC0B
:102EF000EFF004E3E92BDA51E95DECE3DA6B469499
:102F000012B0F7D004A0F4D00401EF51EE1101E0AB
:102F1000EFD0010E05EC38F015C1D9FF16C1DAFF6C
:102F2000DF50E86F020E05EC38F015C1D9FF16C16D
:102F3000DAFFDF50E827000119BA09D0030E05ECCB
:102F400038F015C1D9FF16C1DAFFDF50E827040EAB
:102F500005EC38F015C1D9FF16C1DAFFDF50E827BC
:102F6000050E05EC38F015C1D9FF16C1DAFFDF50A8
:102F7000E827E86711D00301ED6B0EA805D000012A
:102F80000E982AEC2BF0FF0000011BACB1D0010E13
:102F900086EC3CF01B9CACD00301ED2B050EED65DF
:102FA00002D0010EED6FED5105EC38F015C1D9FFDF
:102FB00016C1DAFFDF50E86FE86701D099D0EDC3A2
:102FC00018F1000E2CEC41F018C1D1F119C1D2F169
:102FD000EDC3EBF3D1C1F9F6D2C1FAF60D0E06013D
:102FE000FB6FD890FA33F933FB2FFBD7F951030B62
:102FF0000301C26FEB050DE1000113AC0AD0000E16
:103000000101D1115F6F800ED211606F00EC80F072
:1030100006D0D1C15FF1D2C160F100EC80F0E96F60
:10302000030E0401EF6FE80EEE6F0101E96706D0B1
:10303000EBC318F1000E90EC27F05AD013AC04D07B
:10304000010E0301EB6506D00301EB51030AD8A47E
:1030500062EC0FF013AC04D0010E0301EB6536D027
:103060000301D96745D000010C8087ECCCF019E250
:10307000500E0101206FE20E1F6F57EC37F0030175
:10308000EB51030A0AE11EA808D0D42B038CD451BB
:10309000050A03E1198AD46B049E0301EB29D36F5F
:1030A00013D00301CB6BCC6BEBC318F1000E90EC8B
:1030B00027F00301EB51030A04E11EA802D0D46BF0
:1030C000048E060E0301D96F0C9012D000010C8003
:1030D00038EC11F005E2020E0301D36FD52BF4D7C3
:1030E0000301D56BEBC318F1000E90EC27F0ECD781
:1030F00000F012B0A4EF8FF0000103A003D0000E87
:10310000AAEC11F0000103A2A4EF8FF0010EAAECCB
:1031100011F0A4EF8FF0E8CF5EF16DC615F101015B
:103120005E5131EC40F002E2D890120005012251CC
:10313000740A03E02251540A4FE12351720A03E05A
:103140002351520A16E1D351050AEEE10101616BE8
:10315000C20E6125176F186B500E1823000E196BE5
:1031600050EC35F00101612B250E6165F1D78AEF36
:103170009FF0050ED36101D0D7D725EED3F0070E0F
:10318000DF6401D0D1D71F0ED325D96EDA6A050EC0
:10319000DA22DF6A230E01015C6F050E5D6F5CC1F0
:1031A0001BF15DC11CF1FCEC17F01BC15FF11CC1F0
:1031B00060F1000E5F5D010E6059B6E260515F1173
:1031C000B3E05FC1F2F2186B550E176FF2C219F13E
:1031D00050EC35F08AEF9FF022516E0A03E0225145
:1031E0004E0A31E1050ED36101D09ED725EED3F012
:1031F000060EDF6401D098D71F0ED325D96EDA6A88
:10320000050EDA22DF6A230E01015C6F050E5D6F89
:103210005CC11BF15DC11CF1FCEC17F01BC15FF13F
:103220001CC160F1110E5F5D000E605901E37CD797
:103230005FC1DCF1186B760E176FDCC119F150EC31
:1032400035F08AEF9FF02251690A04E02251490AC1
:1032500001E0AED02351690A03E02351490A5CE141
:103260000C0ED36101D060D725EED3F0140EDF64CD
:1032700001D05AD7050E0101616F21D01F0E010147
:103280006125D96EDA6A050EDA22D00E6125E16E6B
:10329000E26A050EE222DFCFE7FF850E6125176F98
:1032A000186B010E18231F0E6125D96EDA6A050E00
:1032B000DA22DF50196F50EC35F00101612B050166
:1032C000D3510101615DDAE3D10E6125D96EDA6A6D
:1032D000050EDA22DF6A850E6125176F186B010E65
:1032E0001823000E196B50EC35F00F980501D551DD
:1032F00057E0050E01011C6FD50E1B6FFC0E1E6FF3
:10330000DA0E1D6F206B070E1F6F47EC27F01C5164
:103310001B1146E00F8844D00B0ED36101D004D7B7
:1033200025EED3F0130EDF6401D0FED6040E0101AA
:10333000616F21D01F0E01016125D96EDA6A050E79
:10334000DA22D10E6125E16EE26A050EE222DFCFBC
:10335000E7FFC90E6125176F186B000E18231F0EAB
:103360006125D96EDA6A050EDA22DF50196F50EC4A
:1033700035F00101612B0501D3510101615DDAE3F3
:10338000D10E6125D96EDA6A050EDA22DF6AC90E1E
:103390006125176F186B000E1823196B50EC35F070
:1033A00006980996000113BCCFEC43F08AEF9FF01A
:1033B0002251610A04E02251410A01E0BED02351AA
:1033C000610A03E02351410A4CE1060ED36101D0AA
:1033D000ABD625EED3F01F0EDF6401D0A5D6050EC7
:1033E0000101616F24D018A40FD01F0E01016125C7
:1033F000D96EDA6A050EDA226B0E6125E16EE26A99
:10340000070EE222DFCFE7FF1B0E01016125176FD8
:10341000186B030E18231F0E6125D96EDA6A050E8C
:10342000DA22DF50196F50EC35F00101612B0501F4
:10343000D3510101615DD7E318A407D06B0E61255C
:10344000D96EDA6A070EDA22DF6A1B0E01016125E6
:10345000176F186B030E1823000E196B50EC35F024
:103460004AD0050ED36101D05FD625EED3F01E0EF3
:10347000DF6401D059D6040E0101616F24D018B465
:103480000FD01F0E01016125D96EDA6A050EDA220E
:103490006C0E6125E16EE26A070EE222DFCFE7FFE4
:1034A000940E01016125176F186B000E18231F0E73
:1034B0006125D96EDA6A050EDA22DF50196F50ECF9
:1034C00035F00101612B0501D3510101615DD7E3A5
:1034D00018B407D06C0E6125D96EDA6A070EDA22AD
:1034E000DF6A940E01016125176F186B000E182317
:1034F000196B50EC35F013BC55D7EF0E0101176F67
:10350000A50E166F010E4EEC32F0070E0101176F7B
:10351000700E166F000E4EEC32F0220ECBEC42F025
:103520000D0ECBEC42F0130E01012A6F880E296FAD
:103530002BEC37F019EC1CF035D72251700A03E060
:103540002251500A7CE12351700A03E02351500AB2
:1035500031E1060ED36101D0E7D525EED3F0090E97
:10356000DF6401D0E1D5050E0101616F13D0800E3B
:103570006125176F186B010E18231F0E01016125BD
:10358000D96EDA6A050EDA22DF50196F50EC35F089
:103590000101612B0501D3510101615DE8E3800E5A
:1035A0006125176F186B010E1823000E196B50EC74
:1035B00035F0F6D6050ED36101D0B6D525EED3F0A1
:1035C000080EDF6401D0B0D5040E0101616F21D077
:1035D0001F0E01016125D96EDA6A050EDA22F10E9D
:1035E0006125E16EE26A050EE222DFCFE7FFC40E3D
:1035F0006125176F186B000E18231F0E6125D96EF9
:10360000DA6A050EDA22DF50196F50EC35F001014D
:10361000612B0501D3510101615DDAE3F10E6125F2
:10362000D96EDA6A050EDA22DF6AC40E6125176FD9
:10363000186B000E1823196B50EC35F0B1D62251DF
:10364000640A03E02251440A57E12351690A03E066
:103650002351490A51E125EED3F0140EDF6401D065
:1036600063D5D351050A0CE1010E0101186F750EE7
:10367000176F000E196B50EC35F00701AB6B92D64B
:10368000050E0101616F21D01F0E01016125D96E68
:10369000DA6A050EDA22A60E6125E16EE26A070EED
:1036A000E222DFCFE7FF700E6125176F186B010E66
:1036B00018231F0E6125D96EDA6A050EDA22DF5053
:1036C000196F50EC35F00101612B0501D351010157
:1036D000615DDAE3A60E6125D96EDA6A070EDA2299
:1036E000DF6A700E6125176F186B010E1823000E2C
:1036F000196B50EC35F056D62251640A03E0225182
:10370000440A4CE12351640A03E02351440A46E190
:1037100025EED3F0250EDF6401D006D5060ED36169
:1037200001D002D5050E0101616F21D01F0E0101EC
:103730006125D96EDA6A050EDA224B0E6125E16E3B
:10374000E26A070EE222DFCFE7FF500E6125176F16
:10375000186B010E18231F0E6125D96EDA6A050E4B
:10376000DA22DF50196F50EC35F00101612B0501B1
:10377000D3510101615DDAE34B0E6125D96EDA6A3E
:10378000070EDA22DF6A500E6125176F186B010EE3
:103790001823000E196B50EC35F004D62251770A2D
:1037A00003E02251570A69E125EED3F0130EDF64DE
:1037B00001D0BAD4050ED36101D0B6D4040E0101F4
:1037C000616F1CD01F0E01016125D96EDA6A0501F7
:1037D000050EDA22DF50800A500F01E2A5D41F0E39
:1037E00001016125D96EDA6A0501050EDA22DF5082
:1037F000800A460F01E398D40101612B0501D351E2
:103800000101615DDFE3040E616F21D01F0E010134
:103810006125D96EDA6A050EDA22B70E6125E16EEE
:10382000E26A070EE222DFCFE7FFAF0E6125176FD6
:10383000186B000E18231F0E6125D96EDA6A050E6B
:10384000DA22DF50196F50EC35F00101612B0501D0
:10385000D3510101615DDAE3B70E6125D96EDA6AF1
:10386000070EDA22DF6AAF0E6125176F186B000EA4
:103870001823196B50EC35F095D52251720A03E0EC
:103880002251520A34E1050ED36101D04DD425EE08
:10389000D3F0070EDF6401D047D41F0ED325D96EB5
:1038A000DA6A050EDA22DF6A230E01015C6F050E6B
:1038B0005D6F5CC11BF15DC11CF1FCEC17F01BC11D
:1038C0005FF11CC160F1000E5F5D010E605901E304
:1038D0002BD460515F1101E127D45FC1DEF2186B78
:1038E000730E176FDEC219F150EC35F013D322516D
:1038F0006F0A03E022514F0A36E1050ED36101D071
:1039000013D425EED3F0070EDF6401D00DD41F0EC3
:10391000D325D96EDA6A050EDA22DF6A230E010199
:103920005C6F050E5D6F5CC11BF15DC11CF1FCECB1
:1039300017F01BC15FF11CC160F1000E5F5D010E4D
:10394000605902E394EF98F060515F1102E194EF47
:1039500098F05FC1E1F2186B700E176FE1C219F1B8
:1039600050EC35F0D7D222516D0A03E022514D0AB6
:1039700038E1050ED36102D094EF98F025EED3F034
:10398000070EDF6402D094EF98F01F0ED325D96E96
:10399000DA6A050EDA22DF6A230E01015C6F050E7A
:1039A0005D6F5CC11BF15DC11CF1FCEC17F01BC12C
:1039B0005FF11CC160F1000E5F5D010E605902E312
:1039C00094EF98F060515F1102E194EF98F05FC1BD
:1039D000DDF1186B720E176FDDC119F150EC35F087
:1039E00099D22251660A03E02251460A39E1D351A5
:1039F000050A02E094EF98F00101196B750E186F3B
:103A000090EC2EF0616F05012351300A06E1199EFA
:103A10001A90F90E010161171AD02351310A06E1FB
:103A2000198E1A9001016183619511D02351320AD8
:103A300006E1199E1A8001016185619308D0235126
:103A4000330A05E1198E1A80060E01016113010186
:103A5000186B750E176F61C119F150EC35F05AD221
:103A60002251650A03E02251450A25E1D351050A96
:103A700002E094EF98F00101196B4F0E186F90EC73
:103A80002EF0616F05012351300A04E11E980101F7
:103A9000619908D02351310A05E11E88010161892D
:103AA0004BECDFF00101186B4F0E176F61C119F17C
:103AB00050EC35F02FD22251730A03E02251530A01
:103AC0000FE1D351050A02E094EF98F02351300A38
:103AD00001E120D22351310A01E11CD294EF98F088
:103AE0002251630A04E02251430A01E0D3D0D351AA
:103AF000050A20E12351310A03E100010A820AD2BA
:103B00002351320A03E100010A8404D22351330A0B
:103B100003E10001098EFED12351340A03E10001C3
:103B2000098CF8D12351360A02E094EF98F0000195
:103B30000A86F0D1D3510A0A44E1EF0E0101176F52
:103B4000C80E166F010E4EEC32F005012351CBEC7E
:103B500042F005012451CBEC42F03A0ECBEC42F09E
:103B600005012551CBEC42F005012651CBEC42F08A
:103B70003A0ECBEC42F005012751CBEC42F00501A7
:103B80002851CBEC42F0FE0E0101176F580E166F54
:103B9000000E4EEC32F0130E01012A6F880E296FD1
:103BA0002BEC37F002E3000117841BEC45F0FFEC2F
:103BB00044F0E90E0101295D030E2A5901E3AAD15F
:103BC000F6D7D351100A01E0A5D1FC0E0101176F01
:103BD000D20E166F010E4EEC32F005012751CBECE0
:103BE00042F005012851CBEC42F02F0ECBEC42F015
:103BF00005012551CBEC42F005012651CBEC42F0FA
:103C00002F0ECBEC42F005012351CBEC42F0050125
:103C10002451CBEC42F02C0ECBEC42F005012951A3
:103C2000CBEC42F005012A51CBEC42F03A0ECBEC42
:103C300042F005012B51CBEC42F005012C51CBECAD
:103C400042F03A0ECBEC42F005012D51CBEC42F0A4
:103C500005012E51CBEC42F0FE0E0101176F580EFC
:103C6000166F000E4EEC32F0130E01012A6F880E13
:103C7000296F2BEC37F002E3000117841BEC45F0B1
:103C8000FFEC44F0E90E0101295D030E2A5901E31E
:103C900041D1F6D72251790A05E02251590A02E0B2
:103CA00094EF98F02351790A04E02351590A01E076
:103CB00098D0060ED36102D094EF98F025EED3F0A1
:103CC0000E0EDF6402D094EF98F02451310A42E1E5
:103CD000060E0101616F24D018A40FD01F0E010140
:103CE0006125D96EDA6A050EDA22D90E6125E16EF8
:103CF000E26A060EE222DFCFE7FF350E0101612501
:103D0000176F186B030E18231F0E6125D96EDA6A20
:103D1000050EDA22DF50196F50EC35F00101612BEE
:103D20000501D3510101615DD7E318A407D0D90E75
:103D30006125D96EDA6A060EDA22DF6A350E0101D4
:103D40006125176F186B030E1823000E196B50ECCA
:103D500035F0DCD02451320A02E094EF98F0060EE0
:103D60000101616F24D018A40FD01F0E010161253D
:103D7000D96EDA6A050EDA22E20E6125E16EE26A98
:103D8000060EE222DFCFE7FF3E0E01016125176F2D
:103D9000186B030E18231F0E6125D96EDA6A050E03
:103DA000DA22DF50196F50EC35F00101612B05016B
:103DB000D3510101615DD7E318A407D0E20E61255C
:103DC000D96EDA6A060EDA22DF6A3E0E010161253B
:103DD000176F186B030E1823000E196B50EC35F09B
:103DE00095D0050ED36102D094EF98F025EED3F074
:103DF0000D0EDF6402D094EF98F02351310A41E1B7
:103E0000050E0101616F24D018B40FD01F0E0101FF
:103E10006125D96EDA6A050EDA22DA0E6125E16EC5
:103E2000E26A060EE222DFCFE7FFE80E010161251C
:103E3000176F186B000E18231F0E6125D96EDA6AF2
:103E4000050EDA22DF50196F50EC35F00101612BBD
:103E50000501D3510101615DD7E318B407D0DA0E33
:103E60006125D96EDA6A060EDA22DF6AE80E0101F0
:103E70006125176F186B000E1823196B50EC35F085
:103E800045D02351320A02E094EF98F0050E01016B
:103E9000616F24D018B40FD01F0E01016125D96EB7
:103EA000DA6A050EDA22E30E6125E16EE26A060E99
:103EB000E222DFCFE7FFF10E01016125176F186BDA
:103EC000000E18231F0E6125D96EDA6A050EDA225C
:103ED000DF50196F50EC35F00101612B0501D35112
:103EE0000101615DD7E318B407D0E30E6125D96EF7
:103EF000DA6A060EDA22DF6AF10E01016125176F18
:103F0000186B000E1823196B50EC35F0000113AC40
:103F100019EC1CF080ECF5F001015E39F00B616FDB
:103F20000AA207D00A928A0E406F615188ECF0F025
:103F300038D00AA408D00A948B0E0101406F615159
:103F400088ECF0F02ED009AE08D0099E8C0E01014D
:103F5000406F615188ECF0F024D009AC08D0099C86
:103F60008D0E0101406F615188ECF0F01AD00AA06B
:103F700008D00A908E0E0101406F615188ECF0F07C
:103F800010D00AA608D00A968F0E0101406F615129
:103F900088ECF0F006D0830E0101406F615188EC8F
:103FA000F0F040C15FF141C160F119A204D00001FD
:103FB0001992D880120006016D5198EC44F0F9E393
:103FC0005E5169EC3DF00101616F5FC139F160C183
:103FD0003AF15EC13BF161C13CF1030E3D6F56EC1D
:103FE00034F0E7D72D671BD005010A6B0B6B0C6B08
:103FF0000D6B0294029604D0C4ECE7F002B40FD02B
:1040000005010D51800A800F08E1000E0C5D05E1ED
:10401000EA0E0B5D02E1610E0A5DEEE30C0C050198
:104020000A6B0B6B0C6B0D6B02A6029408D0C4ECF0
:10403000E7F002A404D002940201CE6717D0010178
:104040002C51800A2E6F05010A510101295D0501DD
:104050000B5101012A5905010C5101012B59050190
:104060000D51800A01012E59D9E3E1D702960101D1
:104070002F6BA00E01012F25D96EDA6A080EDA2205
:104080008F0E2F25E16EE26A060EE222DFCFE7FFF8
:104090008F0E2F25D96EDA6A060EDA22DF5004E081
:1040A0002F2B310E2F65E5D7060E01011C6F8F0EE9
:1040B0001B6FF90E1E6F6F0E1D6F206B0A0E1F6FA8
:1040C00047EC27F01C511B1106E1000102A4020C71
:1040D00000010286020C060E01011C6F8F0E1B6F81
:1040E000F40E1E6F740E1D6F206B0C0E1F6F47ECCD
:1040F00027F01C511B1106E1000102A42F0C000146
:1041000002862F0C060E01011C6F8F0E1B6FFD0E19
:104110001E6F120E1D6F206B070E1F6F47EC27F0EE
:104120001C511B11D2E0060E01011C6F8F0E1B6F7C
:10413000EF0E1E6FD90E1D6F206B100E1F6F47EC18
:1041400027F01C511B1106E1000102A4060C00011E
:104150000286060C060E01011C6F8F0E1B6FFB0EF4
:104160001E6FB70E1D6F206B080E1F6F47EC27F0F8
:104170001C511B1106E1000102A4240C000102865F
:10418000240C060E01011C6F8F0E1B6FFD0E1E6F9F
:104190006F0E1D6F206B020E1F6F47EC27F01C5136
:1041A0001B1106E1000102A4080C00010286080CA4
:1041B000060E0101236F8F0E226F070E256FDB0E97
:1041C000246F21EC26F02351221106E0000102A405
:1041D000030C00010286030C060E01011C6F8F0EFA
:1041E0001B6FF90E1E6F200E1D6F206B010E1F6FCF
:1041F00047EC27F01C511B1106E1000102A40D0C35
:10420000000102860D0C060E01011C6F8F0E1B6F44
:10421000FB0E1E6FAC0E1D6F206B010E1F6F47EC67
:1042200027F01C511B1106E1000102A4100C000133
:104230000286100C060E01011C6F8F0E1B6FF60E0E
:104240001E6F260E1D6F206B010E1F6F47EC27F0AF
:104250001C511B1106E1000102A4110C0001028691
:10426000110C060E01011C6F8F0E1B6FEF0E1E6FDF
:10427000E80E1D6F206B010E1F6F47EC27F01C51DD
:104280001B1106E1000102A40F0C000102860F0CB5
:10429000060E01011C6F8F0E1B6FFE0E1E6F8E0E21
:1042A0001D6F206B050E1F6F47EC27F01C511B1173
:1042B00006E1000102A43A0C000102863A0C060E47
:1042C00001011C6F8F0E1B6FFF0E1E6F2E0E1D6FD8
:1042D000206B040E1F6F47EC27F01C511B1106E1E9
:1042E000000102A43B0C000102863B0C060E0101FA
:1042F0001C6F8F0E1B6FF60E1E6F040E1D6F206B52
:104300000B0E1F6F47EC27F01C511B1101E1DDD68E
:10431000060E01011C6F8F0E1B6FF60E1E6F280E0E
:104320001D6F206B0B0E1F6F47EC27F01C511B11EC
:1043300001E1E2D6060E01011C6F8F0E1B6FF60E17
:104340001E6F100E1D6F206B0B0E1F6F47EC27F0BA
:104350001C511B1106E1000102A4430C000102865E
:10436000430C060E01011C6F8F0E1B6FF00E1E6FAB
:104370004F0E1D6F206B0F0E1F6F47EC27F01C5167
:104380001B1106E1000102A4440C00010286440C4A
:10439000060E01011C6F8F0E1B6FEF0E1E6F030EBA
:1043A0001D6F206B110E1F6F47EC27F01C511B1166
:1043B00006E1000102A4450C00010286450C060E30
:1043C00001011C6F8F0E1B6FF00E1E6F3F0E1D6FD5
:1043D000206B0F0E1F6F47EC27F01C511B1106E1DD
:1043E000000102A4390C00010286390C060E0101FD
:1043F0001C6F8F0E1B6FFA0E1E6F980E1D6F206BB9
:10440000090E1F6F47EC27F01C511B1106E100013C
:1044100002A43E0C000102863E0C060E01011C6F38
:104420008F0E1B6FF30E1E6FDE0E1D6F206B0D0EB9
:104430001F6F47EC27F01C511B1106E1000102A47D
:10444000400C00010286400C060E01011C6F8F0E0D
:104450001B6FF90E1E6F170E1D6F206B0A0E1F6F5C
:1044600047EC27F01C511B1106E1000102A4420C8D
:1044700000010286420C060E01011C6F8F0E1B6F9D
:10448000F90E1E6F220E1D6F206B0A0E1F6F47EC78
:1044900027F01C511B1106E1000102A43F0C000192
:1044A00002863F0C060E01011C6F8F0E1B6FF40E6F
:1044B0001E6F5A0E1D6F206B0C0E1F6F47EC27F0FE
:1044C0001C511B1106E1000102A4410C00010286EF
:1044D000410C060E01011C6F8F0E1B6FF10E1E6F3B
:1044E0000F0E1D6F206B0E0E1F6F47EC27F01C5137
:1044F0001B1106E1000102A4090C00010286090C4F
:10450000060E01011C6F8F0E1B6FF30E1E6FFA0E4D
:104510001D6F206B0D0E1F6F47EC27F01C511B11F8
:1045200006E1000102A42C0C000102862C0C060EF0
:1045300001011C6F8F0E1B6FFA0E1E6FA20E1D6FF6
:10454000206B090E1F6F47EC27F01C511B11D2E0A6
:10455000060E01011C6F8F0E1B6FFA0E1E6FA60E4A
:104560001D6F206B050E1F6F47EC27F01C511B11B0
:10457000C1E0060E01011C6F8F0E1B6FFA0E1E6F3D
:10458000AC0E1D6F206B090E1F6F47EC27F01C51FE
:104590001B1106E1000102A4320C00010286320C5C
:1045A000060E01011C6F8F0E1B6FF90E1E6F2D0E74
:1045B0001D6F206B0A0E1F6F47EC27F01C511B115B
:1045C00006E1000102A41C0C000102861C0C060E70
:1045D00001011C6F8F0E1B6FF90E1E6F380E1D6FC1
:1045E000206B0A0E1F6F47EC27F01C511B1106E1D0
:1045F000000102A41D0C000102861D0C060E010123
:104600001C6F8F0E1B6FF90E1E6F430E1D6F206BFC
:104610000A0E1F6F47EC27F01C511B1106E1000129
:1046200002A41E0C000102861E0C060E01011C6F66
:104630008F0E1B6FF90E1E6F4E0E1D6F206B0A0E34
:104640001F6F47EC27F01C511B1106E1000102A46B
:104650001F0C000102861F0C060E01011C6F8F0E3D
:104660001B6FF90E1E6F590E1D6F206B0A0E1F6F08
:1046700047EC27F01C511B1106E1000102A4200C9D
:1046800000010286200C060E01011C6F8F0E1B6FAD
:10469000F90E1E6F640E1D6F206B0A0E1F6F47EC24
:1046A00027F01C511B1106E1000102A4210C00019E
:1046B0000286210C060E01011C6F8F0E1B6FFF0E70
:1046C0001E6FFC0E1D6F206B010E1F6F47EC27F055
:1046D0001C511B1106E1000102A4250C00010286F9
:1046E000250C060E01011C6F8F0E1B6FFD0E1E6F39
:1046F0006A0E1D6F206B070E1F6F47EC27F01C51D1
:104700001B1106E1000102A4260C00010286260C02
:10471000060E01011C6F8F0E1B6FFE0E1E6F880EA2
:104720001D6F206B050E1F6F47EC27F01C511B11EE
:1047300006E1000102A42B0C000102862B0C060EE0
:1047400001011C6F8F0E1B6FFB0E1E6FA50E1D6FE0
:10475000206B080E1F6F47EC27F01C511B1106E160
:10476000000102A4040C00010286040C060E0101E3
:104770001C6F8F0E1B6FFB0E1E6F9C0E1D6F206B30
:10478000080E1F6F47EC27F01C511B1106E10001BA
:1047900002A40B0C000102860B0C060E01011C6F1B
:1047A0008F0E1B6FFB0E1E6FAE0E1D6F206B080E63
:1047B0001F6F47EC27F01C511B1106E1000102A4FA
:1047C0000A0C000102860A0C060E01011C6F8F0EF6
:1047D0001B6FFD0E1E6FB80E1D6F206B060E1F6F38
:1047E00047EC27F01C511B1106E1000102A4150C37
:1047F00000010286150C060E01011C6F8F0E1B6F47
:10480000FE0E1E6F7C0E1D6F206B050E1F6F47EC9A
:1048100027F01C511B1106E1000102A4230C00012A
:104820000286230C060E01011C6F8F0E1B6FFD0EFE
:104830001E6FBF0E1D6F206B060E1F6F47EC27F01B
:104840001C511B1106E1000102A4130C0001028699
:10485000130C060E01011C6F8F0E1B6FFD0E1E6FD9
:10486000020E1D6F206B070E1F6F47EC27F01C51C7
:104870001B1106E1000102A4140C00010286140CB5
:10488000060E01011C6F8F0E1B6FFD0E1E6FB80E02
:104890001D6F206B060E1F6F47EC27F01C511B117C
:1048A000A4E0060E01011C6F8F0E1B6FFA0E1E6F27
:1048B0005C0E1D6F206B090E1F6F47EC27F01C511B
:1048C0001B1106E1000102A4180C00010286180C5D
:1048D000060E01011C6F8F0E1B6FFA0E1E6F660E07
:1048E0001D6F206B090E1F6F47EC27F01C511B1129
:1048F00006E1000102A4160C00010286160C060E49
:1049000001011C6F8F0E1B6FFA0E1E6F700E1D6F54
:10491000206B090E1F6F47EC27F01C511B1106E19D
:10492000000102A4190C00010286190C060E0101F7
:104930001C6F8F0E1B6FFA0E1E6F7A0E1D6F206B91
:10494000090E1F6F47EC27F01C511B1106E10001F7
:1049500002A41A0C000102861A0C060E01011C6F3B
:104960008F0E1B6FFA0E1E6F840E1D6F206B090ECB
:104970001F6F47EC27F01C511B1106E1000102A438
:104980001B0C000102861B0C060E01011C6F8F0E12
:104990001B6FFA0E1E6F8E0E1D6F206B090E1F6FA0
:1049A00047EC27F01C511B1106E1000102A4170C73
:1049B00000010286170C060E01011C6F8F0E1B6F83
:1049C000FE0E1E6F820E1D6F206B050E1F6F47ECD3
:1049D00027F01C511B1106E1000102A4270C000165
:1049E0000286270C060E01011C6F8F0E1B6FF60E40
:1049F0001E6F400E1D6F206B0B0E1F6F47EC27F0D4
:104A00001C511B1106E1000102A4280C00010286C2
:104A1000280C060E01011C6F8F0E1B6FF00E1E6F0F
:104A20006F0E1D6F206B0F0E1F6F47EC27F01C5190
:104A30001B1106E1000102A4350C00010286350CB1
:104A4000060E01011C6F8F0E1B6FF40E1E6F080EF9
:104A50001D6F206B0D0E1F6F47EC27F01C511B11B3
:104A600006E1000102A4290C00010286290C060EB1
:104A700001011C6F8F0E1B6FF00E1E6F5F0E1D6FFE
:104A8000206B0F0E1F6F47EC27F01C511B1106E126
:104A9000000102A4360C00010286360C060E01014C
:104AA0001C6F8F0E1B6FF60E1E6F340E1D6F206B6A
:104AB0000B0E1F6F47EC27F01C511B1106E1000184
:104AC00002A42D0C000102862D0C060E01011C6FA4
:104AD0008F0E1B6FF60E1E6F1C0E1D6F206B0B0EC4
:104AE0001F6F47EC27F01C511B1106E1000102A4C7
:104AF0002E0C000102862E0C060E01011C6F8F0E7B
:104B00001B6FF40E1E6F4D0E1D6F206B0C0E1F6F72
:104B100047EC27F01C511B1106E1000102A4300CE8
:104B200000010286300C060E01011C6F8F0E1B6FF8
:104B3000F40E1E6F670E1D6F206B0C0E1F6F47EC7F
:104B400027F01C511B1106E1000102A43C0C0001DE
:104B500002863C0C060E01011C6F8F0E1B6FF30EBC
:104B60001E6FEC0E1D6F206B0D0E1F6F47EC27F0B4
:104B70001C511B1106E1000102A4310C0001028648
:104B8000310C060E01011C6F8F0E1B6FF90E1E6F8C
:104B90000C0E1D6F206B0A0E1F6F47EC27F01C5187
:104BA0001B1106E1000102A43D0C000102863D0C30
:104BB000060E01011C6F8F0E1B6FFA0E1E6F480E42
:104BC0001D6F206B090E1F6F47EC27F01C511B1146
:104BD00006E1000102A4330C00010286330C060E2C
:104BE00001011C6F8F0E1B6FFA0E1E6F520E1D6F90
:104BF000206B090E1F6F47EC27F01C511B1106E1BB
:104C0000000102A4340C00010286340C060E0101DE
:104C10001C6F8F0E1B6FFD0E1E6FB10E1D6F206B74
:104C2000060E1F6F47EC27F01C511B1106E1000117
:104C300002A4370C00010286370C060E01011C6F1E
:104C40008F0E1B6FFD0E1E6F0A0E1D6F206B070E61
:104C50001F6F47EC27F01C511B1106E1000102A455
:104C6000380C00010286380C000C049604980101EF
:104C7000D96B0201D46BF76B01019C6B9D6B5405E2
:104C800001E0BFD000010B8A9C9EA8847C867D6ACF
:104C9000670EAB6E9C8E9C88A88AA49AA59AA38A5C
:104CA0008E9C8D981BEC45F0FFEC44F0590E0101F1
:104CB000295D020E2A59F8E38D881BEC45F0FFECC4
:104CC00044F0650E0101295D000E2A59F8E38E8C2F
:104CD000270E0201B36F100EB26F0001FC6B10D0F3
:104CE0000201B351B2110CE1EF0E0101166F270E54
:104CF000156F100E176FDDEC43F08E9C8D9812002F
:104D00000001FC51030AECE1030E0201B36FE80E4F
:104D1000B26F0001FC6BFF0E0101176FA00E166F42
:104D2000010E4EEC32F00ED00201B351B2110AE185
:104D3000EF0E0101166F390E156F100E176FDDECB7
:104D400043F0DBD70001FC05EFE1170E0201B36F62
:104D5000700EB26F0001FC6BFB0E0101176FD20EDB
:104D6000166F010E4EEC32F00ED00201B351B211AB
:104D70000AE1EF0E0101166F4B0E156F100E176F43
:104D8000DDEC43F0BAD70001FC05EFE1EE0E0101C6
:104D9000176F260E166F010E4EEC32F0010E010158
:104DA0002A6FF40E296F2BEC37F0170E0201B36F48
:104DB000700EB26F0001FC6BEC0E0101176F590E03
:104DC000166F010E4EEC32F00ED00201B351B2114B
:104DD0000AE1EF0E0101166F5D0E156F100E176FD1
:104DE000DDEC43F08AD70001FC51020AEEE1EF0E40
:104DF0000101166FEA0E156F100E176FDDEC43F010
:104E00009DD20796198CFA0E0101176FD40E166FFA
:104E1000010E4EEC32F04C0E01012A6F080E296F84
:104E20002BEC37F0ED0E0101176F2B0E166F010EF4
:104E30004EEC32F0130E01012A6F880E296F2BEC15
:104E400037F0EB0E0101176FE70E166F010E4EECF7
:104E500032F0130E01012A6F880E296F2BEC37F008
:104E6000EC0E0101176F380E166F010E4EEC32F08A
:104E7000070E01012A6FD00E296F2BEC37F0880E38
:104E80000101296F130E2A6F000E2B6B2C6B2D6BFB
:104E9000F2EC9FF00101AA6FAA51400A19E0F60E48
:104EA000176F580E166F010E4EEC32F0030E010113
:104EB0002A6FE80E296F2BEC37F0EE0E01012C6FF4
:104EC0008E0E2B6F2E6B130E2D6FACEC04F0C2D038
:104ED000F00E176F0C0E166F010E4EEC32F0070E2F
:104EE00001012A6FD00E296F2BEC37F0880E0101DB
:104EF000296F130E2A6F000E2B6B2C6B2D6BF2ECAF
:104F00009FF00101AA6FAA51420A0DE054EC39F05A
:104F1000EE0E01012C6FDE0E2B6F2E6B120E2D6F1D
:104F2000ACEC04F097D0EE0E176F260E166F010E44
:104F30004EEC32F0010E01012A6FF40E296F2BECBA
:104F400037F011AE33D00101A66BA6515225556F33
:104F5000000E5321566F0E0E5525D96E000E5621A8
:104F6000DA6EEB0E0101A625E16EE26A070EE2227F
:104F7000DFCFE7FFA62B060EA665E7D7F90E176F62
:104F8000BC0E166F010E4EEC32F0070E0101176FCA
:104F9000EB0E166F000E4EEC32F0EC0E0101176FA7
:104FA000AE0E166F000E4EEC32F042D1F10E010142
:104FB000176F2D0E166F010E4EEC32F0E80E010148
:104FC000296F030E2A6F000E2B6B2C6B2D6BF2ECEE
:104FD0009FF00101AA6FAA51020A0DE054EC39F0CA
:104FE000ED0E01012C6F8B0E2B6F2E6B130E2D6FA0
:104FF000ACEC04F02FD00C8E0201DD6B130E01011E
:105000002A6F880E296F2BEC37F0FC0E0201DD258C
:10501000D96EDA6A080EDA22DF6A0C9EE80E010108
:10502000296F030E2A6F000E2B6B2C6B2D6BF2EC8D
:105030009FF00101AA6FAA513E0A0EE054EC39F02C
:10504000ED0E01012C6F8B0E2B6F2E6B130E2D6F3F
:10505000ACEC04F0199C5ED0A76BA86BA96B37D0A1
:10506000000E0101A725D96EDA6A090EDA222E0E8A
:10507000DF622BD0FE0E556F080E566FA7515527D5
:10508000000E562355C11BF156C11CF1FCEC17F064
:105090001BC19EF11CC19FF1FB0E0101A725D96E1A
:1050A000DA6A080EDA22460EDF6205D00C889EC14D
:1050B00099F19FC19AF101019E51A85D9F51A95993
:1050C00004E29EC1A8F19FC1A9F10101A72B000E26
:1050D0000101A725D96EDA6A090EDA22DF50C0E194
:1050E0000CA853D00F0EA85D000EA95919E254EC7C
:1050F00039F0199CA80E0301BD6FC00EBC6FEF0EF6
:1051000001012C6FFB0E2B6F2E6B100E2D6FACEC74
:1051100004F057D0000119A01200000EE3EF35F0A3
:10512000090E0101226F000E216FFF0E246F420E47
:10513000236FA8C125F1A9C126F186ECCEF0A951B3
:105140009A1902E1A851991908E1F00E176F1D0E86
:10515000166F010E4EEC32F007D0F00E176F8F0E67
:10516000166F010E4EEC32F0090E0101176F000EA2
:10517000166F000E4EEC32F0EC0E0101176FAE0E02
:10518000166F000E4EEC32F053D007B402D011AAC5
:1051900041D00F0E0101A85D000EA95914E254EC94
:1051A00039F0199CA80E0301BD6FC00EBC6FEF0E45
:1051B00001012C6FFB0E2B6F2E6B100E2D6FACECC4
:1051C00004F0119AA7D7090E0101226F000E216F7A
:1051D000FF0E246F420E236FA8C125F1A9C126F14D
:1051E00086ECCEF0F00E176F8F0E166F010E4EECA0
:1051F00032F0090E0101176F000E166F000E4EEC13
:1052000032F0EC0E0101176FAE0E166F000E4EEC71
:1052100032F00ED007B40CD0000111BA09D054EC12
:1052200039F0199CA80E0301BD6FC00EBC6FC00CF5
:10523000119A030E01012A6FE80E296F2BEC37F04B
:10524000880E0101296F130E2A6F000E2B6B2C6B39
:105250002D6BF2EC9FF00101AA6FAA513F0A15E0F5
:1052600054EC39F0EE0E01012C6F110E2B6F2E6BEA
:10527000140E2D6FACEC04F0000119A003D0000E49
:10528000E3EC35F00001199C120054EC39F0030EE8
:1052900001012A6FE80E296F2BEC37F0500E010147
:1052A000186FE70E176F460E196F50EC35F0500E61
:1052B0000101186FE80E176F4C0E196F50EC35F0A6
:1052C000500E0101186FE90E176F530E196F50EC55
:1052D00035F0500E0101186FEA0E176F310E196F7D
:1052E00050EC35F0EC0E01012C6F930E2B6F2E6BF2
:1052F0001A0E2D6FACEC04F0030E01012A6FE80EBC
:10530000296F2BEC37F0F80E0101176FBC0E166FEA
:10531000010E4EEC32F0030E01012A6FE80E296FE8
:105320002BEC37F01284070E0301BF6FD00EBE6F57
:10533000000119A0D00C010EE3EF35F00D9C10D048
:105340000101540506E1FA0E166FCA0E156F090E1B
:105350000CD1FA0E2C6FCA0E2B6F2E6B090E0CD1CE
:1053600052C11DF153C11EF13C0E01011F6F54C10A
:1053700020F113EC36F00101AB6FABC1A9FFA8A27D
:10538000FED71BB8DDD70101AB513A0AE9E19C4BCE
:105390009D2B52C127F153C128F10A0E296F54C128
:1053A0002AF188EC3DF0AB6F1BB8CAD7ABC1A1F1B5
:1053B000A1C1D0F252C127F153C128F10A0E010157
:1053C000296F54C12AF188EC3DF0AB6F1BB8B8D7F8
:1053D0000101AB51566F556B576B5651586F57C102
:1053E000A2F158C1A3F1A46BA56B52C127F153C11F
:1053F00028F10A0E296F54C12AF188EC3DF0AB6FF9
:105400001BB89ED70101AB51A21352C127F153C162
:1054100028F10A0E296F54C12AF188EC3DF09B6FE8
:105420001BB88ED704A892D10101D890A42B000EEE
:10543000A5238CD152C127F153C128F10A0E296F3F
:1054400054C12AF188EC3DF0A06F1BB879D7010157
:10545000A551A211A311A41117E10B0E5225556FEE
:10546000000E5321566F55C11BF156C11CF1FB0EA6
:105470001E6FE40E1D6F206B080E1F6F47EC27F0A8
:105480001C511B1101E00D800101A351040A600EA3
:10549000D8B4A219A411A51117E1090E5225556F10
:1054A000000E5321566F55C11BF156C11CF1FF0E62
:1054B0001E6F330E1D6F206B040E1F6F47EC27F01D
:1054C0001C511B1101E007820101A551800A800FC8
:1054D00008E1010EA45D05E1EC0EA35D02E1010E01
:1054E000A25D01E3188A0101A22B000EA323A423CD
:1054F000A523A1070101A1299DE152C12DF153C1AD
:105500002EF10A0E2F6F54C130F1B2EC35F001E3E9
:1055100004861BB815D724D752C12DF153C12EF1E3
:105520000A0E2F6F54C130F1B2EC35F001E304865E
:105530001BB806D704A610D00101540506E1FB0EE6
:10554000166FC90E156F080E10D0FB0E2C6FC90E0A
:105550002B6F2E6B080E10D00DA011D00101540539
:1055600007E1F90E166F7A0E12D0176FDDEF43F0D8
:10557000F90E2C6F7A0E11D02D6FACEF04F007A24C
:1055800010D00101540506E1F90E166F850E156F56
:105590000A0EEBD7F90E2C6F850E2B6F2E6B0A0EB1
:1055A000EBD718AA10D00101540506E1F10E166FD1
:1055B0001E0E156F0E0ED9D7F10E2C6F1E0E2B6F0F
:1055C0002E6B0E0ED9D70101010E226F590E216FDD
:1055D000EC0E246F160E236F9CC125F19DC126F1A0
:1055E00086ECCEF02151AB6F540515E1010E166F1C
:1055F000590E156FABC117F1DDEC43F0270E010119
:105600009D6F100E9C6F9C07D8A09D0701019D51B6
:105610009C111CE0F8D7010E2C6F590E2B6FABC1FB
:105620002DF12E6BACEC04F0EC0E01012C6F1B0E77
:105630002B6F2E6B1C0E2D6FACEC04F0F80E0101DD
:10564000176FBC0E166F010E4EEC32F00B0E0101FF
:105650002A6FB80E296F2BEC37F0500E0101186F2E
:10566000E70E176F460E196F50EC35F0500E010122
:10567000186FE80E176F4C0E196F50EC35F0500E86
:105680000101186FE90E176F530E196F50EC35F0CA
:10569000500E0101186FEA0E176F300E196F50ECA3
:1056A00035F0130E01012A6F880E296F2BEC37F0AD
:1056B000FF001200A06B0DD052C127F153C128F199
:1056C0000A0E296F54C12AF188EC3DF0A0131BB8D3
:1056D00037D60101A107A129EFE1A051F00B100A73
:1056E00002E1048801D0049852C12DF153C12EF17A
:1056F0000A0E01012F6F54C130F1B2EC35F007D71B
:1057000052C127F153C128F10A0E296F54C12AF161
:1057100088EC3DF0A06F1BB813D60101A107A129A9
:10572000EFE1A0C155F10F0E5517550502E10488B0
:1057300001D0049852C12DF153C12EF10A0E01017E
:105740002F6F54C130F1B2EC35F0E1D601019B511D
:1057500001E1CFD6010A01E1DFD6030AABE0060A78
:10576000DCE0FED50301BF51BE1103E0BE07D8A0A7
:10577000BF070201B351B21103E0B207D8A0B307CB
:1057800004009E90D10ECF6E200ECE260301AE4BAC
:10579000AF2BB64BB72B05010A2B000E0B230C23A6
:1057A0000D230301B24BB32B13A409D01394030EA2
:1057B000216EEE0E206E72EC23F08F80138A0301AF
:1057C000BB51BA1108E0BA07D8A0BB07BB51BA1148
:1057D00002E10201E86B0401EF51EE1103E0EE0774
:1057E000D8A0EF070301A84BA92BA951800A286E66
:1057F000A651A85DA751800A285801E31D8A04011B
:10580000D607D8A0D707D751D61102E110AE119212
:1058100014A20AD00301E02B040EE06505D0E06B72
:105820000001148442EC3CF00301D3670AD00CA0C1
:1058300007BC07D015BA12B004D012B802D08D8AB6
:105840008D9C0301D35119E00201EC5102E0EC07F9
:105850003ED00BBE06D08D9A8D9C0201EC690B8E5A
:1058600036D08D9A8D8C0201EC690B9E0301D30713
:10587000D3672DD08D8A8D9C2AD012A812D0020118
:10588000ED2B270EED6523D0ED6B8D8C8D8A0301FA
:10589000D62BD651050A1BE18D9C8D9AD66B12989A
:1058A00016D00CA007D00201ED2B310EED6502D011
:1058B000ED6B0CD007AC0BD00401F44BF52BE80ECC
:1058C000F45D030EF55903E3F46BF56B8D7A13A8C1
:1058D00008D00301DD2B310EDD6503D0DD6B13989D
:1058E0008F900CA20ED00301E22B310EE26509D09D
:1058F000E26B8F70E12B3B0EE16503D0E16B0C9204
:105900008F900CA410D00301E52B310EE5650BD070
:10591000E56B8F70E42B3B0EE46505D0E46B8F9054
:105920000C941AB40C8413AA08D00301DE2B310E98
:10593000DE6503D0DE6B139A8F900201EB2B1D0EF8
:10594000EB6505D0EB6B0301E76B0201EA6B46B434
:105950000ED20301E32B180EE36509D2E36B0101BC
:10596000E56BB8C323F0B9C324F0FEEC26F00101C7
:10597000E76F14B20AAE06D00201F951E00B010143
:10598000E71905D00101E7510201F9190101E56F9D
:10599000ECC31FF0E551CBEC2EF0296E295001E14C
:1059A0008DD014AE8AD029A015D014A205D0010143
:1059B000E55123EC29F00ED00101E5A106D0206AC3
:1059C000220E1F6E5EEC1BF005D0206A240E1F6EA7
:1059D0005EEC1BF029A215D014A205D00101E551FF
:1059E000A7EC24F00ED00101E5A306D0206A260E14
:1059F0001F6E5EEC1BF005D0206A280E1F6E5EEC59
:105A00001BF029A415D014A205D00101E55164ECC6
:105A100029F00ED00101E5A506D0206A2A0E1F6EDE
:105A20005EEC1BF005D0206A2C0E1F6E5EEC1BF0A6
:105A300029A615D014A205D00101E551E6EC29F004
:105A40000ED00101E5A706D0206A2E0E1F6E5EEC77
:105A50001BF005D0206A300E1F6E5EEC1BF029A8EB
:105A600015D014A205D00101E551A5EC29F00ED006
:105A70000101E5A906D0206A360E1F6E5EEC1BF010
:105A800005D0206A380E1F6E5EEC1BF029AA15D0D7
:105A900014A205D00101E55139EC44F00ED001010A
:105AA000E5AB06D0206A900E1F6E5EEC1BF005D0B1
:105AB000206A920E1F6E5EEC1BF0148EE5C1ECF3B3
:105AC000E5C1E6F115A007D000011590206A400E4F
:105AD0001F6E5EEC1BF007AE07D00001079E206A28
:105AE000320E1F6E5EEC1BF008A007D0000108907C
:105AF000206A340E1F6E5EEC1BF01BA60CD000015A
:105B00001B96206A440E1F6E5EEC1BF013BC03D084
:105B10000FA60FB8128611AC07D00001119C206AA5
:105B20003E0E1F6E5EEC1BF016AC07D00001169CFB
:105B3000206A460E1F6E5EEC1BF00DA807D0000118
:105B40000D98206A880E1F6E5EEC1BF00DA208D027
:105B500000010D92020E206EB40E1F6E5EEC1BF063
:105B60000FA007D000010F90206A8E0E1F6E5EEC12
:105B70001BF00EAE08D000010E9E020E206EB60E77
:105B80001F6E5EEC1BF008AC07D00001089C206A79
:105B9000960E1F6E5EEC1BF014A607D00001149643
:105BA000206A3A0E1F6E5EEC1BF014A807D00001AD
:105BB0001498206A3C0E1F6E5EEC1BF017A607D0EF
:105BC00000011796206A8A0E1F6E5EEC1BF017AE5E
:105BD00007D00001179E206A8C0E1F6E5EEC1BF032
:105BE00017AA08D00001179A020E206EB80E1F6E79
:105BF0005EEC1BF018A208D000011892020E206E75
:105C0000BA0E1F6E5EEC1BF00201CC510AE0DE0EF4
:105C1000CC251F6E206A020E20225EEC1BF00201D2
:105C2000CC6B0AA807D000010A98206A200E1F6ECC
:105C30005EEC1BF00BA607D000010B96206A860EC7
:105C40001F6E5EEC1BF00BA007D000010B90206ACA
:105C5000940E1F6E5EEC1BF0010E05A0000E286E68
:105C6000010E04AE000E281A15E0060E04BE070E43
:105C70000301F86F990EF96FFA6F850EFB6F490EED
:105C8000FC6F900EFD6F050EFE6F168E168C059044
:105C900004BE05800201C76722D014BE0CBA1FD013
:105CA00006A003D006B451D052D006AC03D007B042
:105CB0004CD04DD00DAE03D00EB247D048D00DA47D
:105CC00003D00DBA42D043D008A403D008B83DD0C9
:105CD0003ED01AA604D00201F35137E138D000F0CB
:105CE0000201C86741D0000114AE3ED000010CBCD7
:105CF0003BD006A204D0000106B42FD030D006AEAF
:105D000004D0000107B029D02AD00EA004D0000191
:105D10000EB223D024D00DB614A204D0000106BACE
:105D20001CD01DD00DA604D000010DBA16D017D07E
:105D300008A604D0000108B810D011D000011AA89C
:105D400013D00201F45109E10AD08A8C02D08A9C56
:105D5000C6D7030E0201C76FC2D78A8E02D08A9EB1
:105D600003D0030E0201C86F00F0B7EC3BF012BC89
:105D700002D012AE03D00201DB6B03D0010E020190
:105D8000DB6F0401E24BE32BE051E25DE151E359AB
:105D900034E3E26BE36B0201DB6708D018B403D095
:105DA0008A988A962AD08D968D9427D0DB0525E196
:105DB0001DAE16D01D9E18B408D018B003D08A9816
:105DC0008A860AD08A888A9607D017B803D08D961B
:105DD0008D8402D08D868D940401E16B640E0CD00D
:105DE0001D8E18B403D08A988A9602D08D968D9411
:105DF0001F0E0401E16F400EE06F0401E64BE72B3C
:105E0000E451E65DE551E75960E3E66BE76B04B00A
:105E100002D00301D86B0301D86723D01EA00CD099
:105E20001E9018B403D08D868D9402D08A888A96ED
:105E30000401E56B640E13D01E8018B403D08D9658
:105E40008D9402D08A988A9604B005D0010E040180
:105E5000E56F900E04D0090E0401E56FC40EE46FE7
:105E600034D0D80512E11EA02AD01E9018B403D059
:105E70008D868D9402D08A888A9613BCECD7D8D7A9
:105E80008A988A9613BCD4D7E6D7D851020A0AE179
:105E90001EA015D01E9018B402D08D860CD08A8812
:105EA0008A86EBD7D851030A10E11EA008D01E90B5
:105EB00018B403D08D968D84E0D78A98F1D71E80D0
:105EC00018B4DED78D968D94DDD712A004D08D96B0
:105ED0008D948A988A960401F04BF12BE80EF05DC0
:105EE000030EF15969E30201F351D8A4F307F45109
:105EF000D8A4F4070401F06BF16BE84BE92B000127
:105F000012A033EC17F00301DF0714A206D0020140
:105F1000CD5103E0CD2F01D01B820401FF51D8A445
:105F2000FF070201F851D8A4F80719BC0DD0E151C0
:105F3000E22BE25D02E3E26B15860301CF2B1D0E1F
:105F4000CF6502D0CF6B1A8A1AAC08D0580E040164
:105F5000DA5D020EDB5902E2DA4BDB2B06A60AD031
:105F60000401D951D81103E18A9C069603D0D807C1
:105F7000D8A0D9071BAA09D00401F751F61102E1F4
:105F80001B9A03D0F607D8A0F70714A00AD0040183
:105F9000F351F21103E18A9E149003D0F207D8A0C6
:105FA000F3070201C751D8A4C707C851D8A4C8072E
:105FB0000301D951D8A4D9070401EC4BED2B600E95
:105FC000EC5DEA0EED59D8A01200EC6BED6B03010D
:105FD000BD51BC1103E0BC07D8A0BD07BC05BD1175
:105FE00004E107860301BC6BBD6BE92B14A208D04A
:105FF0000201CA5105E0CA2F03D0099008BE8A9C4D
:106000000101DD510201E62BE65D02E3E66B1B8038
:106010000201DE510301DB2BDB5D02E3DB6B1A8E39
:106020000201CF2B020ECF6501D0CF6B0401EA4BEA
:10603000EB2B0A0EEA5D000EEB591AE3EA6BEB6BF1
:106040000301D22B8F0ED26502D0D26B09880201D8
:10605000F251F12BF15D0CE3F16B1B8618881AA647
:1060600002D0140EF36F1AA803D0140E0201F46FBD
:106070000201E52B020EE565020CE56B0001148AB6
:1060800012000101266B500E01012625D96EDA6A35
:10609000060EDA222651186F196B18BF190790ECFB
:1060A0002EF0DF6E262B2651800A610FECE3266B63
:1060B000000E01012625D96EDA6A050EDA22800E5D
:1060C00090DB90EC2EF0DF6E262B2651800A7A0FA3
:1060D000EFE3196B550E186F90EC2EF00201F26F82
:1060E0000101196B4B0E186F90EC2EF0236F226B91
:1060F000196B4A0E186F90EC2EF022110301B86F45
:10610000010123510301B96F0101196B520E186F80
:1061100090EC2EF00201F96F0101196B560E186F09
:1061200090EC2EF00201D16F0101196B570E186F20
:1061300090EC2EF00301C66F0101196B760E186FFB
:1061400090EC2EF0DC6F196B590E186F90EC2EF05E
:10615000236F226B196B5A0E186F90EC2EF02211E0
:10616000CF6F2351D06F196B4F0E186F90EC2EF03C
:10617000266F1E94010126B51E841E9626B71E8624
:10618000266B85DB9A0E21DB90EC2EF0DF6E7FDB39
:10619000DF5005E0262B2651800A700FF2E3010143
:1061A000266B5DDBBA0E11DB90EC2EF0DF6E57DB59
:1061B000DF5005E0262B2651800A7B0FF2E31E9864
:1061C0000701CB5104E00501FA5101E01E880101ED
:1061D000196B750E186F90EC2EF0266F179C01014D
:1061E00026B1178C199E26B3198E119426B71184E7
:1061F000079426BF0784129226BD12821A9026B5F4
:106200001A800C9A0690069C0D9E0D9408941A967E
:106210000C9C0692069E0E900D9608961A98196B85
:106220004C0E186F90EC2EF0266F266702D00C8A69
:1062300018D026B1FCD726A302D0068012D026A5FE
:1062400002D0068C0ED026A702D00D8E0AD026A929
:1062500002D00D8406D026AB02D0088402D026BD21
:106260001A860101196B4D0E186F90EC2EF0266FF7
:10627000266702D00C8C18D026B1FCD726A302D0FA
:10628000068212D026A502D0068E0ED026A702D0F6
:106290000E800AD026A902D00D8606D026AB02D0E9
:1062A000088602D026BD1A88030E0101196F500E10
:1062B000186F90EC2EF0236F226B030E196F510EA6
:1062C000186F90EC2EF022110201B86F01012351DA
:1062D0000201B96F030E0101196F520E186F90EC95
:1062E0002EF0236F226B030E196F530E186F90EC74
:1062F0002EF022110201BA6F010123510201BB6F7E
:10630000030E0101196F540E186F90EC2EF0236FDD
:10631000226B030E196F550E186F90EC2EF02211A0
:106320000201BC6F010123510201BD6F030E010187
:10633000196F560E186F90EC2EF0236F226B030E20
:10634000196F570E186F90EC2EF022110201BE6FDC
:10635000010123510201BF6F030E0101196F580E95
:10636000186F90EC2EF0236F226B030E196F590EED
:10637000186F90EC2EF022110201C06F0101235121
:106380000201C16FE80EB85D030EB95917E3030EA1
:106390000101186F500E176F030E196F50EC35F096
:1063A000030E0101186F510E176F3E0E196F50EC5E
:1063B00035F0030E0201B96F3E0EB86FE80EBA5DFC
:1063C000030EBB5917E3030E0101186F520E176F2E
:1063D000030E196F50EC35F0030E0101186F530EC8
:1063E000176F3E0E196F50EC35F0030E0201BB6FB4
:1063F0003E0EBA6FE80EBC5D030EBD5917E3030EE7
:106400000101186F540E176F030E196F50EC35F021
:10641000030E0101186F550E176F3E0E196F50ECE9
:1064200035F0030E0201BD6F3E0EBC6FE80EBE5D7F
:10643000030EBF5917E3030E0101186F560E176FB5
:10644000030E196F50EC35F0030E0101186F570E53
:10645000176F3E0E196F50EC35F0030E0201BF6F3F
:106460003E0EBE6FE80EC05D030EC15917E3030E6A
:106470000101186F580E176F030E196F50EC35F0AD
:10648000030E0101186F590E176F3E0E196F50EC75
:1064900035F0030E0201C16F3E0EC06F0101196B92
:1064A0006C0E186F90EC2EF0E16F1C920101E1B7B9
:1064B0001C82070EE117196B680E186F90EC2EF016
:1064C000E26F1C9C0101E2B71C8C070EE217196BEE
:1064D000690E186F90EC2EF0E36F1D920101E3B787
:1064E0001D82070EE317196B6A0E186F90EC2EF0E1
:1064F000E46F1D980101E4B71D88070EE417196BBE
:10650000540E186F90EC2EF0266F2651F00B09E117
:10651000069A199426C122F10F0E01012217222991
:1065200024D02651F00B100A0EE1068A199426C1D8
:1065300022F10F0E010122172229D46F0301AD6B46
:10654000010EAC6F14D02651F00B200A03E1069A1D
:106550001984E0D72651F00B300A03E1068A19842A
:10656000E6D7069A07981994010E0201CB6F1CA278
:106570001CBC04D01DB202D01DA802D0198601D0C7
:1065800019960101196B640E186F90EC2EF0020140
:10659000D56F0101196B650E186F90EC2EF002019A
:1065A000D66F0101196B660E186F90EC2EF0020188
:1065B000D96F0101196B670E186F90EC2EF0020174
:1065C000D26F0101196B6B0E186F90EC2EF0266FD5
:1065D000109E010126B1108E0A9E26B50A8E089ED5
:1065E00014A207D0088E0C9A0690069C0D9E0D945E
:1065F00008940101196B700E186F90EC2EF00201D7
:10660000E16F0101196B720E186F90EC2EF0DD6FC7
:10661000196B710E186F90EC2EF00301D76F01010A
:10662000196B730E186F90EC2EF00201DE6F0101F2
:10663000266BE0D88A0EC9D890EC2EF0DF6EDAD83F
:10664000DF5005E0262B2651800A700FF2E30F98E9
:106650000501D55107E0E0D847EC27F01C511B118C
:1066600001E00F880101266BC5D8CD0EBAD890EC99
:106670002EF0DF6EBFD8DF5005E0262B2651800AB2
:10668000700FF2E30F960501D55107E0C5D847EC2E
:1066900027F01C511B1101E00F860101266BD0D899
:1066A000B30E9FD890EC2EF0DF6ECAD8DF5005E015
:1066B000262B2651800A700FF2E30101266BEFD8DA
:1066C000DD0E8FD890EC2EF0DF6EE9D8DF5005E0BC
:1066D000262B2651800A700FF2E30101256B980EDC
:1066E000246F18A404D0030E256F200E246F01011F
:1066F000266B9FD887D890EC2EF0DF6E9AD8DA22DE
:10670000DF5005E0262B2651800A650FF2E30101D8
:10671000256BED0E246F18A404D0030E256F3B0EDD
:10672000246F0101266B94D86DD890EC2EF0DF6EAB
:106730008FD8DA22DF5005E0262B2651800A770F0A
:10674000F2E30101256BF60E246F18A404D0030EAA
:10675000256F440E246F0101266BA9D853D890EC05
:106760002EF0DF6EA4D8DA22DF5005E0262B26516A
:10677000800A770FF2E30101266B79D8550E25D8F0
:1067800090EC2EF0DF6E73D8DF5005E0262B2651FB
:10679000800A600FF2E30101266B71D8750E15D8DF
:1067A00090EC2EF0DF6E6BD8DF5005E0262B2651E3
:1067B000800A700FF2E3420E0101196F3A0E186F52
:1067C00090EC2EF00201F66F1200226F010E236F83
:1067D00022512625186F000E26BFFF0E2321196FA8
:1067E00012002625186FE86AD8B0E82A26BFE80606
:1067F000196F1200D50E01012625D96EDA6A050E31
:10680000DA221200DA2224512625186F000E26BF44
:10681000FF0E2521196F1200050E01011C6FD50E08
:106820001B6FFC0E1E6FDA0E1D6F206B070E1F6FA5
:10683000070C700E01012625D96EDA6A070E1200C8
:10684000BB0E01012625D96EDA6A070EDA22120084
:10685000DF0E01012625D96EDA6A060E1200FA0E45
:1068600001012625D96EDA6A050EDA221200500ED1
:1068700001012625D96EDA6A070EDA221200AB0E64
:1068800001012625D96EDA6A070EDA221200CB0E34
:1068900001012625D96EDA6A070EDA221200DB0E14
:1068A00001012625D96EDA6A070EDA221200E80EF7
:1068B00001012625D96EDA6A060E1200E8CF95F29C
:1068C000020195050FE1020E0101166F4E0E156FC4
:1068D00036EC3FF00201946F946701D01200E56B33
:1068E000149A28D0946B14D002019451800A400F5E
:1068F00021E21F0E9425D96EDA6A050EDA224E0EB9
:106900009425E16EE26A020EE222DFCFE7FF942BCC
:10691000D3C5B8F10101B96B94C2BAF1BB6BBABF70
:10692000BB07BB51800ABC6FB851BA5DB951800A30
:10693000BC59DAE30201E56B149A950567E1020E92
:1069400001011C6F4E0E1B6FFE0E1E6FC40E1D6FDD
:10695000206B050E1F6F47EC27F01C511B1118E12F
:10696000130E5D6F6A0E5C6F5F6B1E0E5E6F020E24
:106970000101616F4E0E606F95C262F163ECC8F069
:1069800001015D515C1104E10201955142EC41F0BD
:10699000020E01011C6F4E0E1B6FFB0E1E6FDB0EF5
:1069A0001D6F206B080E1F6F47EC27F01C511B1149
:1069B0002DE1130E186F6A0E176F000E196B50EC55
:1069C00035F0130E0101186F790E176F000E196B59
:1069D00050EC35F00101196B750E186F90EC2EF02C
:1069E00002018E6F8E51F70B8F6F0101186B750EC0
:1069F000176F8FC219F150EC35F0F00E0101166FD0
:106A00007F0E156F0F0E176FDDEC43F00201950539
:106A100029E1020E01011C6F4E0E1B6FFE0E1E6F50
:106A2000BE0E1D6F206B050E1F6F47EC27F01C512B
:106A30001B1118E1186BFF0E1769196950EC35F03E
:106A40004F0E0101186FD60E176F000E196B50EC28
:106A500035F0ED0E0101166FA20E156F160E176FB1
:106A6000DDEC43F0020E01011C6F4E0E1B6FFE0E9B
:106A70001E6FB20E1D6F206B050E1F6F47EC27F0C7
:106A80001C511B1149E114A202D006BAB9D24F0E13
:106A90000101196FD30E186F90EC2EF0B86FB8ADDE
:106AA0002BD0020E0101226F4E0E216FF40E246FC7
:106AB0008E0E236F130E266FFA0E256F86ECCEF026
:106AC00021510201946F955109E0020E0101166FE8
:106AD0004E0E156F94C217F1DDEF43F0020E010167
:106AE0002C6F4E0E2B6F0201945101012D6F2E6BF6
:106AF0002DBF2E07ACEF04F0020E0101226F4E0EE7
:106B0000216FF40E246F810E236F130E266FFA0E81
:106B1000256F86ECCEF0D4D7020E01011C6F4E0E0D
:106B20001B6FA2EC1AF01BC192F21CC193F24F0E24
:106B3000196FD50E186F90EC2EF0B86F4F0E196FBD
:106B4000D40E186F90EC2EF00201916F0101B85134
:106B50000201906F530E0101B86F020EB96FB8C1F8
:106B60001BF1B9C11CF1FE0E1E6FA60E1D6F206B2E
:106B7000050E1F6F47EC27F01C511B1121E102018C
:106B80009151931902E19051921901E0C1D04F0E39
:106B90000101196FD30E186F90EC2EF00201946F63
:106BA0003F0E94174F0E0101186FD30E176F94C24A
:106BB00019F150EC35F002019551B0EC41F097D04D
:106BC000530EB86F020EB96FB8C11BF1B9C11CF1F9
:106BD000FE0E1E6FAC0E1D6F206B050E1F6F47EC77
:106BE00027F01C511B1120E102019151931902E180
:106BF0009051921901E08CD04F0E0101196FD30E04
:106C0000186F90EC2EF00201946F948D4F0E0101DD
:106C1000186FD30E176F94C219F150EC35F00201C2
:106C20009551B0EC41F063D0530EB86F020EB96FBE
:106C3000B8C11BF1B9C11CF1FE0E1E6FB80E1D6F5D
:106C4000206B050E1F6F47EC27F01C511B114FE105
:106C500002019451800A720F06E39151931902E1E7
:106C60009051921901E054D00A0E946F4E0E942563
:106C7000D96EDA6A020EDA22DF50800A500F0AE378
:106C80004E0E9425D96EDA6A020EDA22DF50800A9F
:106C9000460F01E33DD0942B9451800A720FE6E336
:106CA0005C6B580E0101B86F020EB96FB8C11BF1D1
:106CB000B9C11CF1A2EC1AF01BC192F21CC193F2F3
:106CC0004F0E186FD40E176F020193510101196F07
:106CD00050EC35F04F0E0101186FD50E176F92C2B0
:106CE00019F150EC35F002019551B0EF41F04F0E23
:106CF0000101196FD30E186F90EC2EF0B86FB8AD7C
:106D00000AD002019151931902E19051921903E0C6
:106D10009551C6EF41F0530E0101B86F020EB96FE5
:106D2000B8C11BF1B9C11CF1FF0E1E6F470E1D6FDC
:106D3000206B040E1F6F47EC27F01C511B1141E123
:106D400046B604D0000113A0C6EC07F001015D6B4C
:106D50005C6B040E5F6F5E6B020E616F4E0E606FB8
:106D600095C262F163ECC8F001015D515C1104E170
:106D70000201955142EC41F0000146B61200010EAD
:106D80000101186F000E176B196B50EC35F0010EF6
:106D90000101186F110E176F000E196B50EC35F0D2
:106DA000010E0101186F220E176F000E196B50ECC7
:106DB00035F0010E0101186F330E176F196B50EF8C
:106DC00035F0530EB86F020EB96FB8C11BF1B9C1DF
:106DD0001CF1FF0E1E6F510E1D6F206B040E1F6FF6
:106DE00047EC27F01C511B1111E1040E5D6F5C6B29
:106DF0000D0E5F6FE80E5E6F020E0101616F4E0EA9
:106E0000606F95C262F163ECC8F06FD0530EB86F3B
:106E1000020EB96FB8C11BF1B9C11CF1FF0E1E6F94
:106E20005B0E1D6F206B040E1F6F47EC27F01C518B
:106E30001B1112E1130E5D6F880E5C6F2E0E5F6FDB
:106E4000B30E5E6F020E0101616F4E0E606F95C250
:106E500062F163ECC8F049D0530EB86F020EB96FFF
:106E6000B8C11BF1B9C11CF1FF0E1E6F380E1D6FAA
:106E7000206B040E1F6F47EC27F01C511B1112E111
:106E8000420E5D6F3B0E5C6F0B0E5F6FB80E5E6F58
:106E9000020E0101616F4E0E606F95C262F163ECEC
:106EA000C8F023D0530EB86F020EB96FB8C11BF1F2
:106EB000B9C11CF1FF0E1E6F560E1D6F206B040E24
:106EC0001F6F47EC27F01C511B1118E1510E5D6F2D
:106ED0005C6B2F0E5F6F5E6B020E0101616F4E0ED9
:106EE000606F95C262F163ECC8F001015D515C1105
:106EF000D8A412000201955142EF41F0530EB86F31
:106F0000020EB96FB8C11BF1B9C11CF1FE0E1E6FA4
:106F1000CA0E1D6F206B050E1F6F47EC27F01C512A
:106F20001B111AE114A202D006BA6AD0020195051B
:106F30000AE0EC0E01012C6FC80E2B6F2E6B180EA1
:106F40002D6FACEF04F0020E0101536F4E0E526F25
:106F500095C254F135EFA6F0530EB86F020EB96F1B
:106F6000B8C11BF1B9C11CF1FB0E1E6FED0E1D6FF8
:106F7000206B080E1F6F47EC27F01C511B1106E118
:106F800014A202D006BA3CD0118EDDD7530EB86FD2
:106F9000020EB96FB8C11BF1B9C11CF1FC0E1E6F16
:106FA000E30E1D6F206B060E1F6F47EC27F01C5180
:106FB0001B1106E114A202D006BA22D0118AC3D74F
:106FC000530EB86F020EB96FB8C11BF1B9C11CF1F5
:106FD000FF0E1E6F4C0E1D6F206B040E1F6F47ECD3
:106FE00027F01C511B1110E114A202D006BA08D0E0
:106FF00001017D6B7C6B040E7F6F7E6B020E20D0D7
:107000000201955158EF41F0530EB86F020EB96F5F
:10701000B8C11BF1B9C11CF1FF0E1E6F600E1D6FD0
:10702000206B040E1F6F47EC27F01C511B110FE162
:10703000130E7D6F880E7C6F2E0E7F6FB30E23D0E4
:10704000816F4E0E806F95C282F182EFD0F0530EA9
:10705000B86F020EB96FB8C11BF1B9C11CF1FF0EB8
:107060001E6F3D0E1D6F206B040E1F6F47EC27F047
:107070001C511B11D8A41200420E7D6F3B0E7C6F79
:107080000B0E7F6FB80E7E6F020E0101D9D7E8CFCD
:107090003CF10101446B010E436F96DB3A6F3A39C4
:1070A0000F0B5BEC43F0DF6E442B8EDB0F0B5BECC6
:1070B00043F0DF6E442B432B020E4365EED73D0EAB
:1070C0004425D96EDA6A010EDA22DF6A3CC144F146
:1070D000C451310A0CE170DBF20E246F1D0E236FD8
:1070E000010E266F3D0E256F86ECCEF049D3C451BC
:1070F000910A0CE161DBF20E246F2C0E236F010E5E
:10710000266F3D0E256F86ECCEF03AD3C451320A7D
:107110000CE152DBF20E246F860E236F010E266FF8
:107120003D0E256F86ECCEF02BD3C451920A0CE1B4
:1071300043DBF20E246F950E236F010E266F3D0E7A
:10714000256F86ECCEF01CD3C451330A0CE134DB3E
:10715000F20E246FEF0E236F010E266F3D0E256F8A
:1071600086ECCEF00DD3C451930A0CE125DBF20E70
:10717000246FFE0E236F010E266F3D0E256F86ECE9
:10718000CEF0FED2C451340A0CE116DBF30E246FAC
:107190001C0E236F010E266F3D0E256F86ECCEF080
:1071A000EFD2C451940A0CE107DBF30E246F2B0ECF
:1071B000236F010E266F3D0E256F86ECCEF0E0D2D8
:1071C000C451990A0CE1F8DAF30E246F490E236FCB
:1071D000010E266F3D0E256F86ECCEF0D1D2C45144
:1071E000390A0CE1E9DAF30E246F580E236F010E11
:1071F000266F3D0E256F86ECCEF0C2D2C451890AAF
:107200000CE1DADAF30E246F670E236F010E266F9E
:107210003D0E256F86ECCEF0B3D2C451900A0CE13E
:10722000CBDAF30E246F760E236F010E266F3D0E20
:10723000256F86ECCEF0A4D2C451980A0CE1BCDADA
:10724000F10E246FD20E236F010E266F3D0E256FB7
:1072500086ECCEF095D2C451350A0CE1ADDAF10ED0
:10726000246F870E236F010E266F3D0E256F86EC6F
:10727000CEF086D2C451950A0CE19EDAF10E246F4D
:10728000960E236F010E266F3D0E256F86ECCEF015
:1072900077D2C451960A0CE18FDAF10E246FA50E55
:1072A000236F010E266F3D0E256F86ECCEF068D25F
:1072B000C451380A0CE180DAF10E246FC30E236F3B
:1072C000010E266F3D0E256F86ECCEF059D2C451CB
:1072D000710A0CE171DAF10E246FB40E236F010E06
:1072E000266F3D0E256F86ECCEF04AD2C451850A3A
:1072F0000CE162DAF20E246F590E236F010E266F35
:107300003D0E256F86ECCEF03BD2C451880A0CE1CD
:1073100053DAF20E246FC20E236F010E266F3D0E5C
:10732000256F86ECCEF02CD2C451460A0CE144DA2B
:10733000F30E246F0D0E236F010E266F3D0E256F89
:1073400086ECCEF01DD2C451450A0CE135DAF30EBD
:10735000246F3A0E236F010E266F3D0E256F86ECCB
:10736000CEF00ED2C451030A05E126DA44DA86ECE7
:10737000CEF006D2C451050A05E11EDA3CDA86ECED
:10738000CEF0FED1C451040A0CE116DAF20E246FDD
:107390004A0E236F010E266F3D0E256F86ECCEF050
:1073A000EFD1C451060A05E107DA1CDA86ECCEF00B
:1073B000E7D1C451080A05E1FFD914DA86ECCEF012
:1073C000DFD1C451070A0CE1F7D9F20E246FB30ED6
:1073D000236F010E266F3D0E256F86ECCEF0D0D1C7
:1073E000C451360A0CE1E8D9F10E246FFF0E236F69
:1073F000010E266F3D0E256F86ECCEF0C1D1C45133
:10740000370A0CE1D9D9F20E246F0E0E236F010E4C
:10741000266F3D0E256F86ECCEF0B2D1C451990A8D
:107420000CE1CAD9F10E246F4B0E236F010E266FAB
:107430003D0E256F86ECCEF0A3D1C451390A0CE184
:10744000BBD9F10E246F5A0E236F010E266F3D0E2D
:10745000256F86ECCEF094D1C46712D01F0E0101C7
:107460004425216F226B050E2223F10E246FE10EBD
:10747000236F010E266F3D0E256F86ECCEF080D176
:10748000C451780A0CE198D9F10E246FF00E236FE5
:10749000010E266F3D0E256F86ECCEF071D1C451E2
:1074A000700A0CE189D9F10E246F780E236F010E5A
:1074B000266F3D0E256F86ECCEF062D1C451400A96
:1074C0000CE17AD9F20E246F680E236F010E266F3D
:1074D0003D0E256F86ECCEF053D1C451410A0CE12C
:1074E0006BD9F20E246FD10E236F010E266F3D0E65
:1074F000256F86ECCEF044D1C451420A0CE15CD930
:10750000F20E246F770E236F010E266F3D0E256F4E
:1075100086ECCEF035D1C451430A0CE14DD9F20EC0
:10752000246FE00E236F010E266F3D0E256F86EC53
:10753000CEF026D121EEC4F09F0EDF642DD0B00E28
:10754000C4612AD0C451610F426F0A0E426115D046
:107550001F0E01014425216F226B050E2223F00E20
:10756000246FBF0E236F010E266F3D0E256F42C1A3
:1075700027F1286B86ECCEF003D11ED9F30E246FD1
:10758000940E236F010E266F3D0E256F42C127F129
:10759000286B86ECCEF0F4D021EEC4F0AF0EDF64A1
:1075A0002DD0C00EC4612AD0C451510F426F0A0EB3
:1075B000426115D01F0E01014425216F226B050E7B
:1075C0002223F00E246FAF0E236F010E266F3D0EA7
:1075D000256F42C127F1286B86ECCEF0D1D0ECD8D4
:1075E000F30E246F850E236F010E266F3D0E256F5F
:1075F00042C127F1286B86ECCEF0C2D021EEC4F058
:10760000CF0EDF642DD0E00EC4612AD0C451310FFB
:10761000426F0A0E426115D01F0E01014425216FF1
:10762000226B050E2223F00E246FDF0E236F010E56
:10763000266F3D0E256F42C127F1286B86ECCEF0F8
:107640009FD0BAD8F30E246FB20E236F010E266FAF
:107650003D0E256F42C127F1286B86ECCEF090D00D
:1076600021EEC4F0DF0EDF642DD0F00EC4612AD00D
:10767000C451210F426F0A0E426115D01F0E010145
:107680004425216F226B050E2223F00E246FCF0EAE
:10769000236F010E266F3D0E256F42C127F1286B27
:1076A00086ECCEF06DD088D8F30E246FA30E236F36
:1076B000010E266F3D0E256F42C127F1286B86EC27
:1076C000CEF05ED021EEC4F0BF0EDF642DD0D00E20
:1076D000C4612AD0C451410F426F0A0E426115D0D5
:1076E0001F0E01014425216F226B050E2223F00E8F
:1076F000246FEF0E236F010E266F3D0E256F42C1E2
:1077000027F1286B86ECCEF03BD056D8F30E246FD1
:10771000C10E236F010E266F3D0E256F42C127F16A
:10772000286B86ECCEF02CD0C451230A1EE0C45145
:10773000240A1BE0C451250A18E0C451260A15E0AA
:10774000C451270A12E0C451280A0FE0C451300A7C
:107750000CE0C451150A09E0C451790A06E0C4518D
:10776000840A03E0C451830A0DE126D8F10E246F88
:10777000690E236F010E266F3D0E256F86ECCEF04D
:107780002151436F43513C25C6ECEFF01F0E010120
:107790003A6F050E3B6F3C513A27000E3B23435195
:1077A0003A27000E3B230E0E3A25D96E000E3B21E0
:1077B000DA6EDF6A94EF20F01F0E01014425216F7D
:1077C000226B050E222312003D0E4425D96EDA6A83
:1077D000010EDA22C10E4325E16EE26A010EE222B9
:1077E000E7501200F20E246FA40E236F010E266FD5
:1077F0003D0E256F1200F20E246F3B0E236F010E1B
:10780000266F3D0E256F1200E8CF3BF1460E0601B4
:10781000C16F01013B51310A0FE1FCDAD8B4B8194C
:1078200002E0E3DA12D0060E0101226FC10E216FD1
:10783000F70E246F480E59D13B51910A16E1EADA4E
:10784000D8B4B81909E0060ED9DA236FB8C225F109
:10785000B9C226F186EFCEF0060E0101226FC10EED
:10786000216FF70E246F540E40D13B51320A0FE1C5
:10787000D5DAD8B4BA1902E0B8DA12D0060E01018E
:10788000226FC10E216FF70E246F9C0E2ED13B513B
:10789000920A16E1C3DAD8B4BA1909E0060EAEDAD4
:1078A000236FBAC225F1BBC226F186EFCEF0060ED9
:1078B0000101226FC10E216FF70E246FA80E15D1A2
:1078C0003B51330A0FE1B2DAD8B4BC1902E08DDAC9
:1078D00012D0060E0101226FC10E216FF70E246F28
:1078E000F00E03D13B51930A16E1A0DAD8B4BC19CB
:1078F00009E0060E83DA236FBCC225F1BDC226F172
:1079000086EFCEF0060E0101226FC10E216FF70E39
:10791000246FFC0EEAD03B51340A0FE183DAD8B46D
:10792000BE1902E062DA12D0060E0101226FC10E0A
:10793000216FF80E246F140ED8D03B51940A16E133
:1079400071DAD8B4BE1909E0060E58DA236FBEC248
:1079500025F1BFC226F186EFCEF0060E0101226F9F
:10796000C10E216FF80E246F200EBFD03B51990A33
:107970000FE14CDAD8B4C01902E037DA12D0060EA3
:107980000101226FC10E216FF80E246F380EADD0A9
:107990003B51390A16E13ADAD8B4C01909E0060EAB
:1079A0002DDA236FC0C225F1C1C226F186EFCEF0D9
:1079B000060E0101226FC10E216FF80E246F440ED6
:1079C00094D03B51890A09E1060E0101226FC10ED4
:1079D000216FF80E246F500E88D03B51900A09E1B8
:1079E000060E0101226FC10E216FF80E246F5C0E8E
:1079F0007CD03B51980A09E1060E0101226FC10EAD
:107A0000216FF70E246F0C0E70D03B51350A09E13F
:107A1000060E0101226FC10E216FF60E246FD00EEB
:107A200064D03B51950A09E1060E0101226FC10E97
:107A3000216FF60E246FDC0E58D03B51960A09E1F7
:107A4000060E0101226FC10E216FF60E246FE80EA3
:107A50004CD03B51380A09E1060E0101226FC10EDC
:107A6000216FF70E246F000E40D03B51710A09E1DF
:107A7000060E0101226FC10E216FF60E246FF40E67
:107A800034D03B51850A09E1060E0101226FC10E77
:107A9000216FF70E246F780E28D03B51880A09E138
:107AA000060E0101226FC10E216FF70E246FCC0E5E
:107AB0001CD03B51460A09E1060E0101226FC10E9E
:107AC000216FF80E246F080E10D03B51450A09E1D2
:107AD000060E0101226FC10E216FF80E246F2C0ECD
:107AE00004D03B51030A04E106D0236F86EFCEF0A9
:107AF0003B51050A09E1060E0101226FC10E216FFB
:107B0000F70E246F600EF1D73B51040A09E1060E0F
:107B10000101226FC10E216FF70E246F6C0EE5D7A5
:107B20003B51060A01E103D03B51080A09E1060E68
:107B30000101226FC10E216FF70E246FB40ED5D74D
:107B40003B51070A09E1060E0101226FC10E216FA8
:107B5000F70E246FC00EC9D73B51360A09E1060E55
:107B60000101226FC10E216FF70E246F300EBDD7B9
:107B70003B51370A09E1060E0101226FC10E216F48
:107B8000F70E246F3C0EB1D73B51990A09E1060E5E
:107B90000101226FC10E216FF60E246FA00EA5D732
:107BA0003B51390A09E1060E0101226FC10E216F16
:107BB000F60E246FAC0E99D73B6709D0060E010173
:107BC000226FC10E216FF70E246F180E8ED73B5116
:107BD000780A09E1060E0101226FC10E216FF70E2E
:107BE000246F240E82D73B51700A09E1060E010171
:107BF000226FC10E216FF60E246FC40E76D73B5153
:107C0000400A09E1060E0101226FC10E216FF70E35
:107C1000246F840E6AD73B51410A09E1060E010127
:107C2000226FC10E216FF70E246FD80E5ED73B5125
:107C3000420A09E1060E0101226FC10E216FF70E03
:107C4000246F900E52D73B51430A09E1060E010101
:107C5000226FC10E216FF70E246FE40E46D79F0EE0
:107C60003B651BD0B00E3B6118D03B51610F3A6FA2
:107C70000A0E3A6109D0060E0101226FC10E216F72
:107C8000F40E246FF60E80D0060E0101226FC10E95
:107C9000216FF80E246F800E77D0AF0E3B651BD09E
:107CA000C00E3B6118D03B51510F3A6F0A0E3A613A
:107CB00009D0060E0101226FC10E216FF40E246F50
:107CC000E90E62D0060E0101226FC10E216FF80E7F
:107CD000246F740E59D0CF0E3B651BD0E00E3B6174
:107CE00018D03B51310F3A6F0A0E3A6109D0060E97
:107CF0000101226FC10E216FF50E246F100E44D0CA
:107D0000060E0101226FC10E216FF80E246F980E2E
:107D10003BD0DF0E3B651BD0F00E3B6118D03B51D2
:107D2000210F3A6F0A0E3A6109D0060E0101226F47
:107D3000C10E216FF50E246F030E26D0060E010131
:107D4000226FC10E216FF80E246F8C0E1DD0BF0E56
:107D50003B6520D0D00E3B611DD03B51410F3A6FA7
:107D60000A0E3A6109D0060E0101226FC10E216F81
:107D7000F50E246F1D0E08D0060E0101226FC10EF4
:107D8000216FF80E246FA40E236F3AC125F1266BE4
:107D900086EFCEF03B51230A1FE03B51240A1CE042
:107DA0003B51250A19E03B51260A16E03B51270AB0
:107DB00013E03B51280A10E03B51300A0DE03B51E3
:107DC000150A0AE03B51790A07E03B51840A04E0B6
:107DD0003B51830AD8A41200060E0101226FC10E86
:107DE000216FF60E246FB80E80D6060E0101226FA9
:107DF000C10E216FF40E246FCF0E12000101226F0D
:107E0000C10E216FF40E246FDC0E12000201C1516D
:107E1000030A3E0C0201B951030A3E0C0201BB5198
:107E2000030A3E0C0201BF51030A3E0C0201BD5180
:107E3000030A3E0C20EE01F02651D9262751DA2202
:107E4000DF50286F26C1D9FF27C1DAFFDF502D6F21
:107E500028512C6F090E2C5D000E2D5919E3290EA7
:107E60002C5D000E2D5914E220EE04F022DA130EE0
:107E7000DF6E26C1D9FF27C1DAFFDF6A0CDAF80FFF
:107E8000DF6E26C11EF127C11FF137EC1EF001D2B3
:107E9000290E2C5D000E2D590AE3490E2C5D000EB3
:107EA0002D5905E227DA43DAF6D9D80FE9D7560E6D
:107EB0002C5D000E2D5913E3760E2C5D000E2D590E
:107EC0000EE220EE04F0F5D9380EDF6E26C1D9FFA0
